:100000000C94C4080C94E3080C94E3080C94730952
:100010000C94A9090C94E3080C94E3080C94E308ED
:100020000C94E3080C94E3080C94E3080C94E308A4
:100030000C94E3080C94E3080C94E3080C94C90CAA
:100040000C94E3080C94E3080C94E3080C94E30884
:100050000C948F670C94405F0C94E3080C94E308B5
:100060000C94E3080C9415600C94E3080C9409605C
:100070000C94E3080C94E3080C94E3080C94E30854
:100080000C94C2720C94E3080C94E3080C94E308FB
:100090000C9453600C94E3080C9447600C94E308B0
:1000A0000C94E3080C94E3080C94E3080C94E30824
:1000B0000C94E3080C94E3080C94E3080C94E30814
:1000C0000C94E3080C94E3080C94E3080C94E30804
:1000D0000C94E3080C94E3080C94E3080C94E308F4
:1000E0000C94E3080C9448670C9452670C943E6798
:1000F0000C94FE660C9483670C9474670C94686788
:100100000C945C670C94E3080C94E3080C94E308EB
:100110000C94E3080C94E3080C94E3080C94E308B3
:10012000FB7B1A7C997C887DA87DC87DD07D7D7DF8
:10013000084AD73B3BCE016E84BCBFFDC12F3D6C4E
:1001400074319ABD56833DDA3D00C77F11BED9E4B4
:10015000BB4C3E916BAAAABE000000803F076342E1
:1001600036B79BD8A71A39685618AEBAAB558C1D4E
:100170003CB7CC5763BD6DEDFD753EF6177231BFD0
:10018000000000803F08000000BE922449123EABF0
:10019000AAAA2ABECDCCCC4C3E00000080BEABAAA1
:1001A000AAAA3E00000000BF000000803F0000003F
:1001B0000000084178D3BB4387D1133D190E3CC3DF
:1001C000BD4282AD2B3E68EC8276BED98FE1A93E5E
:1001D0004C80EFFFBE01C4FF7F3F00000000002500
:1001E000730A005854414C5F5452494D3D256400F8
:1001F00025730A0025730A00546573742036202580
:10020000730A005465737420352025730A00546501
:10021000737420342025730A0054657374203320CE
:1002200025730A005465737420322025730A005424
:1002300065737420312025730A006368616E3D2563
:10024000640A0074787077723D25640A0035303096
:100250006B0A003235306B0A003131356B0A0035DC
:10026000366B0A0033386B0A0025730A0025730ABF
:100270000073656E743D252D75206475703D252DC8
:10028000752069676E6F7265643D252D75207474E5
:100290006C5F7A65726F3D252D750A0025372E3308
:1002A000662025372E33660025352E326620004520
:1002B00072726F72203020566F6C74004E6F742013
:1002C000737570706F727465640A004572726F7234
:1002D000203020566F6C74004572726F722030208F
:1002E000566F6C740025630074746C3D252D64207A
:1002F0000074746C3D252D6420004E657720747465
:100300006C3D252D6420002563004D533536313179
:1003100020503D252D372E326620252D372E326672
:100320006D0A00424D5030383520256C64205061F4
:100330002020252D372E32666D00256300545F483E
:100340004541545F4944583D252D352E32662000E5
:10035000545F4445573D252D352E326620004148D7
:100360003D252D352E32662000545F5348543258B7
:100370003D252D352E3266200052485F53485432B9
:10038000583D252D352E32662000545F52483D25BC
:100390002D342E3166200052483D252D342E3166F5
:1003A0002000256300256300256300256300256385
:1003B000007265706F72745F616C6C3D0072657085
:1003C0006F72743D0025630025630025630025637B
:1003D00000204F534343414C3D2564200020467587
:1003E00073653A2065653D253032782068663D2585
:1003F000303278206C663D25303278206C623D25A5
:10040000303278004D43553D2530366C78002563F9
:100410000074785F6C656E3D252D6C752C6C6F7764
:100420005F766F6C746167653D252D6C750A0025DC
:1004300063004F4B0A0025630025630025630025F8
:1004400063002563002563002563006465627567AA
:100450005F616C6C3D0064656275673D0064656258
:1004600075673D0025730A00646565700A006E6F4C
:100470006E650A00707772733D00696E74725F7307
:1004800065635F70313D252D372E33660A00696E36
:1004900074725F70313D252D6C640A00696E747250
:1004A0005F7365635F70303D252D372E33660A001C
:1004B000696E74725F70303D252D6C640A00765F42
:1004C0006D63753D252D352E32660A00745F6D63B0
:1004D000753D252D352E32660A00707077723D25E8
:1004E000730A0064656275673D0072636D643D2543
:1004F000730A0025730A006175746F0A006C6F67D8
:100500005F6D6F64653D007573625F7077723D2546
:10051000730A0072656C61793D25730A0074746C0E
:100520003D252D640A0052494D455F616464723D6A
:10053000252D642E252D640A006E65696768626F3B
:10054000725F7461626C655F73697A653D25640AE8
:10055000006C6F775F766F6C746167653D252D3336
:100560002E32660A00747870773D25640A0063684D
:10057000616E3D25640A006932633D0069643D0097
:100580007478743D25730A0053797374656D205334
:10059000756D6D6172790A006D61736B3D002C00A1
:1005A000696E74657276616C3D252D750023252D6D
:1005B000642C00745F686561745F69647800745FBF
:1005C00064657700616800705F6D733536313100A6
:1005D00072685F736874327800745F73687432781D
:1005E0000070610070006164340061643300616414
:1005F00032006164310061330061320061310076A4
:100600005F696E00726800757074696D65007031A5
:100610005F6C73740070315F740070310070305F14
:100620006C73740070305F7400703000765F6D63BF
:100630007500745F6D637500743100740069640047
:1006400065363400747874002D002B006175746F6A
:10065000006E6F6E6500706F7765725F73617665AF
:100660005F6C656472790072656C61795F6C65645A
:100670007900636F6D7061737300616363656C0013
:100680007072657300705F707772006165730070DF
:10069000315F6C6564790070305F6C656472006511
:1006A00076656E74006C6564006F7700706B740023
:1006B00074785F6C6564790072785F6C6564720051
:1006C0006F706572006E6F6E65002530327800764F
:1006D0005F6164343D252D382E3666002000765F3C
:1006E0006164333D252D382E3666002000765F612B
:1006F00064323D252D382E3666002000765F616419
:10070000313D252D382E3666002000765F6C6967F6
:1007100068743D252D382E3666002000765F6132E4
:100720003D252D372E3366002000765F61313D2553
:100730002D372E3366002000765F696E3D252D35FE
:100740002E326600204E657665722D7573656420C5
:10075000737461636B203E20256420627974657335
:100760000A00757074696D653D252D642D6461798D
:10077000732D253032643A253032643A25303264A4
:100780002D686F7572730A0074657374205B6F66F1
:10079000667C317C327C337C347C355D20202020AB
:1007A000202020202D2074657374206D6F64657384
:1007B0000A0D007478205B706B74207061796C6F27
:1007C00061645D2020202020202020202020202D5A
:1007D0002073656E6420726164696F20706B742091
:1007E0006B6579626F6172640A0D00776474205BD7
:1007F0006F6E7C6F66667C746573745D202020204C
:10080000202020202020202D207761746368646FD1
:10081000670A0D007570677220202020202020209C
:1008200020202020202020202020202020202020C8
:100830002D207265626F6F742076696120626F6F20
:10084000746C6F616465720A0D0075617274205B6F
:1008500033386B7C35366B7C3131356B7C323530DF
:100860006B7C3530306B5D202D2073657420746592
:10087000726D2F756172742073706565640A0D0066
:10088000626F6F7420202020202020202020202034
:100890002020202020202020202020202D207265B4
:1008A000626F6F740A0D0070777273205B64656508
:1008B000707C6E6F6E655D2020202020202020201F
:1008C0002020202D206D637520736C656570206D70
:1008D0006F64650A0D007265737420656570726FD0
:1008E0006D202020202020202020202020202020BB
:1008F00020202D20726573746F726520656570729B
:100900006F6D0A0D0070707772205B6F6E7C6F6682
:10091000665D202020202020202020202020202054
:10092000202D2070726F6772616D6D61626C652041
:100930007077720A0D00747874205B737472696E3C
:10094000675D202020202020202020202020202023
:1009500020202D20536574207265706F727420748E
:1009600065787420737472696E670A0D007478700C
:1009700077205B31352D305D202020202020202065
:100980002020202020202020202D20545820507767
:10099000722E20486967686573742030202833649C
:1009A000426D290A0D0074746C205B302D31355D69
:1009B0002020202020202020202020202020202037
:1009C00020202D2074696D652D746F2D6C697665FE
:1009D00020666F72207061636B6574730A0D00731B
:1009E00073202020202020202020202020202020B4
:1009F00020202020202020202020202D20737973EB
:100A000074656D2073756D6D6172790A0D00727376
:100A100020202020202020202020202020202020D6
:100A2000202020202020202020202D207261646999
:100A30006F2073746174730A0D007269205B236EFA
:100A40005D205B696E745D20202020202020202006
:100A50002020202020202D207265706F7274206964
:100A60006E74657276616C0A0D0072636D64205B52
:100A70006F6E7C6F66665D20202020202020202065
:100A80002020202020202D20616C6C6F7720636D4A
:100A9000642066726F6D206E65746F726B0A0D0054
:100AA0007265205B236E5D205B2B7C2D5D205B6D72
:100AB00061736B7C6175746F2C6D61736B5D202D40
:100AC000206D6F7465207265706F72742073657429
:100AD0002F6D6F646966790A0D006F7720202020E2
:100AE0002020202020202020202020202020202006
:100AF0002020202020202D206F6E652D77697265C3
:100B00002073656E736F72730A0D006C6F67205BE4
:100B10006175746F7C6F6E7C6F66665D202020202F
:100B2000202020202020202D206D6F7465732064EC
:100B3000617461206F6E205553420A0D006E65206E
:100B40005B666C7573685D202020202020202020AB
:100B50002020202020202020202D206E656967681D
:100B6000626F72207461626C650A0D00657272209A
:100B70002020202020202020202020202020202075
:100B800020202020202020202D206572726F7220CE
:100B900073746174730A0D006D637520202020202A
:100BA0002020202020202020202020202020202045
:100BB000202020202D206D637520696E666F0A0D40
:100BC000006964205B72657365745D2020202020BD
:100BD000202020202020202020202020202D2069BF
:100BE000642068616E646C696E670A0D0068756DDB
:100BF00020202020202020202020202020202020F5
:100C00002020202020202020202D2068756D696460
:100C10006974792073656E736F720A0D0072656C6A
:100C20006179205B6F6E7C6F66667C737461747330
:100C30005D20202020202020202D2072656C6179ED
:100C4000206E6574776F726B207265706F7274734B
:100C50000A0D006465205B6D61736B5D20202020B0
:100C60002020202020202020202020202020202D77
:100C70002064656275670A0D006368616E205B31F0
:100C8000312D32365D2020202020202020202020E1
:100C900020202020202D206368616E2031312D32EC
:100CA000362028322E3430352D32343830204D68FD
:100CB0007A290A0D0063616C69205B5B765F696E5F
:100CC0007C61317C61325D20766F6C747C726573FF
:100CD00065747C6E6F6E655D202D2063616C69624A
:100CE000726174650A0D0061646320202020202059
:100CF00020202020202020202020202020202020F4
:100D00002020202D2073686F7720765F696E2C205D
:100D100061312C20613220766F6C74616765730AD3
:100D20000D007520202020202020202020202020A1
:100D300020202020202020202020202020202D20A6
:100D4000757074696D650A0D0076202020202020C2
:100D50002020202020202020202020202020202093
:100D600020202020202D2076657273696F6E0A0D79
:100D7000006820202020202020202020202020204B
:100D8000202020202020202020202020202D20680E
:100D9000656C700A0D00256300756E6B6E6F776E63
:100DA00020636D640A00484D43353838330025739D
:100DB00000257300202573002025362E3266200082
:100DC000253032780074656D705F65787465726E79
:100DD0003D252D362E326600202573002025362E27
:100DE0003266204F6E2D426F61726400253032787A
:100DF0000074656D705F626F6172643D252D362EE3
:100E00003266000A00503A20256C64205061202090
:100E1000252D372E3266206D0A00256300256300DC
:100E20004932433A2000452025642E256420636C16
:100E30006F636B20256C752063707520256C7520A1
:100E40006C706D20256C752069727120256C752081
:100E5000676C656420256C7520796C656420256C51
:100E60007520726C656420256C7520747820256C63
:100E700075206C697374656E20256C752073656EC2
:100E8000736F727320256C752073657269616C20B5
:100E9000256C750A00532025642E256420636C6F31
:100EA000636B20256C7520747820256C7520727812
:100EB00020256C752072747820256C7520727278EC
:100EC00020256C75207265786D697420256C7520FD
:100ED00061636B747820256C75206E6F61636B7431
:100EE0007820256C752061636B727820256C7520E5
:100EF00074696D65646F757420256C75206261641A
:100F000061636B727820256C7520746F6F6C6F6EE7
:100F10006720256C7520746F6F73686F727420255D
:100F20006C752062616473796E636820256C75202E
:100F300062616463726320256C7520636F6E7465F3
:100F40006E74696F6E64726F7020256C75207365A6
:100F50006E64696E6764726F7020256C75206C6CAE
:100F6000747820256C75206C6C727820256C750A5D
:100F700000257325730A004F6E6C696E650A000ABE
:100F8000002C20636865636B207261746520257591
:100F900020487A0025732025732C206368616E6ECB
:100FA000656C20257520706F776572202575000AA5
:100FB0000025783A004D4143206164647265737383
:100FC000200052616E646F6D2045554936342061B2
:100FD0006464726573732067656E657261746564BD
:100FE0000A000A2A2A2A2A2A2A2A426F6F74696E5C
:100FF000672025732A2A2A2A2A2A2A0A00454550C8
:10100000524F4D20697320636F72727570742C207B
:10101000726577726974696E672077697468206495
:10102000656661756C74732E0A006C6F63616C6821
:101030006F73740041544D454741313238726661D7
:101040003100020000FFFE0000016E616E00696E5B
:10105000660000407A10F35A00A0724E1809001082
:10106000A5D4E80000E87648170000E40B5402001D
:1010700000CA9A3B000000E1F50500008096980048
:10108000000040420F000000A08601000000102771
:1010900000000000E8030000000064000000000001
:1010A0000A00000000000100000000002C76D88833
:1010B000DC674F0823DFC1DFAE59E1B1B796E5E346
:1010C000E453C63AE651997696E8E6C28426EB895F
:1010D0008C9B62ED407C6FFCEFBC9C9F40F2BAA5FC
:1010E0006FA5F490055A2AF75C936B6CF9676DC194
:1010F0001BFCE0E40D47FEF520E6B500D0ED902E98
:101100000300943577050080841E080000204E0AF5
:10111000000000C80C333333330F986E1283114133
:10112000EF8D2114893BE65516CFFEE6DB18D184FE
:101130004B381BF77C1D901DA4BBE4242032847225
:101140005E228100C9F124ECA1E53D274E414E49C4
:101150004E495459494E46CDCCCC3D0AD7233C1775
:10116000B7D13877CC2B329595E6241FB14F0A00C2
:101170000020410000C84200401C4620BCBE4CCAB2
:101180001B0E5AAEC59D740011241FBECFEFD1E4D3
:10119000DEBFCDBF19E0A0E0B2E0EEE7F1E201E092
:1011A0000BBF02C007900D92A636B107D9F711E325
:1011B000A6E6B9E001C01D92A731B107E1F70E9490
:1011C0009F7E0C94BD900C94000084E794E09F9364
:1011D0008F930E94968D80915402909155020F90AA
:1011E0000F9093FF03C08EE694E002C088E694E07F
:1011F0009F938F930E94968D0F900F900895E0918A
:101200001F1BEF71F0E0EC58F44E808380911F1BA0
:101210008F5F80931F1B8091512888608093512895
:101220004EE352E061E1CA010E942F4F80E090E05E
:101230000895CF93DF93EC0180916D0990916E0931
:1012400086FF1DC08E811F928F938D811F928F9379
:101250008C811F928F938B811F928F938A811F9213
:101260008F9389E593E09F938F930E94848D8DB730
:101270009EB70C960FB6F8949EBF0FBE8DBFBE01F1
:1012800084EA99E00E946150BE0184E092E0DF911F
:10129000CF910C94D64F87EE93E08115910511F014
:1012A0000197F1F708958823B9F052985A981DBA1A
:1012B00080916900806280936900EA9A53985B98F4
:1012C000EB9A809169008068809369008091680042
:1012D0008160809368000895109269005A9AEA9894
:1012E0005B9AEB9808951F920F920FB60F921124FC
:1012F0008F939F93AF93BF938091680080FF20C02E
:1013000080912C2890912D28A0912E28B0912F28E3
:101310000196A11DB11D80932C2890932D28A09398
:101320002E28B0932F2880916D0990916E0987FF28
:1013300007C0749882E090E090937B0280937A02D9
:10134000BF91AF919F918F910F900FBE0F901F9003
:1013500018951F920F920FB60F9211248F939F939F
:10136000AF93BF938091680080FF20C080913028A8
:1013700090913128A0913228B09133280196A11D77
:10138000B11D8093302890933128A0933228B093D8
:10139000332880916D0990916E0990FF07C0739872
:1013A00082E090E090937B0280937A02BF91AF91AC
:1013B0009F918F910F900FBE0F901F901895809363
:1013C0007C0080917B00877F80937B0080917C00F4
:1013D000806C80937C0085E080937A0080917A0015
:1013E000806880937A0080917B0087FFFCCF80919A
:1013F0007B0085FFFCCF80917A00806480937A0027
:1014000080917A0086FDFCCF1092790010927800CE
:1014100084E090E060E070E020917A002064209306
:101420007A0020917A0026FDFCCF2091780030913F
:101430007900620F731F0197009771F710927C007B
:1014400080917A008F7780937A007695679576956C
:10145000679580E090E00E94F583089580E00E9407
:10146000DF09209176023091770240917802509105
:1014700079020E94D58521EE3AE744E95EE30E94B5
:101480008E82089580E18093510160E16093510163
:101490008091510185FF03C06F5F6F31B9F78BE415
:1014A000689FB0011124882777FD8095982F0E94AE
:1014B000F78320E030E64FE954E40E948E8220E07A
:1014C00030E04AE754E40E9458830895CF93DF93B5
:1014D000EC0188819981009799F082389F4021F032
:1014E0001982188283E011C0623171F40E94420AAD
:1014F0006093C7237093C8238093C9239093CA2312
:1015000082E89FE09983888381E0DF91CF910895FD
:1015100080917B00886080937B0089EC80937C00C5
:1015200085E080937A0080917A00806880937A00C9
:1015300080917B0087FFFCCF80917B0085FFFCCFF3
:1015400080917A00806480937A0080917A0086FD91
:10155000FCCF80917A00806480937A0080917A0039
:1015600086FDFCCF609178007091790080917A00BF
:101570008F7780937A0080E090E00E94F58327EDDA
:1015800033EA40E95FE30E94D58526E636E648E87F
:1015900053E40E948D820895BF92CF92DF92EF9222
:1015A000FF920F931F93CF93DF93CDB7DEB72997A9
:1015B0000FB6F894DEBF0FBECDBF6C011092660966
:1015C0008FEF898700E31BE1B12C7E0189E0E80EF3
:1015D000F11C89858823E9F1E8E0BE16E1F1BE013E
:1015E0006F5F7F4FC7010E94CA5889858F3F11F0F6
:1015F0008E3F19F4809366092CC0CE010196C11468
:10160000D10471F40E94E35880934E28FE01319674
:10161000A6E4B8E281918D93EE15FF05D9F71DC0C0
:101620000E94E358F8018083FE01319620E030E00B
:10163000A801485051098191DA01A20FB31F8C9380
:101640002F5F3F4F28303105B1F7B394075F1F4F2D
:10165000C0CF8B2D03C088E001C081E029960FB672
:10166000F894DEBF0FBECDBFDF91CF911F910F91D8
:10167000FF90EF90DF90CF90BF90089583E09EE0C1
:101680009F938F930E94968D0F900F9008952F92A5
:101690003F924F925F926F927F928F929F92AF9202
:1016A000BF92CF92DF92EF92FF920F931F93CF934F
:1016B000DF93EC014B01009711F427E004C0813067
:1016C000910549F426E04AE250E06BE270E089E2DD
:1016D00090E00E94AA57CE010E94CC0A9E0129598F
:1016E000364F5901D9018C93CD2B69F090E3C92E67
:1016F0009BE1D92EC8E2DBE1E12CF12C24EB222E78
:101700002DE0322EA6C086E498E20E94185ABC0151
:10171000882777FD8095982F0E94F7836B017C01C5
:10172000892869F020E030E048EC52E40E945883B8
:101730009F938F937F936F9381EF9DE0ACC0C6E43E
:10174000D8E20CEE1DE089911F928F931F930F93A7
:101750000E94968D0F900F900F900F90B8E2CE34AC
:10176000DB0789F720E030E048EC52E4C701B6011E
:101770000E9458839F938F937F936F938CED9DE08E
:101780009F938F930E94968D0F900F900F900F90C4
:101790000F900F9080914E28882319F088E893E0ED
:1017A00002C08CEF93E09F938F9388ED9DE09F9311
:1017B0008F930E94968D0F900F900F900F9075C091
:1017C00000E010E0FE01E00FF11F80811F928F9377
:1017D000A0ECBDE0BF93AF930E94968D0F5F1F4FAB
:1017E0000F900F900F900F900830110559F720E0DF
:1017F00030E048EC52E4C301B2010E9458839F9349
:101800008F937F936F93A8EBBDE0BF93AF930E943C
:10181000968D0F900F900F900F900F900F90D60114
:101820008C91882309F455C088E893E09F938F93A7
:101830003F922F920E94968D0E943E0BBFEFEB1AB3
:10184000FB0AE9E0CE0ED11C29960F900F900F9065
:101850000F90D5018C9190E0E816F906ECF5CE01D9
:101860000E94185ABC01882777FD8095982F0E9406
:10187000F7832B013C018114910409F4A1CF20E0EE
:1018800030E048EC52E40E9458839F938F937F93FB
:101890006F9385EC9DE09F938F930E94968D0F90A0
:1018A0000F900F900F900F900F90DF91CF911F919D
:1018B0000F91FF90EF90DF90CF90BF90AF909F90EF
:1018C0008F907F906F905F904F903F902F900C94EF
:1018D0003E0B8CEF93E0AACFDF91CF911F910F9138
:1018E000FF90EF90DF90CF90BF90AF909F908F9040
:1018F0007F906F905F904F903F902F900895CF937F
:10190000DF9300D0CDB7DEB78091472889838091DF
:101910004D288A83CE0101960E94234D0F900F908F
:10192000DF91CF910895CF93DF93EC01209146286A
:1019300030914728409148285091492860914A2881
:1019400070914B2880914C2890914D28AFEF0E94C8
:101950000589E1F427E04AE250E06BE270E089E2B9
:1019600090E00E94AA5780E090E00E94CC0AC959FA
:10197000D64F888349E050E06AE070E086E498E260
:101980000E94088FDF91CF910C947F0CDF91CF9153
:1019900008951F920F920FB60F9211240BB60F925B
:1019A000DF92EF92FF920F931F932F933F934F93EA
:1019B0005F936F937F938F939F93AF93BF93CF93D7
:1019C000DF93EF93FF938091512882608093512899
:1019D0008091540286FD2B9A8091540287FD2B9AA8
:1019E00080917A0290917B021816190614F4749A69
:1019F000739A80916D0990916E0985FF02C0749869
:101A000073988091020290910302019790930302D0
:101A100080930202892B09F039C180917B09909152
:101A20007C09019690937C0980937B098091CB235C
:101A30009091CC23A091CD23B091CE230196A11DEE
:101A4000B11D8093CB239093CC23A093CD23B0934F
:101A5000CE2380E190E09093030280930202809174
:101A6000540280FD02C01D9B07C010926B091092AA
:101A70006A0983B7817F09C081E090E090936B0988
:101A800080936A0983B7817F866083BF80916D09E7
:101A900090916E0997FF08C080916A0990916B0937
:101AA000892B61F0749A73980FEC1AE1C8EDD3E2B8
:101AB00034E0E32EF12CDD24D3941FC0739A749884
:101AC000F3CF80917B0990917C0901960E94D68684
:101AD000892BD1F0F801608571856115710509F5D3
:101AE000F801608571856115710569F5065F1F4F05
:101AF0002596FAE1073F1F07D1F1F801608571854E
:101B00006115710539F3DDCF779880916D0990915A
:101B10006E0992FFDFCF7498F0927B02E0927A0216
:101B2000D9CF80917B0990917C0901960E94D6863D
:101B3000892BB1F61C821B82AE0162E186E192E044
:101B40000E942F4FCDCF80917B0990917C090E94FC
:101B5000D686892B59F6D8821A8309831C821B8268
:101B6000AE0162E184E392E00E942F4FBFCF60910B
:101B700058027091590261157105A1F180917B099C
:101B800090917C090E94D686892B61F580912C2842
:101B900090912D28A0912E28B0912F284091BD1B07
:101BA0005091BE1B6091BF1B7091C01B841B950B95
:101BB000A60BB70B8093F71A9093F81AA093F91A13
:101BC000B093FA1A80912C2890912D28A0912E285C
:101BD000B0912F288093BD1B9093BE1BA093BF1B79
:101BE000B093C01B60915602709157026115710548
:101BF000A1F180917B0990917C090E94D686892B66
:101C000061F58091302890913128A0913228B091CF
:101C100033284091C11B5091C21B6091C31B70912E
:101C2000C41B841B950BA60BB70B8093FB1A9093D8
:101C3000FC1AA093FD1AB093FE1A8091302890915F
:101C40003128A0913228B09133288093C11B909302
:101C5000C21BA093C31BB093C41B8091540286FD8A
:101C60002B98809154029091550291FF0FC00E94D1
:101C7000BA638A3119F0C1E0C80F01C0CBE00E94FD
:101C800074628C2F0E94D2630E94BC6240E050E0DC
:101C900060E08CE792E00E942F4FFF91EF91DF917F
:101CA000CF91BF91AF919F918F917F916F915F91F4
:101CB0004F913F912F911F910F91FF90EF90DF90E7
:101CC0000F900BBE0F900FBE0F901F901895809134
:101CD0001F1B9091D723891B08950E94670E8823AC
:101CE00071F0E091D723EF71F0E0EC58F44E808171
:101CF00090E02091D7232F5F2093D72308958FEF73
:101D00009FEF0895CF93DF93EC0110929809109202
:101D10009709888199810097C1F08B36934021F013
:101D20001982188283E0B6C0613109F0B2C0F8941C
:101D300078940E946D0E992790939309809392094D
:101D40008D3009F441C08F3F49F40E94670E811124
:101D5000EECF8BE693E0998388839BC08231910517
:101D600009F458C08F37910509F050C0809190094F
:101D700090919109181619060CF560911131709126
:101D8000123188E090E00E94528D60911131709183
:101D9000123180E290E00E94528D60911131709179
:101DA000123188E090E00E94528D809190099091CC
:101DB00091090197909391098093900980919009DE
:101DC00090919109CF9709F61092D72310921F1B7B
:101DD0008091900990919109FC01E451FC4D108291
:101DE0009093980980939709109291091092900905
:101DF00080914F2890915028009709F4A6CF40E099
:101E000050E06091A6110E942F4F9FCF883091051E
:101E100071F5ACCF60911131709112318DE090E08D
:101E20000E94528D10928F0910928E0980918E0916
:101E300090918F0920919009309191098217930711
:101E40000CF0BCCFFC01E451FC4D8081609111315C
:101E50007091123190E00E94528D80918E09909184
:101E60008F09019690938F0980938E09DFCF60913F
:101E70001131709112310E94528D80919009909190
:101E8000910920919209FC01E451FC4D20830196B7
:101E900091CF81E0DF91CF91089580916A0990916F
:101EA0006B09892BB1F0809154029091550293FDFA
:101EB00010C00E94746283B7817F866083BFF894EC
:101EC00083B7816083BF7894889583B78E7F83BF03
:101ED00078940895CF93DF93EC01888199810097DE
:101EE00019F0853B9F4099F40E9431610E944D0F8B
:101EF00040E050E065E88091AA119091AB110E94FA
:101F00002F4F85EB9FE09983888381E003C019827E
:101F1000188283E0DF91CF910895CF93DF9300D0B3
:101F2000CDB7DEB7892B81F05F934F9381EB9DE0B6
:101F30009F938F9369837A830E94968D0F900F9061
:101F40000F900F907A8169817F936F938EEA9DE065
:101F50009F938F930E94968D0F900F900F900F90EC
:101F60000F900F90DF91CF910895FF920F931F93E1
:101F7000CF93DF930E94316180EB0E94965A8111CA
:101F80001CC00E94FA5A8091C51F9091C61F8160A3
:101F90009093C61F8093C51F81E993E09F938F9311
:101FA0008EEA9DE09F938F930E94968D0F900F90E5
:101FB0000F900F90C1E0D0E002C0C0E0D0E0FEB0D2
:101FC0008F2D8470F82E729A0E9431618EE40E94E7
:101FD000965A811116C00E94FA5A8091C51F90919D
:101FE000C61F82609093C61F8093C51F8E010F5F2E
:101FF0001F4F4CEC58E069E973E0CE010E948D0F51
:10200000E801F11001C072980E9431618EEE0E94C9
:10201000965A811116C00E94FA5A8091C51F90915C
:10202000C61F84609093C61F8093C51F8E010F5FEB
:102030001F4F4CEC58E061EA73E0CE010E948D0F17
:10204000E8010E94316186EA0E94965A811116C009
:102050000E94FA5A8091C51F9091C61F8860909384
:10206000C61F8093C51F8E010F5F1F4F4CEC58E0B9
:1020700068EA73E0CE010E948D0FE8010E94316191
:102080008CE30E94965A81111EC00E94FA5A8091D8
:10209000C51F9091C61F80619093C61F8093C51F76
:1020A0008E010F5F1F4F4CEC58E060EB73E0CE01E8
:1020B0000E948D0F86EA9DE09F938F930E94968DDC
:1020C0000F900F90E8010E94316182ED0E94965AB4
:1020D000811116C00E94FA5A8091C51F9091C61FA7
:1020E00080629093C61F8093C51F8E010F5F1F4FA4
:1020F0004CEC58E068EB73E0CE010E948D0FE801D4
:102100000E94316180E80E94965A811116C00E9497
:10211000FA5A8091C51F9091C61F91609093C61F77
:102120008093C51F8E010F5F1F4F4CEC58E061EC90
:1021300073E0CE010E948D0FE8010E94316180EDB5
:102140000E94965A811116C00E94FA5A8091C51FAA
:102150009091C61F80689093C61F8093C51F8E0103
:102160000F5F1F4F4CEC58E067EC73E0CE010E940C
:102170008D0FE8010E9431618CEE0E94965A811108
:1021800016C00E94FA5A8091C51F9091C61F926096
:102190009093C61F8093C51F8E010F5F1F4F4CEC9D
:1021A00058E06FEC73E0CE010E948D0FE80107E06C
:1021B00010E00E9431618CE70E94965A811113C091
:1021C0000E94FA5A8091C51F9091C61F8064909317
:1021D000C61F8093C51F4CEC58E066ED73E0CE013E
:1021E0000E948D0F05C0015011090115110509F755
:1021F0000E94FA5ADF91CF911F910F91FF900C949A
:102200003E0BCF93DF9300D0CDB7DEB74A8369830F
:102210000E94D15A6981862F0E94025B4A81842FD5
:102220000E94025B0F900F90DF91CF910C94FA5AAD
:10223000AF92BF92DF92EF92FF920F931F93CF93D3
:10224000DF9300D01F92CDB7DEB7182FD22E4A836E
:102250005B8369830E94D15A6981862F0E94025B49
:10226000812F81600E94F85A4A81A42E5B81B52E8D
:1022700000E010E0ED2CF12C81E0E81AF1080D15DA
:1022800080F40E151F0519F40E941D5B02C00E9408
:10229000135BF50180830F5F1F4FFFEFAF1ABF0A7B
:1022A000EECF0F900F900F90DF91CF911F910F9174
:1022B000FF90EF90DF90BF90AF900C94FA5AAF92DE
:1022C000BF92CF92DF92EF92FF920F931F93CF9323
:1022D000DF93CDB7DEB760970FB6F894DEBF0FBEC1
:1022E000CDBFB82EA42E6623E9F18E010F5F1F4FDC
:1022F00080E1F80111928A95E9F728E0A80168E9E0
:1023000080EB0E941811BB2041F02FED33E03F938A
:102310002F930E94848D0F900F906E01F8E0CF0EE6
:10232000D11C56EEE52E53E0F52EF80181918F0178
:102330001F928F93FF92EF920E94848D0F900F90C7
:102340000F900F900C151D0581F788851F928F93B4
:102350002BE334E03F932F930E94848D0F900F90D6
:102360000F900F90AA20E9F18E010F5F1F4F80E1BF
:10237000F80111928A95E9F728E0A80160E880EB5E
:102380000E941811BB2041F08BEE93E09F938F9336
:102390000E94848D0F900F906E01F0E1CF0ED11C42
:1023A00046EEE42E43E0F42EF80181918F011F9256
:1023B0008F93FF92EF920E94848D0F900F900F9059
:1023C0000F900C151D0581F788851F928F938BE365
:1023D00094E09F938F930E94848D0F900F900F90A5
:1023E0000F9060960FB6F894DEBF0FBECDBFDF91A1
:1023F000CF911F910F91FF90EF90DF90CF90BF9002
:10240000AF900895CF93DF9300D0CDB7DEB71A8297
:10241000198222E0AE014F5F5F4F6AEA8EEE0E94A2
:102420001811898190E0982F88272A81822B909318
:10243000951B8093941B22E0AE014F5F5F4F6CEAC7
:102440008EEE0E941811898190E0982F88272A81AA
:10245000822B9093971B8093961B22E0AE014F5FD7
:102460005F4F6EEA8EEE0E941811898190E0982FDE
:1024700088272A81822B9093991B8093981B22E0B6
:10248000AE014F5F5F4F60EB8EEE0E9418118981A5
:1024900090E0982F88272A81822B9093A71B809306
:1024A000A61B22E0AE014F5F5F4F62EB8EEE0E94F3
:1024B0001811898190E0982F88272A81822B909388
:1024C000A91B8093A81B22E0AE014F5F5F4F64EB16
:1024D0008EEE0E941811898190E0982F88272A811A
:1024E000822B9093AB1B8093AA1B22E0AE014F5F1F
:1024F0005F4F66EB8EEE0E941811898190E0982F55
:1025000088272A81822B90939B1B80939A1B22E021
:10251000AE014F5F5F4F68EB8EEE0E94181189810C
:1025200090E0982F88272A81822B90939D1B80937F
:102530009C1B22E0AE014F5F5F4F6AEB8EEE0E9464
:102540001811898190E0982F88272A81822B9093F7
:10255000A11B8093A01B22E0AE014F5F5F4F6CEB8D
:102560008EEE0E941811898190E0982F88272A8189
:10257000822B9093A31B8093A21B22E0AE014F5F9E
:102580005F4F6EEB8EEE0E941811898190E0982FBC
:1025900088272A81822B9093A51B8093A41B0F90E0
:1025A0000F90DF91CF9108952F923F924F925F92BB
:1025B0006F927F928F929F92AF92BF92CF92DF9253
:1025C000EF92FF920F931F93CF93DF93CDB7DEB7B8
:1025D0006A970FB6F894DEBF0FBECDBF182F488F95
:1025E000298F19821A821B828091B81B811107C022
:1025F0006A8F0E94021281E08093B81B6A8D662365
:1026000009F46CC04EE264EF8EEE0E94011169E0A5
:102610007AE180E090E00E94835A22E0AE014F5FB1
:102620005F4F66EF8EEE0E9418112981822F90E095
:10263000A0E0B0E02227382F492F5A2F8A81282B7B
:102640008091AA1B9091AB1B281B390B41095109A2
:10265000A091A81BB091A91B0E94B3866B017C01BD
:102660008FE0F594E794D794C7948A95D1F7609159
:10267000A21B7091A31B882777FD8095982F2BE0D4
:10268000660F771F881F991F2A95D1F72091A41BE9
:102690003091A51B442737FD4095542F2C0D3D1D2F
:1026A0004E1D5F1D0E942087C20ED31ED0929F1B1D
:1026B000C0929E1B88E0C80ED11C34E0D594C7940C
:1026C0003A95E1F7EE24D7FCE094FE2CC092AC1BC7
:1026D000D092AD1BE092AE1BF092AF1B012F029582
:1026E000000F000F007C0C5CA12FB0E0BD8BAC8B09
:1026F000A3E0B0E0012E02C0AA0FBB1F0A94E2F7CC
:1027000025E335E00E94AC86DC01CB010296A11DD9
:10271000B11D8C879D87AE87BF8780E593ECA0E0D5
:10272000B0E004C0B595A795979587951A95D2F70F
:10273000888B998BAA8BBB8B10E0188619861A861A
:102740001B86A8E02A2E312CAC89BD892A1A3B0AA7
:10275000988D191709F436C1402F64EF8EEE0E9450
:1027600001116C857D858E859F850E94835A23E0AB
:10277000AE014F5F5F4F66EF8EEE0E941811E09141
:102780009E1BF0919F1BE05AFF409F01DF010E94BA
:1027900095866B017C018091961B9091971B9F8B76
:1027A0008E8BA090941BB090951B2091981B30911C
:1027B000991B0E9495862B013C013DE0759467941E
:1027C000579447943A95D1F7A0919A1BB0919B1BCF
:1027D000A70196016CE055954795379527956A9521
:1027E000D1F70E94BE86BB2797FDB095AB2F480E50
:1027F000591E6A1E7B1E92E0490E511C611C711C01
:10280000B2E07594679457944794BA95D1F7A0E8CD
:102810005A0E611C711CA091A61BB091A71BA301AD
:1028200092010E94B386DC01CB012FE0B695A795FB
:10283000979587952A95D1F78C839D83AE83BF8327
:1028400029818A8190E0A0E0B0E04424582E692ECE
:102850007A2E622A8B81482A022C04C075946794D0
:10286000579447940A94D2F74501AA2497FCA09460
:10287000BA2C42E0880C991CAA1CBB1C4A95D1F7C3
:10288000A0919C1BB0919D1BA70196010E94BE8642
:102890006B017C0157E1F594E794D794C7945A955E
:1028A000D1F72E893F89DF010E949586EBE095954F
:1028B000879577956795EA95D1F7C60ED71EE81EDE
:1028C000F91E8C0C9D1CAE1CBF1C0C8804C0880C0F
:1028D000991CAA1CBB1C0A94D2F792E0890E911C89
:1028E000A11CB11CF2E0B594A79497948794FA9533
:1028F000D1F7481859086A087B08A3019201688932
:1029000079898A899B890E94C68697FD0DC0660FCA
:10291000771F881F991F2C813D814E815F810E9406
:10292000FE8649015A010CC02C813D814E815F8198
:102930000E94FE8649015A01880C991CAA1CBB1CE6
:102940009927B7FC9A958B2D7A2D692D9B01AC01A7
:102950000E94C6869B01AC01AEEDBBE00E94B3862F
:102960006C01FF24D7FCF094EF2CA3E4B3EEA50197
:1029700094010E94C186BB2797FDB095AB2FC80E6E
:10298000D91EEA1EFB1EAFECCA0EAEE0DA1EE11C39
:10299000F11CA4E0F594E794D794C794AA95D1F7D5
:1029A000C80CD91CEA1CFB1C88859985AA85BB85A7
:1029B0008C0D9D1DAE1DBF1D88879987AA87BB877B
:1029C0001F5FC6CE112391F0212F30E040E050E090
:1029D000688579858A859B850E94FE862093B01B39
:1029E0003093B11B4093B21B5093B31BA98DAA2304
:1029F00089F16091B01B7091B11B8091B21B9091D5
:102A0000B31B611571058105910521F10E94F783C2
:102A100020E836EE45EC57E40E94588321E03EED75
:102A200042E45EE30E9438869B01AC0160E070E006
:102A300080E89FE30E948D822BE43AE34DEB57E35D
:102A40000E9458836093B41B7093B51B8093B61B90
:102A50009093B71B6A960FB6F894DEBF0FBECDBF3A
:102A6000DF91CF911F910F91FF90EF90DF90CF906A
:102A7000BF90AF909F908F907F906F905F904F909E
:102A80003F902F9008950F931F93CF93DF9300D023
:102A900000D000D0CDB7DEB78E010F5F1F4F86E0AC
:102AA000F80111928A95E9F78091C61A811113C035
:102AB00040E061E386EA0E9401114AE06CE286EAA6
:102AC0000E94011181E08093C61A6CE77EE380E0EA
:102AD00090E00E94835A48E06DE286EA0E9401116C
:102AE0006CE77EE380E090E00E94835A26E0A80134
:102AF00062E386EA0E94181147E06DE286EA0E94CE
:102B000001118A8190E0982F88272981822B909348
:102B1000C11A8093C01A2C8130E0322F22274B81BA
:102B2000242B3093C31A2093C21A4E8150E0542FA5
:102B300044276D81462B5093C51A4093C41A5F9366
:102B40004F933F932F939F938F938FEE93E09F9399
:102B50008F930E94848D0FB6F894DEBF0FBECDBF59
:102B600026960FB6F894DEBF0FBECDBFDF91CF9192
:102B70001F910F910895CF92DF92EF92FF920F93E2
:102B80001F93CF93DF93CDB7DEB72A970FB6F89494
:102B9000DEBF0FBECDBF8E010F5F1F4F86E0F80175
:102BA00011928A95E9F741E062E08CE30E940111FD
:102BB00048E560E08CE30E94011162E174E380E08B
:102BC00090E00E94835A26E0A80163E08CE30E9413
:102BD000181143E062E08CE30E940111098110E0CA
:102BE000102F00278A81082B1093A11A0093A01A96
:102BF000EB80F12CFE2CEE248C81E82AF092A31AB3
:102C0000E092A21ACD80D12CDC2CCC248E81C82A53
:102C1000D092A51AC092A41AB801882777FD809592
:102C2000982F0E94F7839B01AC01B701882777FD9D
:102C30008095982F2F83388749875A870E94F7837A
:102C40002F81388549855A850E94018320EE3EE216
:102C500045E652E40E94D58520E030E044E353E4A9
:102C60000E948E829F938F937F936F93DF92CF9278
:102C7000FF92EF921F930F938DEF93E09F938F93AB
:102C80000E94848D0FB6F894DEBF0FBECDBF2A968A
:102C90000FB6F894DEBF0FBECDBFDF91CF911F916D
:102CA0000F91FF90EF90DF90CF900895CF93DF9337
:102CB000EC01888199810097F9F08E399F4021F0CD
:102CC0001982188283E063C08DE799E00E94D55194
:102CD000892BE1F080916D0990916E0993FD18C0E8
:102CE00080916D0990916E0994FD43C080916D09AA
:102CF00090916E0995FD44C060E870E08DE799E021
:102D00000E94AE518EE99FE09983888381E03FC0A5
:102D10008091C51F82FFE4CF21E048E061E083E0BD
:102D20000E94D4128091B71B8F938091B61B8F9312
:102D30008091B51B8F938091B41B8F938091B31BAF
:102D40008F938091B21B8F938091B11B8F93809151
:102D5000B01B8F9385E09EE09F938F930E94968D8A
:102D60008DB79EB70A960FB6F8949EBF0FBE8DBF63
:102D7000B7CF8091C51F83FFB9CF0E944315B6CF4F
:102D80008091C51F84FFB8CF0E94BB15B5CFDF91DE
:102D9000CF910895CF93C82F8CEE0E94F85A8C2FB4
:102DA0000E94025B65E375E080E090E00E94835A38
:102DB0008DEE0E94F85A0E94135BC82F0E941D5B83
:102DC0002C2F30E0322F2227A901482BCA01CF91A6
:102DD0000895CF93DF93C82F8CEE0E94F85A8C2F62
:102DE0000E94025B62E174E380E090E00E94835AFB
:102DF0008CEE0E94F85A80E00E94025B65E375E069
:102E000080E090E00E94835A8DEE0E94F85A0E9462
:102E1000135BC82F0E94135BD82F0E941D5B4D2FA0
:102E200050E060E070E0762F652F542F44276C2B24
:102E3000482BCB01BA01DF91CF9108952F923F9299
:102E40004F925F926F927F928F929F92AF92BF92BA
:102E5000CF92DF92EF92FF920F931F93CF93DF9366
:102E6000CDB7DEB7CD54D1090FB6F894DEBF0FBE93
:102E7000CDBF8091000290910102892BD1F1109277
:102E80000102109200028CEE0E94F85A8EE10E941C
:102E9000025B6BE17EE480E090E00E94835A82EA6C
:102EA0000E94CA1690937A098093790984EA0E9455
:102EB000CA16909378098093770986EA0E94CA1609
:102EC000909376098093750988EA0E94CA169093B8
:102ED0007409809373098AEA0E94CA169093720952
:102EE000809371098CEA0E94CA16909370098093AE
:102EF0006F0988E40E94E9166FAB78AF89AF9AAF8B
:102F000088E50E94E9164B015C018091710990915E
:102F1000720920E030E040E050E0BA0126962FAF81
:102F2000269727963FAF279728964FAF2897299641
:102F30005FAF29972A966FAF2A972B967FAF2B9773
:102F40009C0140E050E060E070E080E090E008E04C
:102F50000E94A7880E9453883901B42FA52FF62F0D
:102F6000E72F8C019401A50160E070E080E090E023
:102F70005301CB2EDA2EEF2EFE2E0E94DE882983FF
:102F80003A832A011B014C01B101C40131504109AE
:102F90005F4F6F4F7F4F8F4F9F4FA1E0B0E025965F
:102FA000BFAFAEAF259721153F4F4F4F5140610541
:102FB00071058105910509F020F425961FAE1EAE1E
:102FC000259725966EAC7FAC259780916F099091DF
:102FD00070095C01C12CD12CE12CF12C00E010E037
:102FE00029813A81A201B101C4010E947687D22EC3
:102FF000E32EF42E052F162FB72FF82FE92FA0E080
:103000000E94058984F42150310940485F4F6F4F79
:103010007F4F8F4F9F4FD22EE32EF42E052F162F6A
:10302000B72FF82FE92F2D2D3E2D4F2D502F612F2B
:103030007B2F8F2F9E2F07E10E94C0882B8F3C8F04
:103040004D8F5E8F6F8F78A389A39AA32053384F3B
:103050004F4F5F4F6F4F7F4F8F4F9F4F2B8B3C8B4F
:103060004D8B5E8B6F8B788F898F9A8F2056304F68
:103070004F4F5F4F6F4F7F4F8F4F9F4F243D3043D8
:1030800041055105610571058105910541F038F053
:1030900025966EAC7FAC2597FFEF6F1A7F0A809163
:1030A0007709909178099C0140E050E060E070E081
:1030B00080E090E000E10E94A7882B833C834D8351
:1030C0005E836A8779878F839887409173095091CF
:1030D0007409A980BA806201710184019A0140E0FB
:1030E00050E060E070E080E090E00E947687D22EB1
:1030F000E32EF42E052F162FB72FF82FE92FA0E07F
:103100000E9405895CF4AFE70E94E788D22EE32E87
:10311000F42E052F162FB72FF82FE92F2D2D3E2D2A
:103120004F2D502F612F7B2F8F2F9E2F07E00E9456
:10313000C08859016A017B018C012B813C814D8142
:103140005E816A8579858F8198850E94DE882B83D0
:103150003C834D835E836F8378878F87988B2E5F48
:103160003F4F434051096E4F7F4F8F4F9F4F22304B
:103170003105494F5F4F644071058105910521F08C
:1031800018F01FEF611A710A8091790990917A09FC
:10319000BC0180E090E020E030E840E050E00E9498
:1031A000CF8729873A874B875C876A8B798B8D8796
:1031B0009E874091750950917609A980BA80620175
:1031C000710184019A0140E050E060E070E080E02D
:1031D00090E00E947687D22EE32EF42E052F162F34
:1031E000B72FF82FE92FA0E00E94058984F4215021
:1031F0003F4F4F4F5F4F6F4F7F4F8F4F9F4FD22E9D
:10320000E32EF42E052F162FB72FF82FE92F2D2D93
:103210003E2D4F2D502F612F7B2F8F2F9E2F08E09B
:103220000E94C08859016A017B018C0129853A8579
:103230004B855C856A8979898D859E850E94DE88AB
:1032400029873A874B875C876D877E87898B9A8B26
:103250002F5F3F4F4140510961097109810991096F
:10326000213030484C4F5F47614071058105910521
:1032700021F018F0BFEF6B1A7B0A2B893C894D892E
:103280005E896F89788D898D9A8D2F3C37404105F5
:103290005105610571058105910511F00CF0A5C17D
:1032A000A980BA806201710184019501A201B10176
:1032B000C4010E947687A12CB12CC12C10E8D12E1C
:1032C000E12CF12C00E010E00E9439872BAF3CAFDD
:1032D0004DAF5EAF6FAF21967FAF219722968FAF34
:1032E000229723969FAF2397AB8CBC8CCD8CDE8C22
:1032F000EF8CF8A009A11AA19501A601B701C80198
:103300000E94768759016A017B01E82F192F02E09C
:103310000E94A7880E2F0E94DE8869017A01162F6D
:10332000272EF82FE92F322E8D2C942EAF2CB62E6F
:10333000072F582EB92FA0E00E9405895CF4A1E068
:103340000E94E788322E832E942EA52EB62E072FAC
:10335000582EB92F232D382D492D5A2D6B2D702F16
:10336000852D9B2F01E00E94C0882E962FAF2E97AF
:103370002D963FAF2D9749A75AA76BA77CA78DA77E
:103380009EA7522E432E4BA35CA36DA37EA38FA3B7
:1033900098A7B22D9601A701612F722D8F2F9E2F16
:1033A000A0E00E9405894CF4A3E00E94E78869012F
:1033B0007A01162FB72FF82FE92F9601A701612F59
:1033C0007B2F8F2F9E2F02E00E94C0882FA738AB43
:1033D00049AB5AAB6BAB7CAB8DAB9EAB19014A01D1
:1033E000B62FA72F24968FAF2497F92F2B893C89CE
:1033F0004D895E896F89788D898D9A8D24323A4FF7
:103400004F4F5F4F6F4F7F4F8F4F9F4F0CF08CC0D0
:103410002B8D3C8D4D8D5E8D6F8D78A189A19AA1EC
:103420002455324F4F4F5F4F6F4F7F4F8F4F9F4FFE
:1034300059016A017B018C010E94768719014A01BA
:10344000B62FA72FFC0103E00E94A7885101640159
:10345000EB2EFA2E8F010E94F38859016A017B013D
:103460008C012E962FAD2E972D963FAD2D9749A509
:103470005AA56BA57CA58DA59EA50E94DE88522E1F
:10348000432E4BA35CA36DA37EA38FA398A79101AA
:10349000A4016B2F7A2FCF0102E00E94A78851016F
:1034A0006401EB2EFA2E8F010E94F38802E00E9445
:1034B000A7880E2F0E94F388F22E032F142FD52EEB
:1034C000E62EB72FF82FE92FA0E00E9405895CF4C3
:1034D000A1E00E94E788F22E032F142FD52EE62EAE
:1034E000B72FF82FE92F2F2D302F412F5D2D6E2D67
:1034F0007B2F8F2F9E2F01E00E94C08859016A0107
:103500007B018C012FA538A949A95AA96BA97CA9CF
:103510008DA99EA90E94DE8819014A01B62FA72F06
:1035200024968FAF2497F92F2B813C814D815E81AA
:103530006F8178858F859889A52CB42CCBA0DCA0D1
:10354000EDA0FEA00FA118A50E94F3882B833C8359
:103550004D835E836F8378878F87988B29853A8523
:103560004B855C856D857E8589899A8951016401C9
:10357000EB2EFA2E24960FAD24971F2F0E94F3886E
:1035800029873A874B875C876D877E87898B9A8BE3
:103590002B893C894D895E896F89788D898D9A8DBB
:1035A000ABACBCACCDACDEACEFAC2196FFAC2197A4
:1035B00022960FAD229723961FAD23970E94F38882
:1035C0002056304F4F4F5F4F6F4F7F4F8F4F9F4F62
:1035D000243D304341055105610571058105910583
:1035E00021F018F02FEF621A720A6FA978AD89AD39
:1035F0009AADAB01BC0180E090E0DC0124964FAFB6
:10360000249725965FAF259726966FAF2697279626
:103610007FAF279728968FAF289729969FAF299736
:103620002A96AFAF2A972B96BFAF2B97A984BA845F
:10363000CB84DC84ED84FE8409891A899A01AB016C
:1036400060E070E080E090E00E947687F22E032F29
:10365000142FD52EE62EB72FF82FE92FA0E00E94C9
:10366000058984F421503109404E5F4F6F4F7F4FE1
:103670008F4F9F4FF22E032F142FD52EE62EB72FEC
:10368000F82FE92F2F2D302F412F5D2D6E2D7B2F01
:103690008F2F9E2F05E10E94C088AB80BC80CD801B
:1036A000DE80EF80F8840F8518890E94F388F22E5F
:1036B000032F142FD52EE62EB72FF82FE92FA0E0D9
:1036C0000E94058984F4215030484F4F5F4F6F4F5F
:1036D0007F4F8F4F9F4FF22E032F142FD52EE62EA4
:1036E000B72FF82FE92F2F2D302F412F5D2D6E2D65
:1036F0007B2F8F2F9E2F0FE00E94C08869017A01D7
:103700008B018A83998329011A014B015C01285E90
:103710003340410951096109710981099109283D25
:10372000304D41405105610571058105910521F03C
:1037300018F0BFEF6B1A7B0A0E94FA5A672859F0FB
:103740009601A701B8018A8199810E9453882901B5
:103750001A014B015C019201A101B401C5010E9453
:10376000F18320E030E048EC52E40E945883C35BD0
:10377000DF4F0FB6F894DEBF0FBECDBFDF91CF9104
:103780001F910F91FF90EF90DF90CF90BF90AF907F
:103790009F908F907F906F905F904F903F902F9071
:1037A00008954F925F926F927F928F929F92AF9205
:1037B000BF92CF92DF92EF92FF922B013C01690101
:1037C0007A0123EC35EF4CE851E4C701B6010E94C1
:1037D000D5854B015C0128EB3EE143E753E4C7018B
:1037E000B6010E948E829B01AC01C501B4010E940A
:1037F00058830E94C5834B015C0120E030E048EC17
:1038000052E4C301B2010E94588321E835E943EC38
:1038100050E40E94D585A50194010E94D5854B01F5
:103820005C0123E333E948E853E4C701B6010E9491
:103830008E829B01AC01C501B4010E94588323E331
:1038400033EB48E553E40E94D585FF90EF90DF907D
:10385000CF90BF90AF909F908F907F906F905F9030
:103860004F9008954F925F926F927F928F929F92A6
:10387000AF92BF92CF92DF92EF92FF9269017A01ED
:103880000E94578520E030E040E050E40E948D82A5
:1038900022E93CE54EED5EE30E9458834B015C015A
:1038A00023EC35EF4CE851E4C701B6010E94D58501
:1038B0002B013C0128EB3EE143E753E4C701B6018D
:1038C0000E948E829B01AC01C301B2010E94588309
:1038D0009B01AC01C501B4010E948E826B017C0189
:1038E00028EB3EE143E753E40E94D5854B015C01A0
:1038F000A701960163EC75EF8CE891E40E948D823C
:103900009B01AC01C501B4010E945883FF90EF9068
:10391000DF90CF90BF90AF909F908F907F906F90EF
:103920005F904F9008954F925F926F927F928F9227
:103930009F92AF92BF92CF92DF92EF92FF922B01B4
:103940003C0169017A0123EC35EF4CE851E4C701F1
:10395000B6010E94D5854B015C0128EB3EE143E7AF
:1039600053E4C701B6010E948E829B01AC01C501E0
:10397000B4010E9458830E94C5834B015C0120E082
:1039800030E048EC52E4C301B2010E945883A50123
:1039900094010E94D58520E030E040E251E40E948D
:1039A0008D8224EE38E34EE05FE30E94D5859B01D3
:1039B000AC01C701B6010E948E82FF90EF90DF90AC
:1039C000CF90BF90AF909F908F907F906F905F90BF
:1039D0004F900895CF92DF92EF92FF920F931F9333
:1039E000CF93DF9380E80E94F85A8AEF0E94025B2F
:1039F0008FE00E94025B65E375E080E090E00E944A
:103A0000835A81E80E94F85A0E94135BC82F0E94D3
:103A1000135B0E94135BD82F0E94135B0E94135B01
:103A2000182F0E94135B0E941D5B082F0E941D5BD4
:103A300080E80E94F85A8CEF0E94025B89EC0E9499
:103A4000025B65E375E080E090E00E94835A81E8C4
:103A50000E94F85A0E94135BD82E0E94135BC82E56
:103A60000E94135B0E94135BF82E0E94135BE82EEA
:103A70000E941D5B1F92CF921F92DF921F920F93A5
:103A80001F921F931F92DF931F92CF931F92EF926B
:103A90001F92FF9282E194E09F938F930E94848D06
:103AA0000E94FA5A8DB79EB742960FB6F8949EBF01
:103AB0000FBE8DBF20E030E040E050E060E070E0FD
:103AC00080E090E0DF91CF911F910F91FF90EF90F8
:103AD000DF90CF9008950F931F93CF93DF93EC0166
:103AE00080E80E94F85A209741F085EE0E94025B20
:103AF00061E077E980E090E007C083EE0E94025B1E
:103B000069E97AEB81E090E00E94835A81E80E94A3
:103B1000F85A0E94135B182F0E94135B082F0E9413
:103B20001D5B0E94FA5A602F70E0712B6C7F80E061
:103B300090E0CD2B69F00E94F58320E030E04AEF61
:103B40005AE30E94D58520E030E040EC50E40CC000
:103B50000E94F58322E538EB4FE25BE30E94D585B6
:103B600026E636E64BE352E40E948D82DF91CF9148
:103B70001F910F9108950F931F93CF93DF93729A24
:103B80008091540283FF08C08EE40E94965A8111EE
:103B900063C0C0E5D0E008C0C0E5D0E00E944B099A
:103BA00021972097D9F7F0CF0E944B0921972097B2
:103BB000D9F78FE40E94965A0E94135B082F0F7367
:103BC0000E94135B182F0E94135BD82F0E941D5B6D
:103BD000C82F0E94FA5A8091540283FF7298602F76
:103BE00070E0762F6627610F711D80E090E00E94E3
:103BF000F58320E134E048EC5BE30E94D5856093D7
:103C0000B91B7093BA1B8093BB1B9093BC1B6D2F89
:103C100070E0762F66276C0F711D76956795769507
:103C2000679580E090E00E94F58324EA3CEF44E24F
:103C30005CE30E94D58520E030E040E252E40E943F
:103C40008D826093522870935328809354289093C8
:103C5000552880E090E002C081E090E0DF91CF91B4
:103C60001F910F9108957298729A8EE40E94965A4D
:103C700080EA0E94025B80E00E94025B80E00E947A
:103C8000025B8FE40E94965A0E94135B8EE40E94AE
:103C9000965A80E80E94025B80E00E94025B80E00E
:103CA0000E94025B0E94FA5A80E090E0089589E940
:103CB0009DE09F938F930E94968D80916D020F904F
:103CC0000F90882361F01F928F9386E99DE09F9368
:103CD0008F930E94968D0F900F900F900F900895E4
:103CE00081E79DE09F938F930E94968D89E49DE0EC
:103CF0009F938F930E94968D82E29DE09F938F9376
:103D00000E94968D87EE9CE09F938F930E94968DE4
:103D100085EB9CE09F938F930E94968D89E79CE0B2
:103D20009F938F930E94968D83E59CE09F938F9342
:103D30000E94968D8DE19CE09F938F930E94968DBB
:103D40008091C51F9091C61F827091702DB73EB7AC
:103D5000205F3F4F0FB6F8943EBF0FBE2DBF892B9B
:103D600041F08DEE9BE09F938F930E94968D0F9074
:103D70000F9081EC9BE09F938F930E94968D88E932
:103D80009BE09F938F930E94968D8CE69BE09F9380
:103D90008F930E94968D8DE39BE09F938F930E945B
:103DA000968D8BE09BE09F938F930E94968D8AED7A
:103DB0009AE09F938F930E94968D80EA9AE09F935A
:103DC0008F930E94968D8AE69AE09F938F930E942C
:103DD000968D8AE39AE09F938F930E94968D8EE052
:103DE0009AE09F938F930E94968D8FED99E09F9319
:103DF0008F930E94968D86EA99E09F938F930E94FD
:103E0000968D8DE699E09F938F930E94968D86E321
:103E100099E09F938F930E94968D85E099E09F9300
:103E20008F930E94968D86ED98E09F938F930E94CA
:103E3000968D8DB79EB780960FB6F8949EBF0FBE35
:103E40008DBF87EA98E09F938F930E94968D80E8BC
:103E500098E09F938F930E94968D8AE498E09F93B9
:103E60008F930E94968D84E198E09F938F930E9498
:103E7000968D8BEE97E09F938F930E94968D83EBA8
:103E800097E09F938F930E94968D88E897E09F9389
:103E90008F930E94968D2DB73EB7225F3F4F0FB68E
:103EA000F8943EBF0FBE2DBF089581E494E00C94BA
:103EB000BA8D4F925F926F927F928F929F92AF9244
:103EC000BF92CF92DF92EF92FF92CF93DF93CDB765
:103ED000DEB728970FB6F894DEBF0FBECDBF809136
:103EE000CB239091CC23A091CD23B091CE23898375
:103EF0009A83AB83BC834090CB235090CC236090BB
:103F0000CD237090CE238091CB239091CC23A09190
:103F1000CD23B091CE238D839E83AF83B8876091EC
:103F2000CB237091CC238091CD239091CE232CE391
:103F3000822E912CA12CB12CA50194010E94FE8609
:103F40007F936F9330E1C32E3EE0D32EE12CF12C12
:103F50006D817E818F819885A70196010E94FE86E2
:103F6000A50194010E94FE863F932F9340E8842E82
:103F700041E5942EAA24A394B12CC301B201A5015A
:103F800094010E94FE86A70196010E94FE863F933F
:103F90002F9369817A818B819C81A50194010E9474
:103FA000FE863F932F9382E697E09F938F930E9424
:103FB000968D0FB6F894DEBF0FBECDBF28960FB614
:103FC000F894DEBF0FBECDBFDF91CF91FF90EF9091
:103FD000DF90CF90BF90AF909F908F907F906F9029
:103FE0005F904F900895E7E1F1E380819181823401
:103FF000924479F0E751F143FF93EF9384E497E023
:104000009F938F930E94968D0F900F900F900F901B
:1040100008953A96E53F81E4F80738F30895CF9381
:10402000DF93EC018C9A0E942E0A9F938F937F93CB
:104030006F9388E397E09F938F930E94968D0F90E4
:104040000F900F900F900F900F90209719F00E94F3
:104050003E0B08C086E397E09F938F930E94968D56
:104060000F900F9081E00E94DF0920917202309141
:10407000730240917402509175020E94D5859F93FE
:104080008F937F936F938AE297E09F938F930E9421
:10409000968D0F900F900F900F900F900F9020978C
:1040A00019F00E943E0B08C088E297E09F938F931F
:1040B0000E94968D0F900F9082E00E94DF09209160
:1040C0006E0230916F0240917002509171020E9415
:1040D000D5859F938F937F936F938CE197E09F9308
:1040E0008F930E94968D0F900F900F900F900F90CE
:1040F0000F90209719F00E943E0B08C08AE197E0CC
:104100009F938F930E94968D0F900F9083E00E9453
:10411000DF099F938F937F936F938BE097E09F933B
:104120008F930E94968D8C980F900F900F900F9008
:104130000F900F90209719F00E943E0B08C089E065
:1041400097E09F938F930E94968D0F900F90809190
:10415000C51F87FF83C021E042E161E080ED0E943E
:104160005A5C9F938F937F936F938CEF96E09F930E
:104170008F930E94968D0F900F900F900F900F903D
:104180000F90209719F00E943E0B08C08AEF96E02E
:104190009F938F930E94968D0F900F9021E042E1A4
:1041A00062E080ED0E945A5C9F938F937F936F93A0
:1041B0008DEE96E09F938F930E94968D0F900F90B7
:1041C0000F900F900F900F90209719F00E943E0BC8
:1041D00008C08BEE96E09F938F930E94968D0F9070
:1041E0000F9021E042E163E080ED0E945A5C9F93D2
:1041F0008F937F936F938EED96E09F938F930E94A2
:10420000968D0F900F900F900F900F900F90CD2BD9
:1042100019F00E943E0B08C08CED96E09F938F939F
:104220000E94968D0F900F9021E042E164E080EDB6
:104230000E945A5C9F938F937F936F938FEC96E0CD
:104240009F938F930E94968D0F900F900F900F90D9
:104250000F900F90DF91CF910C943E0BCD2BD1F3AB
:10426000DF91CF9108950F931F93CF93DF9388230E
:1042700089F049E050E06FEF70E086E498E20E9438
:10428000D88C49E050E06AE070E086E498E20E9451
:10429000088F13C0C6E4D8E20AEC16E089911F9299
:1042A0008F931F930F930E94968D0F900F900F90F6
:1042B0000F9088E2CE34D80789F7DF91CF911F9114
:1042C0000F910C943E0BCF92DF92EF92FF92CF931F
:1042D000DF936B017C0160FF11C08EE794E09F9338
:1042E0008F938EEA9DE09F938F930E94968D0F90FF
:1042F0000F900F900F9081E090E002C080E090E07E
:10430000C1FE09C0EC0121964CEC58E063E874E072
:104310000E948D0FCE01C2FE09C0EC0121964CEC2B
:1043200058E06BE874E00E948D0FCE01C3FE09C017
:10433000EC0121964CEC58E063E974E00E948D0F8B
:10434000CE01C4FE09C0EC0121964CEC58E067E9AF
:1043500074E00E948D0FCE01C5FE09C0EC012196CC
:104360004CEC58E06AE974E00E948D0FCE01C6FE65
:1043700009C0EC0121964CEC58E06EE974E00E9413
:104380008D0FCE01C7FE09C0EC0121964CEC58E020
:1043900064EA74E00E948D0FCE01D0FE09C0EC01EA
:1043A00021964CEC58E06CEA74E00E948D0FCE012F
:1043B000D1FE09C0EC0121964CEC58E064EB74E0AE
:1043C0000E948D0FCE01D2FE09C0EC0121964CEC6B
:1043D00058E068EB74E00E948D0FCE012091C51F5C
:1043E0003091C61F24703270232B59F0D3FE09C0C0
:1043F000EC0121964CEC58E06EEB74E00E948D0FBE
:10440000CE012091C51F23FF0BC0D4FE09C0EC01D3
:1044100021964CEC58E063EC74E00E948D0FCE01C5
:104420002091C51F24FF0BC0D5FE09C0EC012196C9
:104430004CEC58E069EC74E00E948D0FCE01D6FE82
:1044400009C0EC0121964CEC58E061ED74E00E944B
:104450008D0FCE01B701A60144275078452B462B7E
:10446000472B61F04CEC58E06CED74E0DF91CF919C
:10447000FF90EF90DF90CF900C948D0FCD28CE2839
:10448000CF2841F485EC96E09F938F930E94968D00
:104490000F900F90DF91CF91FF90EF90DF90CF9032
:1044A00008950F931F93CF93DF938C01C0E0D0E06A
:1044B0000115110509F48AC060EC76E0C8010E947C
:1044C000B78C892B09F4C16068EB76E0C8010E94C3
:1044D000B78C892B09F4C26060EB76E0C8010E94BA
:1044E000B78C892B09F4C4606CEA76E0C8010E949D
:1044F000B78C892B09F4C86069EA76E0C8010E948C
:10450000B78C892B09F4C06165EA76E0C8010E9486
:10451000B78C892B09F4C0626FE976E0C8010E946C
:10452000B78C892B09F4C06467E976E0C8010E9462
:10453000B78C892B09F4C0686FE876E0C8010E9447
:10454000B78C892B09F4D1606BE876E0C8010E9432
:10455000B78C892B09F4D26065E876E0C8010E9427
:10456000B78C892B09F4D46060E876E0C8010E941A
:10457000B78C892B09F4D8606AE776E0C8010E94FD
:10458000B78C892B09F4D06162E776E0C8010E94FC
:10459000B78C892B09F4D06267E676E0C8010E94E7
:1045A000B78C892B09F4D06466E576E0C8010E94D7
:1045B000B78C892B09F4D06860916B0270916C0202
:1045C00080E090E00E94CB8C8C0172CFCE01DF9115
:1045D000CF911F910F910895AF92BF92CF92DF922A
:1045E000EF92FF920F931F93CF93DF93F22E032F3F
:1045F000142FE52E5B016C01217030E040E050E0AB
:1046000060E070E080E090E0A0E00E94058989F021
:10461000EDEEF4E0FF93EF93EEEAFDE0FF93EF930E
:104620000E94968D0F900F900F900F90E1E0F0E0B8
:1046300002C0E0E0F0E08091C51F80FF17C02F2D81
:10464000247030E040E050E060E070E080E090E016
:10465000A0E00E94058951F0EF0121964CEC58E052
:1046600061EF74E0CF010E948D0FFE012F2D2270AB
:1046700030E040E050E060E070E080E090E0A0E0FA
:104680000E94058951F0EF0121964CEC58E065EF4E
:1046900074E0CF010E948D0FFE012F2D287030E0B5
:1046A00040E050E060E070E080E090E0A0E00E9438
:1046B000058951F0EF0121964CEC58E06DE075E072
:1046C000CF010E948D0FFE012F2D207130E040E0C0
:1046D00050E060E070E080E090E0A0E00E9405899A
:1046E00051F0EF0121964CEC58E068EF74E0CF01F7
:1046F0000E948D0FFE012F2D207230E040E050E02F
:1047000060E070E080E090E0A0E00E94058951F058
:10471000EF0121964CEC58E06BEF74E0CF010E9462
:104720008D0FFE012F2D207430E040E050E060E05E
:1047300070E080E090E0A0E00E94058951F0EF0178
:1047400021964CEC58E061E075E0CF010E948D0F9E
:10475000FE012F2D207830E040E050E060E070E076
:1047600080E090E0A0E00E94058951F0EF012196E1
:104770004CEC58E067E075E0CF010E948D0FFE0120
:1047800020E0302F317040E050E060E070E080E0E9
:1047900090E0A0E00E94058951F0EF0121964CECD9
:1047A00058E06AE075E0CF010E948D0FFE0120E025
:1047B000302F327040E050E060E070E080E090E048
:1047C000A0E00E94058951F0EF0121964CEC58E0E1
:1047D0006FE075E0CF010E948D0FFE0120E0302FC9
:1047E000347040E050E060E070E080E090E0A0E0F5
:1047F0000E94058951F0EF0121964CEC58E066E1EA
:1048000075E0CF010E948D0FFE0120E0302F38703F
:1048100040E050E060E070E080E090E0A0E00E94C6
:10482000058951F0EF0121964CEC58E069E175E003
:10483000CF010E948D0FFE0120E0302F307140E04B
:1048400050E060E070E080E090E0A0E00E94058928
:1048500051F0EF0121964CEC58E06EE175E0CF018C
:104860000E948D0FFE0120E0302F307240E050E0BA
:1048700060E070E080E090E0A0E00E94058951F0E7
:10488000EF0121964CEC58E065E275E0CF010E9403
:104890008D0FFE018091C51F81FF17C020E0302FD2
:1048A000307440E050E060E070E080E090E0A0E034
:1048B0000E94058951F0EF0121964CEC58E06CE222
:1048C00075E0CF010E948D0FFE018091C51F909170
:1048D000C61F90FF17C020E030E040E05E2D507111
:1048E00060E070E080E090E0A0E00E94058951F077
:1048F000EF0121964CEC58E06FE275E0CF010E9489
:104900008D0FFE018091C51F9091C61F90FF17C0AB
:1049100020E030E040E05E2D507260E070E080E02A
:1049200090E0A0E00E94058951F0EF0121964CEC47
:1049300058E062E375E0CF010E948D0FFE01809187
:10494000C51F9091C61F90FF17C020E030E040E0E7
:104950005E2D507460E070E080E090E0A0E00E9486
:10496000058951F0EF0121964CEC58E068E375E0C1
:10497000CF010E948D0FFE0120E0302F307840E003
:1049800050E060E070E080E090E0A0E00E940589E7
:1049900051F0EF0121964CEC58E063E475E0CF0153
:1049A0000E948D0FFE0120E030E0412F417050E069
:1049B00060E070E080E090E0A0E00E94058951F0A6
:1049C000EF0121964CEC58E068E475E0CF010E94BD
:1049D0008D0FFE0120E030E0412F427050E060E09A
:1049E00070E080E090E0A0E00E94058951F0EF01C6
:1049F00021964CEC58E06BE475E0CF010E948D0FDE
:104A0000FE0120E030E0412F447050E060E070E0B3
:104A100080E090E0A0E00E94058951F0EF0121962E
:104A20004CEC58E06EE475E0CF010E948D0FFE0162
:104A30008091C51F87FF17C020E030E0412F4870EC
:104A400050E060E070E080E090E0A0E00E94058926
:104A500051F0EF0121964CEC58E061E575E0CF0193
:104A60000E948D0FFE018091C51F87FF17C020E0B7
:104A700030E0412F407150E060E070E080E090E075
:104A8000A0E00E94058951F0EF0121964CEC58E01E
:104A900065E575E0CF010E948D0FFE018091C51F75
:104AA00087FF17C020E030E0412F407250E060E007
:104AB00070E080E090E0A0E00E94058951F0EF01F5
:104AC00021964CEC58E069E575E0CF010E948D0F0E
:104AD000FE018091C51F87FF17C020E030E0412F05
:104AE000407450E060E070E080E090E0A0E00E9460
:104AF000058951F0EF0121964CEC58E06DE575E029
:104B0000CF010E948D0FFE018091C51F82FF17C04B
:104B100020E030E0412F407850E060E070E080E03D
:104B200090E0A0E00E94058951F0EF0121964CEC45
:104B300058E06CE176E0CF010E948D0FFE0180917C
:104B4000C51F82FF17C020E030E040E05E2D5170AD
:104B500060E070E080E090E0A0E00E94058951F004
:104B6000EF0121964CEC58E061E675E0CF010E9420
:104B70008D0FFE018091C51F9091C61F90FF17C039
:104B800020E030E040E05E2D527060E070E080E0B8
:104B900090E0A0E00E94058951F0EF0121964CECD5
:104BA00058E064E675E0CF010E948D0FFE01809110
:104BB000C51F9091C61F90FF17C020E030E040E075
:104BC0005E2D547060E070E080E090E0A0E00E9414
:104BD000058951F0EF0121964CEC58E06CE675E048
:104BE000CF010E948D0FFE018091C51F9091C61FBD
:104BF00091FF1EC020E030E040E05E2D587060E084
:104C000070E080E090E0A0E00E94058989F04CEC23
:104C100058E065E775E0CF01DF91CF911F910F91CB
:104C2000FF90EF90DF90CF90BF90AF900C948D0FDE
:104C30002F2D302F412F5E2DB501C601A0E00E941F
:104C4000058941F481E596E09F938F930E94968DAC
:104C50000F900F90DF91CF911F910F91FF90EF90E8
:104C6000DF90CF90BF90AF900895AF92BF92DF9248
:104C7000EF920F931F93CF93DF93EC015B01FB0146
:104C800010826CE476E00E94B78C892B59F58091F4
:104C9000C51F7DE4D72EE0E8EE2E82FD02C004E0C1
:104CA00001C004E810E081FF02C060ECE62E26E0BF
:104CB0004AE250E06BE270E089E290E00E94AA577D
:104CC00081E090E00E94CC0A882311F05DE5D52EAA
:104CD0008091C51F9091C61F90FD16E091FF06C000
:104CE000186004C0D12CE12C00E010E06AE476E00A
:104CF000CE010E94B78C892B61F481E0F50180839D
:104D000060916B0270916C0280E090E00E94CB8C0D
:104D1000EC0168E476E0CE010E94B78C892B61F447
:104D20008FEFF501808360916B0270916C0280E0DF
:104D300090E00E94CB8CEC01209709F41AC164E446
:104D400076E0CE010E94B78C892B19F4FD2DF1601D
:104D5000DF2E60E476E0CE010E94B78C892B19F437
:104D60008D2D8460D82E6DE376E0CE010E94B78C45
:104D7000892B19F4ED2DE260DE2E6BE376E0CE0197
:104D80000E94B78C892B19F4FD2DF860DF2E68E3A3
:104D900076E0CE010E94B78C892B19F48D2D8061AD
:104DA000D82E62E376E0CE010E94B78C892B19F4ED
:104DB000ED2DE062DE2E6CE276E0CE010E94B78C33
:104DC000892B19F4FD2DF064DF2E69E276E0CE0127
:104DD0000E94B78C892B19F48D2D8068D82E64E23F
:104DE00076E0CE010E94B78C892B19F4EE2DE1609C
:104DF000EE2E6DE176E0CE010E94B78C892B19F47E
:104E0000FE2DF260EF2E6AE176E0CE010E94B78CB3
:104E1000892B19F48E2D8460E82E65E176E0CE01B1
:104E20000E94B78C892B19F4EE2DE860EE2E6EE00F
:104E300076E0CE010E94B78C892B19F4FE2DF0612B
:104E4000EF2E67E076E0CE010E94B78C892B19F433
:104E50008E2D8062E82E64E076E0CE010E94B78C51
:104E6000892B19F4EE2DE064EE2E6FEF75E0CE0184
:104E70000E94B78C892B19F4FE2DF068EF2E6CEF91
:104E800075E0CE010E94B78C892B09F4016069EFAF
:104E900075E0CE010E94B78C892B09F4026066EFA1
:104EA00075E0CE010E94B78C892B09F4046062EF93
:104EB00075E0CE010E94B78C892B09F408606EEE74
:104EC00075E0CE010E94B78C892B09F400616AEE6F
:104ED00075E0CE010E94B78C892B09F4006266EE62
:104EE00075E0CE010E94B78C892B09F4006464EE52
:104EF00075E0CE010E94B78C892B09F4006861EE41
:104F000075E0CE010E94B78C892B09F4116069ED20
:104F100075E0CE010E94B78C892B09F4126060ED18
:104F200075E0CE010E94B78C892B09F4146067EC00
:104F300075E0CE010E94B78C892B09F4186064ECEF
:104F400075E0CE010E94B78C892B09F410616EEBDD
:104F500075E0CE010E94B78C892B09F4106263EBD7
:104F600075E0CE010E94B78C892B09F0DCCE10646D
:104F7000DACE2D2D3E2DA80160E070E080E090E0BB
:104F8000DF91CF911F910F91EF90DF90BF90AF9085
:104F900008955F926F927F928F929F92AF92BF928D
:104FA000CF92DF92EF92FF920F931F93CF93DF93F5
:104FB000782ECFECDAE100E010E0FDEAEF2EF5E02C
:104FC000FF2E8170582E872D8270682EA8E9CA2E78
:104FD000A5E0DA2EB0EAAB2EB5E0BB2E8EE9882E26
:104FE00085E0982E772051F01F930F93FF92EF9258
:104FF0000E94968D0F900F900F900F905520A1F06A
:1050000089858F9388858F93BF92AF920E94968DEA
:105010000F900F900F900F906620C1F09F928F928B
:105020000E94968D0F900F90662081F0DF92CF92B4
:105030000E94968D288139814A815B816C817D81B6
:105040008E819F810E94EC220F900F900E943E0B58
:105050000F5F1F4F2A960430110521F6DF91CF9183
:105060001F910F91FF90EF90DF90CF90BF90AF9086
:105070009F908F907F906F905F900895CF9388E876
:1050800095E09F938F930E94968D0E94551F86EB0B
:105090009AE19F938F9380E895E09F938F930E946E
:1050A000968D8CE795E09F938F930E94968D80E07C
:1050B0000E94332187E795E09F938F930E94968DFE
:1050C0000E94B50F8091C51F2DB73EB7265F3F4F99
:1050D0000FB6F8943EBF0FBE2DBF80FF05C041E064
:1050E00061E081E00E945F110E94591F809153028C
:1050F0001F928F938EE695E09F938F930E94968DDB
:10510000809169091F928F9385E695E09F938F9315
:105110000E94968DC0E4CF9383E18F9383E38F93B6
:105120008F9381E595E09F938F930E94968D1F92B8
:10513000CF9389E395E09F938F930E94968D809102
:1051400057281F928F93809156281F928F9386E243
:1051500095E09F938F930E94968D809152021F92AB
:105160008F938DE195E09F938F930E94968D809110
:105170005402909155022DB73EB7245E3F4F0FB6B3
:10518000F8943EBF0FBE2DBF96FF03C08EE795E09B
:1051900002C081E895E09F938F9383E195E09F9310
:1051A0008F930E94968D83E00E94C9270F900F90E5
:1051B0000F900F901D9B03C08EE795E002C081E821
:1051C00095E09F938F9387E095E09F938F930E9444
:1051D000968D8DEF94E09F938F930E94968D809192
:1051E00054020F900F900F900F900F900F9081FF2F
:1051F00009C087EF94E09F938F930E94968D0F9044
:105200000F9013C080FF03C08EE795E002C081E8D5
:1052100095E09F938F9383EF94E09F938F930E94E9
:10522000968D0F900F900F900F9080915402909157
:10523000550297FF03C08EE795E002C081E895E034
:105240009F938F938AEE94E09F938F930E94968D05
:1052500083EE94E09F938F930E94968D60916D09E9
:1052600070916E0980E090E00E9463210E943E0BE5
:105270000F900F900F900F900F900F90779903C0A1
:105280008EE795E002C081E895E09F938F938AEDC9
:1052900094E09F938F930E94968D0E94E5080E9450
:1052A000880A9F938F937F936F938CEC94E09F93E6
:1052B0008F930E94968D0E94420A9F938F937F93B3
:1052C0006F938EEB94E09F938F930E94968D81E075
:1052D00090E00E940F2080912C2890912D28A09181
:1052E0002E28B0912F28BF93AF939F938F9380EB7D
:1052F00094E09F938F930E94968D809141288F9385
:10530000809140288F9380913F288F9380913E28F1
:105310008F938CE994E09F938F930E94968D809158
:10532000302890913128A0913228B0913328BF9332
:10533000AF939F938F938EE894E09F938F930E94F7
:10534000968D8DB79EB782960FB6F8949EBF0FBE0E
:105350008DBF809145288F93809144288F938091B1
:1053600043288F93809142288F938AE794E09F93FC
:105370008F930E94968D61E070E080E090E00E9443
:10538000470B0F900F900F900F900F900F9061E0D0
:1053900070E081E090E0CF910C94470BF894E0E04E
:1053A000F0E081E2809357008491E2E0F0E041E296
:1053B000409357004491E4E0F0E091E2909357006D
:1053C000E49190E0A0E0B0E0DC019927882750E06C
:1053D00060E070E0762F652F542F4427840F951FCF
:1053E000A61FB71F8E0F911DA11DB11D8093701BAD
:1053F0009093711BA093721BB093731B78940895C4
:10540000CF93DF93CDB7DEB761970FB6F894DEBFC9
:105410000FBECDBF48E250E068E170E08FEC9AE14A
:105420000E94EA8E2091CF1A3091D01A4091D11A61
:105430005091D21A6091D31A7091D41A8091D51AD2
:105440009091D61AAFEF0E94058909F05DC08DE4F6
:105450008093CF1A80E88093D01A84E08093D11A89
:105460001092D21A1092D31A1092D41A1092D51AFE
:105470001092D61A8CE390E09093D81A8093D71AA2
:105480001092D91A1092DA1A1092DB1A1092DC1AC2
:105490001092DD1A1092DE1A1092DF1A1092E01AA2
:1054A0001092E21A1092E11A1092E31A1092E41A82
:1054B0001092E51A1092E61A1092E71A1092E81A62
:1054C0001092E91A1092EA1A1092EC1A1092EB1A42
:1054D0001092ED1A1092EE1A1092EF1A1092F01A22
:1054E0001092F11A1092F21A1092F31A1092F41A02
:1054F0001092F61A1092F51A48E250E068E170E056
:105500008FEC9AE10E94088F42E050E066E170E083
:10551000CE010F960E94EA8E8F8598898F3F2FEFDC
:10552000920779F48AE090E49093550280935402B4
:1055300042E050E066E170E084E592E00E94088F6E
:1055400004C0909355028093540242E050E06CE412
:1055500070E0CE010F960E94EA8E8F8598898F3F6A
:105560002FEF920769F410926E0910926D0942E0D4
:1055700050E06CE470E08DE699E00E94088F04C072
:1055800090936E0980936D0949E050E06AE070E005
:1055900086E498E20E94EA8E0E947F0C44E050E08C
:1055A00064E470E0CE010B960E94EA8E8B859C85A8
:1055B000AD85BE8544E050E064E470E08F3F9F4FCE
:1055C000AF4FBF4F29F482E792E00E94088F04C0DA
:1055D00082E792E00E94EA8E44E050E060E470E0EE
:1055E000CE010B960E94EA8E8B859C85AD85BE858B
:1055F00044E050E060E470E08F3F9F4FAF4FBF4FFB
:1056000029F48EE692E00E94088F04C08EE692E0B4
:105610000E94EA8E44E050E068E470E0CE010B9610
:105620000E94EA8E8B859C85AD85BE8544E050E066
:1056300068E470E08F3F9F4FAF4FBF4F29F486E77C
:1056400092E00E94088F04C086E792E00E94EA8EF2
:1056500041E050E065E170E0CE0141960E94EA8EA3
:10566000898941E050E065E170E08F3F29F489E6E7
:1056700099E00E94088F04C089E699E00E94EA8EB2
:1056800041E050E064E170E0CE0141960E94EA8E74
:10569000898941E050E064E170E08F3F29F483E5BF
:1056A00092E00E94088F04C083E592E00E94EA8E97
:1056B00041E050E063E170E0CE0141960E94EA8E45
:1056C000898941E050E063E170E08F3F29F482E591
:1056D00092E00E94088F04C082E592E00E94EA8E68
:1056E0004AE050E060E070E0CE0101960E94EA8E50
:1056F00089814AE050E060E070E08F3F29F486EB5A
:105700009AE10E94088F04C086EB9AE10E94EA8E1B
:1057100061960FB6F894DEBF0FBECDBFDF91CF917B
:105720000895CF92DF92EF92FF9260916B02709199
:105730006C0280E090E00E94CB8C65E875E00E94EE
:10574000DF8C892B09F0F1C08DE48093CF1A80E8BB
:105750008093D01A84E08093D11A1092D21A1092BA
:10576000D31A1092D41A1092D51A1092D61A8CE32A
:1057700090E09093D81A8093D71A1092D91A109269
:10578000DA1A1092DB1A1092DC1A1092DD1A1092BB
:10579000DE1A1092DF1A1092E01A1092E21A10929A
:1057A000E11A1092E31A1092E41A1092E51A10927C
:1057B000E61A1092E71A1092E81A1092E91A10925B
:1057C000EA1A1092EC1A1092EB1A1092ED1A10923B
:1057D000EE1A1092EF1A1092F01A1092F11A10921B
:1057E000F21A1092F31A1092F41A1092F61A1092FA
:1057F000F51A48E250E068E170E08FEC9AE10E940F
:10580000088F8AE090E4909355028093540242E01E
:1058100050E066E170E084E592E00E94088F10920B
:105820006E0910926D0942E050E06CE470E08DE684
:1058300099E00E94088F42E2C42EDD24DA944CECF9
:10584000E42E4BE3F42EC0927202D0927302E092E7
:105850007402F092750244E050E064E470E082E784
:1058600092E00E94088FC0926E02D0926F02E09286
:105870007002F092710244E050E060E470E08EE665
:1058800092E00E94088F87ED94E3AFEEBCE3809333
:10589000760290937702A0937802B093790244E065
:1058A00050E068E470E086E792E00E94088F109272
:1058B000690980E00E94166541E050E065E170E012
:1058C00089E699E00E94088F8AE1809353020E9442
:1058D000BD6341E050E064E170E083E592E00E9446
:1058E000088F8FE08093520241E050E063E170E066
:1058F00082E592E00E94088F8AE0E6EBFAE1DF01A0
:105900001D928A95E9F74AE050E060E070E0CF012F
:105910000E94088F81E00E94332180E090E0FF9098
:10592000EF90DF90CF900C94930CFF90EF90DF906E
:10593000CF9008952F923F924F925F926F927F92F5
:105940008F929F92AF92BF92CF92DF92EF92FF928F
:105950000F931F93CF93DF93CDB7DEB72B970FB67F
:10596000F894DEBF0FBECDBF9B878A874A01FC013A
:1059700080819181892B11F00C94513D60916B02D3
:1059800070916C02CA010E94CB8C60E470E0C4018B
:105990000E94FE8C009759F4609111317091123180
:1059A0008AE090E00E94528D81E00C94563D813057
:1059B000910561F4F401B0801B2D110F110B012F23
:1059C000412E512E612E712EA12EBCC08230910528
:1059D000B9F4F4018081992787FD9095982F882745
:1059E0002181820F911D27FD9A95B82E192F092F1D
:1059F000000F000B402E502E602E702EA02EA2C045
:105A000083309105B1F5F4012081922F990F990B04
:105A1000392F492F592F692F792F892F00E10E94A3
:105A2000A78819012A013B01B82FA92F2181922FA4
:105A3000990F990B392F492F592F692F792F892FBA
:105A400008E00E94A78859016A017B018C0191013D
:105A5000A201B3018B2F9A2F0E94DE88A2801A2DFB
:105A6000110F110BB12EC12ED12EE12EF12E012FCF
:105A700055C004970CF45DC0F4012081922F990F5A
:105A8000990B392F492F592F692F792F892F08E129
:105A90000E94A78819012A013B01B82FA92F218153
:105AA000922F990F990B392F492F592F692F792F41
:105AB000892F00E10E94A78859016A017B018C01AE
:105AC0009101A201B3018B2F9A2F0E94DE88A3803F
:105AD0001A2D110F110BB12EC12ED12EE12EF12E48
:105AE000012F0E94DE8819012A013B01B82FA92F3E
:105AF0002281922F990F990B392F492F592F692FF6
:105B0000792F892F08E00E94A78859016A017B013B
:105B10008C019101A201B3018B2F9A2F0E94DE8884
:105B2000B22E132F042F452E562E672E782EA92E17
:105B300009C07AE0B72E10E000E0412C512C612C16
:105B4000712CA12C0E943E0B2B2D312F402F542D58
:105B5000652D762D872D9A2D2736FFE63F07FCE62B
:105B60004F075105610571058105910511F40C94EC
:105B7000A6372736EFE63E07ECE64E0751056105EE
:105B800071058105910511F008F093C12936F2E7FE
:105B90003F0741055105610571058105910511F426
:105BA0000C948F3A2936E2E73E074105510561051D
:105BB00071058105910511F008F0A3C02536F4E6C2
:105BC0003F0741055105610571058105910509F4FE
:105BD00074C52536E4E63E074105510561057105AA
:105BE0008105910509F0A8F5A6E70E94058909F449
:105BF0006CC70E94058909F060F4A8E60E94058937
:105C000009F4A1C5A5E70E94058909F448C70C94C9
:105C10004F3D2B2D312F402F542D652D762D872D67
:105C20009A2D2A33F6E23F074105510561057105BA
:105C30008105910509F412C3243631464105510509
:105C4000610571058105910511F40C94083B0C94D4
:105C50004F3D2B2D312F402F542D652D762D872D27
:105C60009A2D2737FFE63F0741055105610571056C
:105C70008105910511F40C94C3382737EFE63E07F0
:105C800041055105610571058105910509F0C0F4D3
:105C90002436F9E63F074105510561057105810587
:105CA000910509F4D5C625363E46410551056105E5
:105CB00071058105910511F40C94F7380C944F3D52
:105CC0002B2D312F402F542D652D762D872D9A2D7C
:105CD0002333F1E73F074105510561057105810552
:105CE000910511F40C94083B2536324741055105C6
:105CF000610571058105910511F40C94B1390C947D
:105D00004F3D2B2D312F402F542D652D762D872D76
:105D10009A2D2837F4E63F07F1E64F075105610554
:105D200071058105910509F4A9C22837E4E63E070B
:105D3000E1E64E075105610571058105910511F0F8
:105D400008F050C02837F4E73F07410551056105C9
:105D500071058105910509F481C22837E4E73E0702
:105D600041055105610571058105910509F0C8F4EA
:105D70002337F2E73F0741055105610571058105AC
:105D8000910511F40C94E03A23373347410551054E
:105D9000610571058105910511F40C94F43A0C9498
:105DA0004F3D2B2D312F402F542D652D762D872DD6
:105DB0009A2D2133F4E63F07F1E64F0751056105BF
:105DC00071058105910509F45DC2233634464146CB
:105DD0005105610571058105910511F40C94083B8D
:105DE0000C944F3D2B2D312F402F542D652D762DAA
:105DF000872D9A2D2336FDE63F07F8E64F0751051C
:105E0000610571058105910509F460C22336EDE64F
:105E10003E07E8E64E0751056105710581059105CC
:105E200009F0C8F42236F5E63F07F4E64F075105BE
:105E3000610571058105910509F43FC42237324798
:105E400045465105610571058105910511F40C94D4
:105E500028380C944F3D2B2D312F402F542D652D7C
:105E6000762D872D9A2D2336F2E33F07F9E64F076B
:105E70005105610571058105910509F423C2243698
:105E8000E3E63E07ECE64E07510561057105810525
:105E9000910511F40C94A3372D363547484651052A
:105EA000610571058105910511F00C944F3D0C942D
:105EB0001E3B2B2D312F402F542D652D762D872DF8
:105EC0009A2D2037ECE63E07E5E64E07E8E65E074A
:105ED000610571058105910509F435C42037FCE69B
:105EE0003F07F5E64F07F8E65F0761057105810595
:105EF000910511F008F0CDC02437E8E73E07E4E74C
:105F00004E075105610571058105910509F444C6E7
:105F10002437F8E73F07F4E74F075105610571059E
:105F20008105910511F008F055C02133E1E33E07EA
:105F3000E1E74E075105610571058105910511F4F1
:105F40000C945D382133F1E33F07F1E74F0751052A
:105F5000610571058105910509F0D0F42537E3E667
:105F60003E07EDE64E075105610571058105910576
:105F700011F40C945D3820333143414751056105DC
:105F800071058105910511F40C9428380C944F3D4E
:105F90002B2D312F402F542D652D762D872D9A2DA9
:105FA0002037E5E63E07E2E74E075105610571053A
:105FB0008105910511F40C94B1392C3634474447CE
:105FC0005105610571058105910511F40C948C3C16
:105FD0000C944F3D2B2D312F402F542D652D762DB8
:105FE000872D9A2D2936ECE63E07E1E64E07E3E6DB
:105FF0005E07610571058105910509F49CC129368B
:10600000FCE63F07F1E64F07F3E65F076105710520
:106010008105910509F0E0F42437E4E63E07E7E75F
:106020004E075105610571058105910511F40C9428
:10603000DA3C24373F464F465246610571058105DB
:10604000910511F00C944F3D0C9400000C94513DBF
:106050002B2D312F402F542D652D762D872D9A2DE8
:106060002E36E1E63E07E8E64E07E3E65E07610509
:1060700071058105910509F465C526333946454703
:106080005546610571058105910509F460C30C94BD
:106090004F3D2B2D312F402F542D652D762D872DE3
:1060A0009A2D2136ECE63E07E5E64E07E2E75E076D
:1060B000610571058105910509F466C32136FCE689
:1060C0003F07F5E64F07F2E75F07610571058105B8
:1060D000910511F008F057C02337E5E63E07E2E7E7
:1060E0004E07E0E75E07610571058105910511F432
:1060F0000C94CE3B2337F5E63F07F2E74F07F0E776
:106100005F07610571058105910509F0D0F421361D
:10611000EDE63E07E5E74E07E8E65E076105710537
:106120008105910511F40C94E13822373747404737
:106130005047610571058105910509F4CBC00C94A8
:106140004F3D2B2D312F402F542D652D762D872D32
:106150009A2D2337E2E73E07E7E74E07E0E75E07C1
:10616000610571058105910511F40C94743924368B
:106170003D4643465247610571058105910509F485
:106180008CC30C944F3D2B2D312F402F542D652D5A
:10619000762D872D9A2D2737E0E73E07E8E74E0753
:1061A000E4E75E07610571058105910509F4A2C464
:1061B0002737F0E73F07F8E74F07F4E75F07610588
:1061C00071058105910509F0D0F42437E3E73E0716
:1061D000E5E64E07E2E75E07610571058105910579
:1061E00011F40C94713924373347454654476105FF
:1061F00071058105910509F4F8C40C944F3D2B2DD0
:10620000312F402F542D652D762D872D9A2D223735
:10621000E7E63E07E0E74E07E5E75E076105710543
:106220008105910509F46CC62C36F1E63F07F4E7C9
:106230004F07F8E75F07610571058105910511F4C6
:106240000C94563C24373247414655476105710549
:106250008105910511F00C944F3D70C383E080934C
:106260003428109236281092352844E358E262E12F
:1062700084E392E00E942F4F0C94513D0E944315FD
:106280000C94513D21E042E161E080ED0E945A5CB6
:1062900021E042E161E080ED0E945A5C21E042E1B0
:1062A00061E080ED0E945A5C21E042E161E080ED16
:1062B0000E945A5C21E042E161E080ED0E945A5C5C
:1062C0000C94513D0E94B50F0C94513D0E94BB159A
:1062D0000C94513D60916B0270916C0280E090E0F3
:1062E0000E94CB8C8C016EE775E00E94DF8C892BBD
:1062F00019F477980C94513D61E875E0C8010E944B
:10630000DF8C892B19F4779A0C94513D779903C04F
:106310008EE795E002C081E895E09F938F9384E635
:1063200094E09F938F930E94968D0F900F900F9003
:106330000F900C94513D60916B0270916C0280E063
:1063400090E00E94CB8C8C0168E475E00E94DF8CA9
:10635000892B09F077C060916B0270916C0280E02C
:1063600090E00E94CB8C8C01009711F40C94513D6D
:106370006CE875E00E94DF8C892BB1F482E29FEF1C
:10638000ACECBBE38093720290937302A09374020F
:10639000B093750244E050E064E470E082E792E07C
:1063A0000E94088F0C94513D62E975E0C8010E947B
:1063B000DF8C892BB1F482E29FEFACECBAE38093DF
:1063C000720290937302A0937402B093750244E03A
:1063D00050E064E470E082E792E00E94088F0C9441
:1063E000513DC8010E94B58B2B013C0120E030E0FB
:1063F000A9010E9454838823D9F081E00E94DF091B
:106400009B01AC01C301B2010E94588360937202E8
:1064100070937302809374029093750244E050E08D
:1064200064E470E082E792E00E94088F0C94513D92
:1064300088ED92E09F938F930E94968D0F900F901E
:106440000C94513D6BE475E0C8010E94DF8C892BF0
:1064500009F077C060916B0270916C0280E090E06F
:106460000E94CB8C8C01009711F40C94513D6CE888
:1064700075E00E94DF8C892BB1F482E29FEFACECD7
:10648000BBE380936E0290936F02A0937002B0936F
:10649000710244E050E060E470E08EE692E00E9419
:1064A000088F0C94513D62E975E0C8010E94DF8CB1
:1064B000892BB1F482E29FEFACECBAE380936E02D9
:1064C00090936F02A0937002B093710244E050E089
:1064D00060E470E08EE692E00E94088F0C94513DDB
:1064E000C8010E94B58B2B013C0120E030E0A901DE
:1064F0000E9454838823D9F082E00E94DF099B0127
:10650000AC01C301B2010E94588360936E02709384
:106510006F02809370029093710244E050E060E457
:1065200070E08EE692E00E94088F0C94513D8BEC57
:1065300092E09F938F930E94968D0F900F900C94F2
:10654000513D63E475E0C8010E94DF8C892B09F09E
:1065500073C060916B0270916C0280E090E00E94C9
:10656000CB8C8C01009711F40C94513D6CE875E0D4
:106570000E94DF8C892BB1F487ED94E3AFEEBCE38E
:106580008093760290937702A0937802B093790279
:1065900044E050E068E470E086E792E00E94088FF3
:1065A0000C94513D62E975E0C8010E94DF8C892B93
:1065B00051F48CEB92E09F938F930E94968D0F90F5
:1065C0000F900C94513DC8010E94B58B2B013C01EA
:1065D00020E030E0A9010E945483882319F180E073
:1065E0000E94DF094B015C0121EE3AE744E95EE3DA
:1065F000C301B2010E948D82A50194010E945883BB
:106600006093760270937702809378029093790278
:1066100044E050E068E470E086E792E00E94088F72
:106620000C94513D8FEA92E09F938F930E94968D38
:106630000F900F900C94513D0E942E0A9F938F93C0
:106640007F936F9388EA92E09F938F930E94968D39
:1066500082E00E94DF0920916E0230916F0240912A
:106660007002509171020E94D585162F072FF82EC7
:10667000E92E81E00E94DF09EF92FF920F931F93B2
:106680002091720230917302409174025091750210
:106690000E94D5859F938F937F936F938CE992E0AF
:1066A0009F938F930E94968D0E943E0B0FB6F89495
:1066B000DEBF0FBECDBF0C94513D60916B02709157
:1066C0006C0280E090E00E94CB8C0097C1F00E94A9
:1066D000512220916D0930916E098217930709F1BB
:1066E00090936E0980936D0942E050E06CE470E095
:1066F0008DE699E00E94088F8DE594E002C086E562
:1067000094E09F938F930E94968D60916D09709194
:106710006E0980E090E00E9463210E943E0B0F9082
:106720000F908BE494E09F938F930E94968D6FEF70
:106730007FEF80E090E00E9463210E943E0B0F906B
:106740000F900C94513D0E94701E0C94513DF40129
:106750008481843329F440E061E080E00E945F118D
:1067600080916D02882311F40C94513D1F928F93F8
:1067700088E494E09F938F930E94968D0F900F90E2
:106780000F900F900C94513DF4018481893709F0EA
:1067900070C060916B0270916C0280E090E00E948A
:1067A000CB8C8C016EE775E00E94DF8C892B31F475
:1067B000809154029091550290640CC061E875E09C
:1067C000C8010E94DF8C892B91F480915402909132
:1067D00055029F7B909355028093540242E050E013
:1067E00066E170E084E592E00E94088F42C067E9AC
:1067F00075E0C8010E94DF8C892B21F58091CE1AAB
:106800008F938091CD1A8F938091CC1A8F93809122
:10681000CB1A8F938091CA1A8F938091C91A8F9344
:106820008091C81A8F938091C71A8F9381E792E065
:106830009F938F930E94968D0FB6F894DEBF0FBE84
:10684000CDBF17C0809154029091550296FF03C0AE
:106850008EE795E002C081E895E09F938F938DE6E7
:1068600092E09F938F930E94968D0F900F900F90C0
:106870000F9080916D02882311F40C94513D1F926A
:106880008F9385E494E09F938F930E94968D0F9051
:106890000F900F900F900C94513D60916B0270918E
:1068A0006C0280E090E00E94CB8C5C016EE775E0AA
:1068B0000E94DF8C0091540210915502892B11F433
:1068C000106808C061E875E0C5010E94DF8C892B63
:1068D00071F41F77109355020093540242E050E088
:1068E00066E170E084E592E00E94088F13C017FF14
:1068F00003C08EE795E002C081E895E09F938F93F7
:1069000089E692E09F938F930E94968D0F900F904F
:106910000F900F9080916D02882311F40C94513DDB
:106920001F928F9382E494E09F938F930E94968DA1
:106930000F900F900F900F900C94513D60916B024F
:1069400070916C0280E090E00E94CB8C5C016DE95C
:1069500075E00E94DF8C892B11F489E108C061EA9F
:1069600075E0C5010E94DF8C892B49F480E180939A
:10697000C4001092C50082E08093C00055C065EA53
:1069800075E0C5010E94DF8C892B11F488E0EFCF00
:106990006AEA75E0C5010E94DF8C892B39F06FEA45
:1069A00075E0C5010E94DF8C892B11F483E0DFCFF5
:1069B0008091C400893141F484E692E09F938F93E3
:1069C0000E94968D0F900F908091C400803141F409
:1069D0008FE592E09F938F930E94968D0F900F907A
:1069E0008091C400883041F489E592E09F938F93B1
:1069F0000E94968D0F900F908091C400833041F4D7
:106A000083E592E09F938F930E94968D0F900F9055
:106A10008091C400883041F48DE492E09F938F937D
:106A20000E94968D0F900F9080916D02882311F433
:106A30000C94513D1F928F938FE394E09F938F931B
:106A40000E94968D0F900F900F900F900C94513DD7
:106A500060916B0270916C0280E090E00E94CB8CA0
:106A60006CE875E00E94DF8C892B11F481E001C095
:106A700080E00E94332180916D02882311F40C94F0
:106A8000513D1F928F938CE394E09F938F930E94CC
:106A9000968D0F900F900F900F900C94513D0E9487
:106AA000591F80916D02882311F40C94513D1F925F
:106AB0008F9389E394E09F938F930E94968D0F901C
:106AC0000F900F900F900C94513D0E94551F809194
:106AD0006D02882311F40C94513D1F928F9386E32D
:106AE00094E09F938F930E94968D0F900F900F903C
:106AF0000F90D7C760916B0270916C0280E090E0BC
:106B00000E94CB8C0E94B98B803168F48093690914
:106B10000E94166541E050E065E170E089E699E089
:106B20000E94088FBEC7809169091F928F9383E4EA
:106B300092E09F938F930E94968D0F900F900F90ED
:106B40000F90AFC760916B0270916C0280E090E093
:106B50000E94CB8C0E94B98B95EF980F903168F40E
:106B6000809353020E94BD6341E050E064E170E015
:106B700083E592E00E94088F94C7809153021F9290
:106B80008F938AE392E09F938F930E94968D0F904C
:106B90000F900F900F9085C760916B0270916C02FF
:106BA00080E090E00E94CB8C009781F04AE050E0BA
:106BB000BC0186EB9AE10E94EF8C4AE050E060E075
:106BC00070E086EB9AE10E94088F6BC786EB9AE132
:106BD0009F938F9384EB95E09F938F930E94848D76
:106BE0000F900F900F900F905CC760916B027091A7
:106BF0006C0280E090E00E94CB8C5C0164ED73E05D
:106C00000E94DF8C892B99F4219A809154029091F3
:106C100055028061909355028093540242E050E007
:106C200066E170E084E592E00E94088F3AC76CE468
:106C300075E0C5010E94DF8C892B99F4229A80911E
:106C400054029091550280629093550280935402B1
:106C500042E050E066E170E084E592E00E94088F37
:106C600020C766EB73E0C5010E94DF8C892B99F485
:106C7000239A80915402909155028064909355021A
:106C80008093540242E050E066E170E084E592E0D7
:106C90000E94088F06C763EF74E0C5010E94DF8C75
:106CA000892B99F4239A809154029091550280681F
:106CB000909355028093540242E050E066E170E008
:106CC00084E592E00E94088FECC665E179E0C50199
:106CD0000E94DF8C892B31F581E08093D8238FECE3
:106CE0009AE19093DA238093D9231092DC231092B7
:106CF000DB2380915402909155029160909355024C
:106D00008093540242E050E066E170E084E592E056
:106D10000E94088F48ED53E262E184E392E00E9412
:106D20002F4FBFC66DED73E0C5010E94DF8C892B2C
:106D3000D1F4EFEFFAE1119211923BE1EF31F30759
:106D4000D1F7809154029091550292609093550230
:106D50008093540242E050E066E170E084E592E006
:106D60000E94088F9EC661E875E0C5010E94DF8C15
:106D70002091540230915502892BA1F42F703C7F51
:106D800030935502209354022B9A42E050E066E182
:106D900070E084E592E00E94088F80913D280E9477
:106DA000D2637FC624FF03C08EE795E002C081E86E
:106DB00095E09F938F938FE292E09F938F930E9431
:106DC000968D809154020F900F900F900F9085FF39
:106DD00003C08EE795E002C081E895E09F938F9312
:106DE00084E292E09F938F930E94968D809154024B
:106DF0000F900F900F900F9086FF03C08EE795E0E5
:106E000002C081E895E09F938F9389E192E09F9380
:106E10008F930E94968D809154020F900F900F9047
:106E20000F9087FF03C08EE795E002C081E895E0F0
:106E30009F938F938EE092E09F938F930E94968D05
:106E400080915402909155020F900F900F900F90E7
:106E500090FF03C08EE795E002C081E895E09F9324
:106E60008F9383E092E09F938F930E94968D809101
:106E70005402909155020F900F900F900F9091FF38
:106E800003C08EE795E002C081E895E09F938F9361
:106E900088EF91E09F938F930E94968D809154028A
:106EA000909155020F900F900F900F9091FFF9C5A0
:106EB0008CEB95E00E94BA8D5FEFA52E5AE1B52EBE
:106EC0000BE010E064EC862E65E0962EF5018081E3
:106ED0009181F2E0AF0EB11C9F938F931F930F939C
:106EE0009F928F920E94848D0F5F1F4F0F900F9083
:106EF0000F900F900F900F900B31110539F7D1C5FE
:106F000082E394E09F938F930E94968D80916D020F
:106F10000F900F90882361F01F928F938FE294E07F
:106F20009F938F930E94968D0F900F900F900F90CC
:106F300088E10FB6F89480936000109260000FBE55
:106F40000C94007CAEC50E940B5CABC560916B02DB
:106F500070916C0280E090E00E94CB8C8C016EE717
:106F600075E00E94DF8C892BA9F40E94BC6280919D
:106F70005402909155028D7F8160909355028093C9
:106F8000540242E050E066E170E084E592E00E9445
:106F9000088F87C561E875E0C8010E94DF8C892BE6
:106FA000A1F40E94746280915402909155028C7FEA
:106FB000909355028093540242E050E066E170E005
:106FC00084E592E00E94088F6CC56FEC75E0C80103
:106FD0000E94DF8C892BA9F40E9474628091540274
:106FE000909155028E7F8260909355028093540257
:106FF00042E050E066E170E084E592E00E94088F94
:1070000050C58091540281FF0FC08FEC95E09F9393
:107010008F9384EF91E09F938F930E94968D0F90B2
:107020000F900F900F903DC580FF03C08EE795E055
:1070300002C081E895E09F938F9380EF91E09F934A
:107040008F930E94968D0F900F900F900F9029C5EF
:107050008091D6238F938091D5238F938091D423D1
:107060008F938091D3238F938091D2238F9380919C
:10707000D1238F938091D0238F938091CF238F93AF
:1070800081E194E09F938F930E94968D80916D0291
:107090000FB6F894DEBF0FBECDBF882309F401C53B
:1070A0001F928F938EE094E09F938F930E94968D12
:1070B0000F900F900F900F90F4C4F89481E090E03F
:1070C00029E0FC0120935700C895E02C80E090E077
:1070D000FC0120935700C895F02C7894F89483E035
:1070E00090E0FC0120935700C895002D82E090E0CD
:1070F000FC0120935700C895102D78948091731B44
:107100008F938091721B8F938091711B8F938091CD
:10711000701B8F9324E034E03F932F930E94968D51
:107120001F92EF921F92FF921F920F931F921F9335
:107130008DED93E09F938F930E94968D0E94F31F95
:10714000809166001F928F9381ED93E09F938F93C0
:107150000E94968D0E943E0B80916D020FB6F894AE
:10716000DEBF0FBECDBF882309F49BC41F928F934F
:107170008EEC93E09F938F930E94968D0F900F90CB
:107180000F900F908EC460E070E080E090E00E946D
:10719000470B60E070E081E090E00E94470B809137
:1071A0006D02882309F47DC41F928F938BEC93E0CA
:1071B0009F938F930E94968D0F900F900F900F903A
:1071C00070C40E94331E0E943E0B80916D02882382
:1071D00009F467C41F928F9388EC93E09F938F9379
:1071E0000E94968D0F900F900F900F905AC460914F
:1071F0006B0270916C0280E090E00E94CB8C64ED99
:1072000075E00E94DF8C892B31F5F89484EA99E0CF
:107210000E941C505C01009769F0C5010F960E9406
:107220002053B50184E092E00E94D64FC5010E9430
:10723000C450F0CF84EA99E00E94A950892B29F02C
:1072400084EA99E00E945550F5CF84EA99E00E94C3
:107250001850789434C084EA99E00E941C505C0174
:107260000AED15E0A114B10451F1F50186811F92D8
:107270008F9380851F928F9385811F928F93818535
:107280001F928F9387811F928F9384811F928F9378
:1072900083811F928F9382811F928F9382851F9289
:1072A0008F931F930F930E94848DC5010E94C45039
:1072B0005C010FB6F894DEBF0FBECDBFD3CF809177
:1072C0006D02882309F4EDC31F928F9385EC93E040
:1072D0009F938F930E94968D0F900F900F900F9019
:1072E000E0C30E94912BDDC360916B0270916C0230
:1072F00080E090E00E94CB8C8C0169E176E00E94F6
:10730000DF8C892B91F48091540290915502977FE4
:10731000909355028093540242E050E066E170E0A1
:1073200084E592E00E94088FBCC362E975E0C80161
:107330000E94DF8C892B91F4809154029091550228
:107340009860909355028093540242E050E066E1C9
:1073500070E084E592E00E94088FA3C30E94E508D4
:10736000A0C360916B0270916C0280E090E00E947B
:10737000CB8CFC0120812332B1F44AE050E060E084
:1073800070E001960E946D891B0160916B02709103
:107390006C0280E090E00E94CB8CF4E02F16310468
:1073A0000CF094C002C0212C312C009709F48EC03F
:1073B0001982BE016F5F7F4F0E94352629013A0175
:1073C0004B01B82FA92F8AE0829DF001839DF00D1B
:1073D0001124E153F54E20812A8331813B83828140
:1073E0008C8393819D8324812E8335813F83868185
:1073F0008887978199879201A301B4018B2F9A2FD7
:10740000AA80BB80CC80DD80EE80FF800885198556
:107410000E94FC8809F45DC08981882351F18CF0B9
:107420002A81422A3B81532A8C81682A9D81792AAC
:107430002E81822A3F81932A8885B82B9985A92B92
:1074400018C0409450946094709480949094B09537
:10745000A0952A8142223B8153228C8168229D8102
:1074600079222E8182223F8193228885B8239985B3
:10747000A923408251826282738284829582B6837C
:10748000A78348E250E068E170E08FEC9AE10E9447
:10749000088F8DEB93E09F938F930E94968D8AE0E7
:1074A000829DF001839DF00D1124E153F54E208162
:1074B00031814281538164817581868197810E94E7
:1074C000EC220E943E0B0F900F9003C082E00E94BE
:1074D000C92781EB93E09F938F930E94968D2FEFA6
:1074E0003FEF4FEF5FEF60E070E080E090E00E94E0
:1074F000EC220E943E0B80916D020F900F9088232A
:1075000009F4CFC21F928F938EEA93E09F938F93DB
:107510000E94968D0F900F900F900F90C2C26091B5
:107520006B0270916C0280E090E00E94CB8CFC01B9
:1075300020812332A1F44AE050E060E070E001963F
:107540000E946D898B0160916B0270916C0280E0EA
:1075500090E00E94CB8C04301105ECF402C000E0F6
:1075600010E00097C1F04AE050E060E070E00E9457
:10757000A18A2AE0209FF001219FF00D1124E15300
:10758000F54E7187608748E250E068E170E08FEC6B
:107590009AE10E94088F81E00E94C92780916D02C4
:1075A000882309F47EC21F928F938BEA93E09F9306
:1075B0008F930E94968D0F900F900F900F9071C235
:1075C0000E94595380916D02882309F46AC21F9268
:1075D0008F9388EA93E09F938F930E94968D0F90EC
:1075E0000F900F900F905DC20E943E2880916D0217
:1075F000882309F456C21F928F9385EA93E09F93E4
:107600008F930E94968D0F900F900F900F9049C20C
:1076100080E090E00E940F2080916D02882309F4A1
:1076200040C21F928F9382EA93E09F938F930E94B0
:10763000968D0F900F900F900F9033C28091C51FC1
:1076400081FF2DC00E94BB1D892B49F58091BC1B79
:107650008F938091BB1B8F938091BA1B8F938091E6
:10766000B91B8F9387E993E09F938F930E94968D28
:10767000809155288F93809154288F93809153281F
:107680008F93809152288F938AE893E09F938F93F2
:107690000E94968D0FB6F894DEBF0FBECDBF0E943C
:1076A0003E0B8091C51F9091C61F90FF63C081E083
:1076B00090E00E946B1D3B014C0180E090E00E9435
:1076C0006B1D1B012C010E94EA1C9F928F927F92DE
:1076D0006F9289E793E09F938F930E94968D5F92BC
:1076E0004F923F922F9289E693E09F938F930E944F
:1076F000968D222D332D442D552D662D772D882DD9
:10770000992D0E94D11B9F938F937F936F938EE54A
:1077100093E09F938F930E94968D222D332D442DBD
:10772000552D662D772D882D992D0E94321C9F9303
:107730008F937F936F9380E593E09F938F930E9445
:10774000968D222D332D442D552D662D772D882D88
:10775000992D0E94931C9F938F937F936F938DE33A
:1077600093E09F938F930E94968D0FB6F894DEBF9F
:107770000FBECDBF0E943E0B80916D02882309F49D
:1077800090C11F928F938AE393E09F938F930E94FF
:10779000968D0F900F900F900F9083C18091C51F11
:1077A00082FF2BC021E048E061E083E00E94D41218
:1077B0008091B71B8F938091B61B8F938091B51BDF
:1077C0008F938091B41B8F938091B31B8F93809183
:1077D000B21B8F938091B11B8F938091B01B8F93BD
:1077E00083E293E09F938F930E94968D0E943E0BBD
:1077F0000FB6F894DEBF0FBECDBF8091C51F90912C
:10780000C61F91FF41C00E941E17B62EA72E982EAC
:10781000892E20E030E048EC52E4D501F4016B2FD2
:107820007A2F8F2F9E2F0E94D58520E836EE45ECCB
:1078300057E40E94588321E03EED42E45EE30E945B
:1078400038869B01AC0160E070E080E89FE30E9415
:107850008D822BE43AE34DEB57E30E9458839F93CC
:107860008F937F936F938F929F92AF92BF928AE094
:1078700093E09F938F930E94968D0E943E0B0FB6CC
:10788000F894DEBF0FBECDBF80916D02882309F44E
:1078900008C11F928F9387E093E09F938F930E947C
:1078A000968D0F900F900F900F90FBC060916B0220
:1078B00070916C0280E090E00E94CB8C6EE176E0EB
:1078C0000E94DF8C892BB1F460916B0270916C0285
:1078D00080E090E00E94CB8C009709F4E2C00E9407
:1078E000B98B803108F0DDC090915201982B9093B4
:1078F0005201D7C0809152018F701F928F9383EEF7
:1079000091E09F938F930E94968D0E943E0B0F9063
:107910000F900F900F90C5C060916B0270916C0238
:1079200080E090E00E94CB8C009711F14AE050E09B
:1079300060E070E00E946D89603198F460935202BB
:107940001F926F938AEF92E09F938F930E94968D80
:1079500041E050E063E170E082E592E00E94088F30
:1079600011C0809152021F928F9381EF92E006C066
:10797000809152021F928F9388EE92E09F938F9393
:107980000E94968D0F900F900F900F900E943E0BCB
:1079900080916D02882309F484C01F928F9385EE35
:1079A00092E09F938F930E94968D0F900F900F906F
:1079B0000F9077C060916B0270916C0280E090E054
:1079C0000E94CB8C8C016EE775E00E94DF8C892BC6
:1079D000A1F40E942561809154029091550290611A
:1079E000909355028093540242E050E066E170E0CB
:1079F00084E592E00E94088F54C061E875E0C801F8
:107A00000E94DF8C892B41F5F8940E94336188E154
:107A10000FB6F89480936000109260000FBE84B798
:107A2000877F84BF8091600088618093600010929E
:107A30006000789480915402909155029F7E9093BB
:107A400055028093540242E050E066E170E084E524
:107A500092E00E94088F25C063E276E0C8010E9490
:107A6000DF8C2091540230915502892B21F434FF90
:107A700018C0F894FFCF34FF03C08EE795E002C032
:107A800081E895E09F938F938FED91E09F938F9383
:107A90000E94968D0F900F900F900F9002C00E9441
:107AA000571EEA85FB851182108283E02B960FB664
:107AB000F894DEBF0FBECDBFDF91CF911F910F9124
:107AC000FF90EF90DF90CF90BF90AF909F908F90FE
:107AD0007F906F905F904F903F902F9008950F93FD
:107AE0001F93CF93DF93EC018A01888199810097DE
:107AF00011F18C389F4021F01982188283E020C058
:107B00006231E9F4A80162E170E085E999E00E9440
:107B10009A2C84E0809334281092362810923528CD
:107B2000109338280093372844E358E262E184E355
:107B300092E00E942F4F8CE89FE09983888381E038
:107B4000DF91CF911F910F9108950E9419616C9A56
:107B50006B9A6A9A6F9A729A749A739A779A8098C3
:107B600080B3897F80BB8398849887E080937E0070
:107B7000549A0E94CE290E94002A81E00E94530953
:107B800080E090E00E94930C0E94905A0E94420A6A
:107B90006093C7237093C8238093C9239093CA230B
:107BA0008091540286FD239A0895CF93DF93EC01D0
:107BB00088819981009741F087379F4009F47BC005
:107BC0001982188283E082C00E94A53D80915402F0
:107BD00080FD05C081FF01C01D9B0E9474628091E1
:107BE00070008C7F809370008091B60080628093DB
:107BF000B6001092B20082E08093B1008091B6008E
:107C00008770E1F7809170008160809370006FEF62
:107C100078E080E090E00E9403610E94551F80E0C0
:107C20000E94332180E29EE09F938F930E94968D65
:107C30000E94B50F8091C51F0F900F9086FD0E9486
:107C4000B75B809169090E941665809153020E947A
:107C5000BD630E94BA6380939409809153020E948D
:107C6000BD63809169091F928F93809194091F923F
:107C70008F9388E296E09F938F930E94848D109259
:107C80009609109295090F900F900F900F900F90FA
:107C90000F9088E492E09093502880934F2883E2DD
:107CA00090E09093A7118093A61187E79FE09983B6
:107CB000888381E00BC06332E1F74CEE53E260E071
:107CC00070E085E999E00E949A2CE3CFDF91CF9193
:107CD00008958436910514F19F938F938AE396E07B
:107CE0009F938F930E94848D8091CF239091D02376
:107CF000A091D123B091D2230196A11DB11D8093F3
:107D0000CF239093D023A093D123B093D2230F906D
:107D10000F900F900F9081E090E0089580E090E048
:107D200008952F923F924F925F926F927F928F921F
:107D30009F92AF92BF92CF92DF92EF92FF920F93FA
:107D40001F93CF93DF93CDB7DEB7C859D1090FB6D4
:107D5000F894DEBF0FBECDBFC157DF4F9983888334
:107D6000CF58D0408A01633871F489E999E0C95647
:107D7000DF4F6883C759D0400E94724DC956DF4F0C
:107D80006881C759D040C157DF4FA881B981CF580A
:107D9000D0402D913C912B32BFE03B0709F483C3C7
:107DA00040F42115310581F021383D4009F4C1C36B
:107DB000B5C32C334FE0340709F491C323343F405B
:107DC00011F40C94894AAAC340EE52E061E870E0D5
:107DD00089E999E00E94584D81E89DE05BC3E3E0AA
:107DE000F0E0EC0FFD1FE00FF11F1082C8010E94B0
:107DF000693E892B89F720E030E040E050E0652DB6
:107E0000627070E080E090E0A0E00E94058909F0D7
:107E1000CAC5C257DF4F2881CE58D040287030E005
:107E200040E050E060E070E080E090E0A0E00E9480
:107E30000589A1F127E04AE250E06BE270E089E2B7
:107E400090E00E94AA5786E498E20E94185ABC016A
:107E5000882777FD8095982F0E94F78320E030E0F7
:107E600048EC52E40E9458839F938F937F936F93C3
:107E70008EE696E09F938F931F9287E78F93CE01B4
:107E8000800F911F03969F938F930E94E78D080F99
:107E9000191F0FB6F894DEBF0FBECDBFC257DF4F1C
:107EA0002881CE58D040207130E040E050E060E0C2
:107EB00070E080E090E0A0E00E940589F1F126E00A
:107EC0004AE250E06BE270E089E290E00E94AA573B
:107ED00081E090E00E94CC0A8093680988E29BE1EF
:107EE0000E94185ABC01882777FD8095982F0E9420
:107EF000F78320E030E048EC52E40E9458839F93DF
:107F00008F937F936F9388E796E09F938F931F9251
:107F100087E78F93C8010296E1E0F0E0EC0FFD1FC8
:107F20008E0F9F1F9F938F930E94E78D080F191F3D
:107F30000FB6F894DEBF0FBECDBFC657DF4F288106
:107F4000CA58D04030E040E050E060E070E080E0AF
:107F500090E0A0E00E94058901F10E94880A9F93A9
:107F60008F937F936F9383E896E09F938F931F92F5
:107F700087E78F93C801029641E050E04C0F5D1FE8
:107F8000840F951F9F938F930E94E78D080F191FF1
:107F90000FB6F894DEBF0FBECDBFC257DF4F2881AA
:107FA000CE58D040207430E040E050E060E070E017
:107FB00080E090E0A0E00E94058931F18091CA2321
:107FC0008F938091C9238F938091C8238F93809141
:107FD000C7238F9381E996E09F938F931F9287E742
:107FE0008F93C8010296A1E0B0E0AC0FBD1F8A0FCD
:107FF0009B1F9F938F930E94E78D080F191F0FB649
:10800000F894DEBF0FBECDBFC257DF4F2881CE58D8
:10801000D040207830E040E050E060E070E080E068
:1080200090E0A0E00E94058941F1F89480912C280D
:1080300090912D28A0912E28B0912F287894BF934D
:10804000AF939F938F938FE996E09F938F931F92A7
:1080500087E78F93C801029621E030E02C0F3D1F87
:10806000820F931F9F938F930E94E78D080F191F14
:108070000FB6F894DEBF0FBECDBF20E0372D3170B4
:1080800040E050E060E070E080E090E0A0E00E941E
:10809000058909F099C420E0372D327040E050E0A6
:1080A00060E070E080E090E0A0E00E94058909F0C7
:1080B00013C520E0372D347040E050E060E070E000
:1080C00080E090E0A0E00E94058909F036C520E03C
:1080D000372D387040E050E060E070E080E090E0E4
:1080E000A0E00E94058909F057C520E0372D3071C6
:1080F00040E050E060E070E080E090E0A0E00E94AE
:10810000058909F0D1C520E0372D307240E050E0FC
:1081100060E070E080E090E0A0E00E94058909F056
:10812000F3C520E0CD56DF4F3881C359D04040E041
:1081300050E060E070E080E090E0A0E00E940589FF
:1081400009F00FC620E0CC56DF4F3881C459D0402B
:1081500040E050E060E070E080E090E0A0E00E944D
:10816000058909F02CC620E030E0482D417050E030
:1081700060E070E080E090E0A0E00E94058909F0F6
:108180004CC620E030E0482D427050E060E070E0E6
:1081900080E090E0A0E00E94058909F071C620E02F
:1081A00030E0CE56DF4F4881C259D04050E060E009
:1081B00070E080E090E0A0E00E94058909F093C69D
:1081C00020E030E0482D487050E060E070E080E052
:1081D00090E0A0E00E94058909F0AFC620E030E001
:1081E000482D407150E060E070E080E090E0A0E059
:1081F0000E94058909F0D1C620E030E0482D407288
:1082000050E060E070E080E090E0A0E00E9405892E
:1082100009F0F3C620E030E0482D407450E060E003
:1082200070E080E090E0A0E00E94058909F015C7A9
:10823000F82DF078EF2E20E030E04F2F50E060E096
:1082400070E080E090E0A0E00E94058909F035C769
:10825000292D2170F22E20E030E040E05F2D60E01B
:1082600070E080E090E0A0E00E94058909F02FC74F
:1082700020E030E04E2D50E060E070E080E090E0E3
:10828000A0E00E94058909F02DC720E030E040E021
:108290005F2D60E070E080E090E0A0E00E94058942
:1082A00009F052C720E030E040E0592D527060E004
:1082B00070E080E090E0A0E00E94058909F076C7B8
:1082C00020E030E040E0592D547060E070E080E044
:1082D00090E0A0E00E94058909F098C720E030E016
:1082E00040E0592D507160E070E080E090E0A0E047
:1082F0000E94058909F0BAC720E030E040E0592D1E
:10830000507260E070E080E090E0A0E00E9405899B
:1083100009F0E9C720E030E040E0592D507460E0FA
:1083200070E080E090E0A0E00E94058911F00C94DC
:10833000B04920E030E040E0592D587060E070E036
:1083400080E090E0A0E00E94058911F00C94EF49D4
:1083500020E030E040E0CB56DF4F5881C559D04097
:1083600060E070E080E090E0A0E00E94058911F0FC
:108370000C94204A779A80916D0990916E0992FD34
:10838000749AC257DF4F2881CE58D040372DA401B0
:10839000652DCF56DF4F7881C159D040842D962D61
:1083A000A0E0FE0133967F010E94058911F00C9434
:1083B000574A809152028061898380918D098A8316
:1083C000F701E00FF11F108280916D0990916E0905
:1083D00098012D5F3F4F790180FF0CC0FF922F93D2
:1083E00080E098E09F938F930E94848D0F900F9070
:1083F0000F900F90B701CE0101960E94A156809177
:10840000540282FF0AC02CE234E2A701BE016F5F72
:108410007F4F8BE592E00E94275B80916D099091E0
:108420006E0982FD73980E94BC6289E999E00E94FE
:10843000744D809154029091550290FF3BC00F5FA4
:108440001F4F0E94BA63F82E89E10E94D2632091E7
:1084500054023091550230FF29C0739880918D09E4
:108460008F5F80938D098A83B8016F5F7F4FCE0144
:1084700001960E94A15689E999E00E94744D40E05E
:1084800050E065E88091AA119091AB110E942F4FA6
:108490008BE29FE0C157DF4FA881B981CF58D04010
:1084A0008D939C9338C000E010E0D1CF8F2D0E94B7
:1084B000D263739A80916A0990916B09892B11F0AC
:1084C0000E94746280918D098F5F80938D098091E5
:1084D0006D0990916E0982FF7FCC739A7DCC85E8FF
:1084E00099E00E94D551892BB1F00E94BC62809125
:1084F000540287FD2B9860E470E085E899E00E94C3
:10850000AE5183E49FE0C157DF4FE881F981CF5836
:10851000D0409183808381E00C949C4AC157DF4F07
:10852000A881B981CF58D0401D921C9283E00C9451
:108530009C4A623181F7809154029091550291FDDD
:108540004BCC23E333E343E150E46091C7237091C4
:10855000C8238091C9239091CA230E94548387FF26
:1085600014C08091D3239091D423A091D523B091AE
:10857000D6230196A11DB11D8093D3239093D423BC
:10858000A093D523B093D62327CCF80180818130E6
:10859000D1F40180F281E02D2081C257DF4F288382
:1085A000CE58D04071808280938054803581CF56E0
:1085B000DF4F3883C159D0404680678020843184A2
:1085C000A12CB12C3DC0823081F4A380B480212C39
:1085D000312CB1E0C257DF4FB883CE58D040712C58
:1085E000812C20E8922E512C24C0833099F08430C5
:1085F00009F0F2CB212C312CA12CB12CE5E0C25793
:10860000DF4FE883CE58D040712C812C912C92E022
:10861000592E0FC0212C312CA12CB12CF5E0C257C2
:10862000DF4FF883CE58D040712C812C912C5524EB
:108630005394CF56DF4F1882C159D040412C612C42
:10864000282D2470CE56DF4F2883C259D04020E019
:1086500030E0CE56DF4F4881C259D04050E060E054
:1086600070E080E090E0A0E00E94058909F08C9A1B
:10867000C257DF4F3881CE58D0403072C657DF4FD7
:108680003883CA58D040232F30E040E050E060E00B
:1086900070E080E090E0A0E00E94058911F00E9467
:1086A000880A472D4074CD56DF4F4883C359D040C8
:1086B00020E0342F40E050E060E070E080E090E0A7
:1086C000A0E00E94058911F00E94BB1D572D507833
:1086D000CC56DF4F5883C459D04020E0352F40E0BE
:1086E00050E060E070E080E090E0A0E00E9405894A
:1086F00051F00E942E0A6093392870933A28809393
:108700003B2890933C28C257DF4F2881CE58D04059
:10871000217030E040E050E060E070E080E090E008
:10872000A0E00E940589F1F086EB9AE19F938F9378
:108730008EE496E09F938F931F9287E78F93CE01ED
:1087400003969F938F930E94E78D7C010E94693E60
:108750000FB6F894DEBF0FBECDBF892B09F03CCB1E
:10876000870102C000E010E0C257DF4F2881CE58D9
:10877000D040227030E040E050E060E070E080E007
:1087800090E0A0E00E94058909F442C0C801029669
:1087900066E576E0A1E0B0E0AC0FBD1F8A0F9B1F3D
:1087A0000E94E88C0D5F1F4FB6E4CB2EB8E2DB2EA3
:1087B00086EEE82E83E0F82E27E7F60181916F011F
:1087C0001F928F93FF92EF921F922F93C8010296F0
:1087D00041E050E04C0F5D1F840F951F9F938F93D6
:1087E000C856DF4F2883C859D0400E94E78D080F34
:1087F000191F0FB6F894DEBF0FBECDBFC856DF4FAE
:108800002881C859D0407EE4C71678E2D706A9F679
:10881000C257DF4F2881CE58D040247030E040E06E
:1088200050E060E070E080E090E0A0E00E94058908
:1088300009F461C0C80102966AE576E0A1E0B0E003
:10884000AC0FBD1F8A0F9B1F0E94E88C0C5F1F4F4F
:108850007E01BAE7EB0EF11C80E1F70111928A95D7
:10886000E9F728E0A70168E980EB0E941811670189
:10887000F8E0CF0ED11C46EE53E027E7D7018D91EB
:108880007D011F928F935F934F931F922F93C80187
:108890000296E1E0F0E0EC0FFD1F8E0F9F1F9F930B
:1088A0008F93C856DF4F2883C859D040CA56DF4F30
:1088B0004883C659D040C956DF4F5883C759D04066
:1088C0000E94E78D080F191F0FB6F894DEBF0FBE88
:1088D000CDBFC856DF4F2881C859D040CA56DF4F98
:1088E0004881C659D040C956DF4F5881C759D0403A
:1088F000EC14FD0419F6792D7078CB56DF4F788390
:10890000C559D04020E030E040E0572F60E070E0F3
:1089100080E090E0A0E00E940589E1F480916A097E
:1089200090916B099F938F938FE596E09F938F9320
:108930001F9287E78F93CE01800F911F03969F931D
:108940008F930E94E78D080F191F0FB6F894DEBFB2
:108950000FBECDBF20E030E040E050E0652D6170FB
:1089600070E080E090E0A0E00E94058909F443CA2D
:10897000E3E0F0E0EC0FFD1FE00FF11F80E28083E9
:10898000EFEEF3E280810F5F1F4F882309F427CABF
:108990008081A1E0B0E0AC0FBD1FA00FB11F129607
:1089A0008C933196EFCFCE01800F911F66E676E073
:1089B00003960E94E88C095F1F4FC8010E94693E20
:1089C000892B09F009CA25CA2114310409F463CBA3
:1089D000F89460912C2870912D2880912E289091E8
:1089E0002F28C657DF4F688379838A839B83CA58B1
:1089F000D04078948091201B9091211BA091221B44
:108A0000B091231BC657DF4F288139814A815B8192
:108A1000CA58D040281B390B4A0B5B0BCA01B9015D
:108A20000E94F5836B017C01B10180E090E00E941F
:108A3000F5839B01AC01C701B6010E9458837C01FC
:108A4000FF928F937F936F938AEA96E09F938F9321
:108A50001F9287E78F939E01200F311F2D5F3F4F9D
:108A60003F932F93C956DF4F6883C759D040CA56EA
:108A7000DF4F7883C659D0400E94E78D080F191F39
:108A8000C956DF4F6881C759D040CA56DF4F788139
:108A9000C659D040862F972FAE2DBF2D80933E28EC
:108AA00090933F28A0934028B0934128C657DF4FAA
:108AB000488159816A817B81CA58D0404093201BEC
:108AC0005093211B6093221B7093231B0FB6F894C5
:108AD000DEBF0FBECDBFDFCA2114310409F4E9CADD
:108AE000F8948091F71A9091F81AA091F91AB09120
:108AF000FA1A78949F938F93809159028F93809163
:108B000058028F9387EB96E09F938F931F9287E78E
:108B10008F93C8010296A1E0B0E0AC0FBD1F8A0F91
:108B20009B1F9F938F930E94E78D080F191F0FB60D
:108B3000F894DEBF0FBECDBFBCCAF8948091302838
:108B400090913128A0913228B09133287894BF9326
:108B5000AF939F938F9387EC96E09F938F931F9291
:108B600087E78F93C801029621E030E02C0F3D1F6C
:108B7000820F931F9F938F930E94E78D080F191FF9
:108B8000C8010E94693E0FB6F894DEBF0FBECDBF8C
:108B9000892B09F021C99BCA2114310409F4A5CA03
:108BA000F89460913028709131288091322890910A
:108BB0003328C657DF4F688379838A839B83CA58DB
:108BC000D04078948091241B9091251BA091261B66
:108BD000B091271BC657DF4F288139814A815B81BD
:108BE000CA58D040281B390B4A0B5B0BCA01B9018C
:108BF0000E94F5836B017C01B10180E090E00E944E
:108C0000F5839B01AC01C701B6010E9458837C012A
:108C1000FF928F937F936F9382ED96E09F938F9354
:108C20001F9287E78F939E01200F311F2D5F3F4FCB
:108C30003F932F93C956DF4F6883C759D040CA5618
:108C4000DF4F7883C659D0400E94E78D080F191F67
:108C5000C956DF4F6881C759D040CA56DF4F788167
:108C6000C659D040862F972FAE2DBF2D8093422816
:108C700090934328A0934428B0934528C657DF4FCC
:108C8000488159816A817B81CA58D0404093241B16
:108C90005093251B6093261B7093271B0FB6F894E7
:108CA000DEBF0FBECDBF21CA232809F42CCAF89419
:108CB0008091FB1A9091FC1AA091FD1AB091FE1AB6
:108CC00078949F938F93809157028F93809156024F
:108CD0008F938FED96E09F938F931F9287E78F93EB
:108CE000C8010296A1E0B0E0AC0FBD1F8A0F9B1F28
:108CF0009F938F930E94E78D080F191F0FB6F8946A
:108D0000DEBF0FBECDBFFFC98091CB239091CC2396
:108D1000A091CD23B091CE23BF93AF939F938F9318
:108D20008FEE96E09F938F931F9287E78F93C801F2
:108D3000029621E030E02C0F3D1F820F931F9F937E
:108D40008F930E94E78D080F191FC8010E94693E8A
:108D50000FB6F894DEBF0FBECDBF892B09F03CC81B
:108D6000E0C98091BC1B8F938091BB1B8F93809136
:108D7000BA1B8F938091B91B8F938AEF96E09F93D4
:108D80008F931F9287E78F93C801029661E070E08E
:108D90006C0F7D1F860F971F9F938F930E94E78D07
:108DA000080F191FC8010E94693E0FB6F894DEBF74
:108DB0000FBECDBF892B11F00C94EC3EC3C980913E
:108DC0003C288F9380913B288F9380913A288F93F2
:108DD000809139288F9385E097E09F938F931F921E
:108DE00087E78F93C8010296E1E0F0E0EC0FFD1FEA
:108DF0008E0F9F1F9F938F930E94E78D080F191F5F
:108E0000C8010E94693E0FB6F894DEBF0FBECDBF09
:108E1000892B11F00C94EC3EA6C981E00E94DF0979
:108E20002091720230917302409174025091750248
:108E30000E94D5859F938F937F936F9382E197E0F4
:108E40009F938F931F9287E78F93C801029641E00B
:108E500050E04C0F5D1F840F951F9F938F930E94CE
:108E6000E78D080F191FC8010E94693E0FB6F894DC
:108E7000DEBF0FBECDBF892B11F00C94EC3E81C933
:108E800082E00E94DF0920916E0230916F024091D2
:108E90007002509171020E94D5859F938F937F93AA
:108EA0006F938FE197E09F938F931F9287E78F9344
:108EB000C8010296A1E0B0E0AC0FBD1F8A0F9B1F56
:108EC0009F938F930E94E78D080F191FC8010E947E
:108ED000693E0FB6F894DEBF0FBECDBF892B11F0EF
:108EE0000C94EC3E5CC983E00E94DF099F938F9352
:108EF0007F936F938CE297E09F938F931F9287E706
:108F00008F93C801029621E030E02C0F3D1F820FA5
:108F1000931F9F938F930E94E78D080F191F8C98C2
:108F2000C8010E94693E0FB6F894DEBF0FBECDBFE8
:108F3000892B11F00C94EC3E43C98091C51F87FF2B
:108F40004DC921E042E161E080ED0E945A5C9F93AF
:108F50008F937F936F9389E397E09F938F931F92F3
:108F600087E78F93C801029661E070E06C0F7D1F68
:108F7000860F971F9F938F930E94E78D080F191FED
:108F8000C8010E94693E0FB6F894DEBF0FBECDBF88
:108F9000892B11F00C94EC3E21C98091C51F87FFED
:108FA0002BC921E042E162E080ED0E945A5C9F9370
:108FB0008F937F936F9387E497E09F938F931F9294
:108FC00087E78F93C8010296E1E0F0E0EC0FFD1F08
:108FD0008E0F9F1F9F938F930E94E78D080F191F7D
:108FE000C8010E94693E0FB6F894DEBF0FBECDBF28
:108FF000892B11F00C94EC3EFFC88091C51F87FFB0
:1090000009C921E042E163E080ED0E945A5C9F9330
:109010008F937F936F9385E597E09F938F931F9234
:1090200087E78F93C801029641E050E04C0F5D1F27
:10903000840F951F9F938F930E94E78D080F191F30
:10904000C8010E94693E0FB6F894DEBF0FBECDBFC7
:10905000892B11F00C94EC3EDDC88091C51F87FF71
:10906000E7C821E042E164E080ED0E945A5C9F93F2
:109070008F937F936F9383E697E09F938F931F92D5
:1090800087E78F93C8010296A1E0B0E0AC0FBD1F47
:109090008A0F9B1F9F938F930E94E78D080F191FC4
:1090A000C8010E94693E0FB6F894DEBF0FBECDBF67
:1090B000892B11F00C94EC3EBBC88091C51F82FF38
:1090C000C7C846E061E083E00E94D412C1C8809125
:1090D000C51F82FFCDC821E046E061E083E00E9429
:1090E000D412C6C88091C51F82FFCFC88091B31B20
:1090F0008F938091B21B8F938091B11B8F9380913E
:10910000B01B8F9381E797E09F938F931F9287E720
:109110008F93C801029641E050E04C0F5D1F840F11
:10912000951F9F938F930E94E78D080F191FC80109
:109130000E94693E0FB6F894DEBF0FBECDBF892BEB
:1091400011F00C94EC3EA1C88091C51F82FFAAC803
:109150008091B71B8F938091B61B8F938091B51B25
:109160008F938091B41B8F9389E797E09F938F93A0
:109170001F9287E78F93C8010296A1E0B0E0AC0F81
:10918000BD1F8A0F9B1F9F938F930E94E78D080F2F
:10919000191FC8010E94693E0FB6F894DEBF0FBECA
:1091A000CDBF892B11F00C94EC3E7CC88091C51F7B
:1091B0009091C61F90FF84C880E090E00E946B1DD4
:1091C0009F938F937F936F9384E897E09F938F9300
:1091D0001F9287E78F93C801029621E030E02C0FA1
:1091E0003D1F820F931F9F938F930E94E78D080F5F
:1091F000191FC8010E94693E0FB6F894DEBF0FBE6A
:10920000CDBF892B11F00C94EC3E5AC88091C51F3C
:109210009091C61F90FF62C881E090E00E946B1D94
:109220009F938F937F936F9384E997E09F938F939E
:109230001F9287E78F93C801029661E070E06C0F80
:109240007D1F860F971F9F938F930E94E78D080FB6
:10925000191FC8010E94693E0FB6F894DEBF0FBE09
:10926000CDBF892B11F00C94EC3E38C88091C51FFE
:109270009091C61F90FF40C881E090E00E946B1D56
:109280006B017C0180E090E00E946B1D9B01AC01B2
:10929000C701B6010E94D11B9F938F937F936F9359
:1092A00085EA97E09F938F931F9287E78F93C8017A
:1092B0000296E1E0F0E0EC0FFD1F8E0F9F1F9F93E1
:1092C0008F930E94E78D080F191FC8010E94693E05
:1092D0000FB6F894DEBF0FBECDBF892B11F00C94F2
:1092E000EC3E0C947C418091C51F9091C61F90FF6D
:1092F00011C881E090E00E946B1D6B017C0180E051
:1093000090E00E946B1D9B01AC01C701B6010E9459
:10931000321C9F938F937F936F9380EB97E09F9383
:109320008F931F9287E78F93C801029641E050E028
:109330004C0F5D1F840F951F9F938F930E94E78DA5
:10934000080F191FC8010E94693E0FB6F894DEBFCE
:109350000FBECDBF892B11F00C94EC3E0C948A41CA
:109360008091C51F9091C61F90FD02C00C94994139
:1093700081E090E00E946B1D6B017C0180E090E039
:109380000E946B1D9B01AC01C701B6010E94931C9A
:109390009F938F937F936F938EEB97E09F938F9321
:1093A0001F9287E78F93C8010296A1E0B0E0AC0F4F
:1093B000BD1F8A0F9B1F9F938F930E94E78D080FFD
:1093C000191FC8010E94693E0FB6F894DEBF0FBE98
:1093D000CDBF892B11F00C94EC3E0C9499418091F7
:1093E000C51F9091C61F91FD02C00C94A8410E9418
:1093F0001E179F938F937F936F9381ED97E09F93B9
:109400008F931F9287E78F93C801029621E030E087
:109410002C0F3D1F820F931F9F938F930E94E78D08
:10942000080F191FC8010E94693E0FB6F894DEBFED
:109430000FBECDBF892B11F00C94EC3E0C94A841CB
:10944000D50116968C9116971F928F9315968C9135
:1094500015971F928F9313968C9113971F928F934A
:1094600012968C911F928F9382EE97E09F938F9329
:109470001F9287E78F93C8010296E1E0F0E0EC0FBE
:10948000FD1F8E0F9F1F9F938F930E94E78D080FE4
:10949000191FC8010E94693E0FB6F894DEBF0FBEC7
:1094A000CDBF892B11F00C94EC3E0C94BA41809105
:1094B0006D0990916E0982FD0CC08091540280FD6F
:1094C00008C081FD02C00C94D9411D9902C00C94C2
:1094D000D941FF92EF9289EF97E09F938F930E947B
:1094E000848D80916D020F900F900F900F908823C4
:1094F00011F40C94D9411F928F938DE19EE09F93BC
:109500008F930E94968D0F900F900F900F900C9458
:10951000D94185E899E00E94D551892B11F40C942A
:109520008B420E9474628091540287FD02C00C94A9
:10953000EC3E2B9A0C94EC3EC856DF4F0FB6F894D5
:10954000DEBF0FBECDBFDF91CF911F910F91FF9076
:10955000EF90DF90CF90BF90AF909F908F907F90D3
:109560006F905F904F903F902F9008950C949B4D7B
:109570004F925F926F927F928F929F92AF92BF9223
:10958000CF92DF92EF92FF920F931F93CF93DF93CF
:10959000CDB7DEB760970FB6F894DEBF0FBECDBF74
:1095A0006B010E94BA63E82FF0E0EE0FFF1FE75156
:1095B000F54E8081918101969183808380916D0920
:1095C00090916E0981FD749880905402909055029C
:1095D0000E94F5557C01FC018081982F92959F7027
:1095E000913099F48F7051F48091CD1A9091CE1AE8
:1095F00001969093CE1A8093CD1A00C1B60186E5EC
:1096000098E20E94114D892B51F08091CB1A9091D4
:10961000CC1A01969093CC1A8093CB1AEFC0C40158
:1096200084E0989F812D99271124F82FF1708F2EB7
:1096300084EA99E00E941C508C01009709F448C00C
:10964000B601C80102960E94114D892BE9F19801DB
:1096500049E159E060E074E6C8010F960E949C520F
:10966000F7019181F8018481981321C082858F5F71
:1096700082878091C91A9091CA1A01969093CA1A4A
:109680008093C91A84E00E941257F801208530E0C7
:109690002817390708F0A1C184E00E941257F80189
:1096A0008087F70180818F70F8018187A7C0F8015A
:1096B000128684E00E941257F8018087F7018081AA
:1096C0008F70F80181878AC1C8010E94C450B4CF4D
:1096D00084E092E00E94B14F8C01009709F48EC0A3
:1096E000B601C80102960E94084DF70181818150A0
:1096F000F801848380E091E0A0E0B0E08387948764
:10970000A587B687128684E00E941257F8018087E9
:10971000F70180818F70F8018187B80184EA99E0B0
:109720000E947C50980149E159E060E074E6C8016C
:109730000F960E949C5299249394F7018181F8011D
:109740008483F70180818F70F801878384E00E9411
:109750001257F801858383E00E9412575C01F801DB
:10976000868387818F3009F0912CF7014180F801C1
:109770008481481A512C612C712C56E0440C551CE4
:10978000661C771C5A95D1F7238534854585568507
:10979000A0ECB0E00E94B386BB27A92F982F872F9B
:1097A000480E591E6A1E7B1E438654866586768641
:1097B00080916D0990916E0981FD2AC080915402BB
:1097C00080FD26C081FD22C08091540290915502F7
:1097D00097FDCEC0992091F082E08093D82310921B
:1097E000DA231092D9231093DC230093DB2348ED76
:1097F00053E262E184E392E00E942F4F80916D0971
:1098000090916E0981FFECC0749AEAC01D9BDCCF79
:10981000A4E6B0E0A30192010E94B386672F782FDF
:10982000892F992724E630E040E050E00E94FE8630
:109830007F936F93452C562C672C77245F924F9221
:10984000BB24BF92AF92F80185811F928F93F701DD
:1098500080818F701F928F9381811F928F93F60169
:1098600081811F928F9380811F928F93C7010296EF
:109870009F938F9381E198E09F938F930E94848DB3
:1098800080916D020FB6F894DEBF0FBECDBF882366
:1098900061F01F928F938AE19EE09F938F930E94C5
:1098A000968D0F900F900F900F9080915402909191
:1098B000550296FF2DC0882059F1F7012081322FE3
:1098C0003F70832F90E00297D4F08FEF830F207FBB
:1098D000822B808389E999E00E94B64A8091C71A59
:1098E0009091C81A01969093C81A8093C71A8091D4
:1098F0006D0990916E0996FF0BC0739809C0809115
:10990000CD1A9091CE1A01969093CE1A8093CD1ACB
:109910008091C51F86FF58CF0E94A95BC70105969D
:109920000E94755BF70181811F928F93F8018681F8
:109930001F928F9385811F928F9385E598E09F9367
:109940008F931F9280E18F939E012F5F3F4F69019C
:10995000DF922F930E94E78D82E00E948F5BC60109
:109960000E94755B0FB6F894DEBF0FBECDBF2CCF43
:1099700086EB9AE12091B61A222309F42BCF9F930C
:109980008F9388E698E09F938F93FE0131966F0145
:10999000DF92EF930E94248E5C01B601C70102960C
:1099A0000E94098D0F900F900F900F900F900F90C5
:1099B000009709F40FCF95012F5F3F4F280F391FF4
:1099C000A9012F5F3F4FFA0180818032C9F362E124
:1099D0008CE092E00E942F4FFDCE812C912CADCED9
:1099E00060960FB6F894DEBF0FBECDBFDF91CF916A
:1099F0001F910F91FF90EF90DF90CF90BF90AF90AD
:109A00009F908F907F906F905F904F9008950895F2
:109A1000FB012081FC012083FB012181FC012183CA
:109A20000895FC019081DB018C91981309C081E0BD
:109A300090E0318111962C91321721F080E0089549
:109A400080E090E00895BC0186E598E20C94084D12
:109A5000DC011996ED91FC911A970280F381E02DBB
:109A6000309709F0099408950F931F93CF93DF93D4
:109A700000D0CDB7DEB78C0188E10E942557BC012C
:109A8000CE0101960E94084DD8011996ED91FC91E6
:109A90001A970190F081E02DBE016F5F7F4FC801E2
:109AA00009950F900F90DF91CF911F910F9108951D
:109AB000EF92FF920F931F93CF93DF93EC018B01F3
:109AC0007A0146EF52E00E94814DFA86E9866AEFFC
:109AD00072E0C801DF91CF911F910F91FF90EF903D
:109AE0000C94DA4D0C94994DCF93DF93EC0166E51D
:109AF00078E288E10E941B57CE01DF91CF910C9450
:109B00009B4DEF92FF920F931F93CF93DF93EC0146
:109B10008B017A010E94B64DF886EF826EEF72E0FB
:109B2000C801DF91CF911F910F91FF90EF900C949E
:109B3000DA4D0C94BE4D0C943668DC011796ED910D
:109B4000FC9118970190F081E02D0994DC011796A3
:109B5000ED91FC9118970280F381E02D309709F088
:109B60000994089588EA91E10C941850FC017383DC
:109B70006283BC0188EA91E10C947C50BC0188EAC4
:109B800091E10C946150CF93DF93EC0188EA91E16D
:109B90000E941C50009749F0FC01228133812C1750
:109BA0003D0729F00E94C450F5CF80E090E0DF919E
:109BB000CF9108950F931F93CF93DF938B010E9452
:109BC000C34DEC01009731F01D830C83C8010E9446
:109BD000676A8E83DF91CF911F910F9108951F9334
:109BE000CF93DF93EC01162FEC81FD813097D1F0FC
:109BF0009093AB118093AA1182E08887CE010696DC
:109C00000995992787FD90950297029710F01338D0
:109C100039F4BE01CE01DF91CF911F910C941C4EFF
:109C200081E08887DF91CF911F910895FC01208505
:109C300020FD0C94EF4D0895CF92DF92EF92FF92AA
:109C40000F931F93CF93DF93EC016B01E090AA1168
:109C5000F090AB110091AC111091AD11F801EC171F
:109C6000FD0739F0309709F44AC00190F081E02DEA
:109C7000F6CF209709F443C08885882309F1188618
:109C80000115110561F0C017D10729F0AE0167E891
:109C9000C8010E94164EF80100811181F1CFEC81BC
:109CA000FD81309769F0CC15DD0551F0D093AB11F3
:109CB000C093AA1140E050E063E8CE0106960995F2
:109CC000E091AC11F091AD11CE17DF0769F48881F6
:109CD00099819093AD118093AC110DC080819181D9
:109CE0008C179D0721F0FC013097C1F704C08881D3
:109CF000998191838083F092AB11E092AA11DF9158
:109D0000CF911F910F91FF90EF90DF90CF9008952A
:109D10001F93CF93DF931092B611C091AC11D091E5
:109D2000AD1111E0209779F08985882341F01887DB
:109D3000198640E050E062E8CE010E94EF4D0990A4
:109D4000D881C02DEFCFDF91CF911F9108958091E1
:109D5000591291E0980F9093591208956091AA11A9
:109D60007091AB110C941C4E8AE88093591210929A
:109D70005712109258121092AD111092AC1110920D
:109D8000AB111092AA1108958091B61181110E9411
:109D9000884E70915812772309F451C0E091571200
:109DA0002E2F30E085E0E89FF0011124E954FE4EAB
:109DB00060816093B511418152815093B4114093F9
:109DC000B311838194819093B2118093B1112F5F6D
:109DD0003F4F2F71332720935712715070935812B1
:109DE000009731F58091AC119091AD119093B01125
:109DF0008093AF118091AF119091B011892BF9F040
:109E00008091B61181110E94884E4091B3115091FA
:109E1000B4116091B5118091AF119091B0110E9471
:109E2000164EE091AF11F091B01180819181DECF9B
:109E3000613819F421E0FC0120870E94164E8091C0
:109E4000B6112091581290E0820F911D08958091D3
:109E5000B6112091581290E0820F911D0895209123
:109E600058122032B9F0E0915712E20FEF71E093EF
:109E7000AE1135E0E39FF0011124E954FE4E6083FA
:109E800052834183948383832F5F2093581280E011
:109E900090E0089581E090E00895CF93DF93C09122
:109EA000AA11D091AB110E94164ED093AB11C09362
:109EB000AA11DF91CF910895AB013091AC1120919F
:109EC000AD11E32FF22FE817F907B1F0309721F029
:109ED0000190F081E02DF7CF009771F0FC01308305
:109EE00021839093AD118093AC1121E020871782DC
:109EF000168261E80C944D4F0895009749F0FC01DB
:109F000020852150223020F421E021872093B611B2
:109F1000089521E030E0FC018085811102C020E03D
:109F200030E0C9010895CF93DF93EC014A815B8152
:109F300060E070E08C819D810E94D88C2A813B81F9
:109F400088819981289FA001299F500D389F500D2D
:109F5000112460E070E08E819F81DF91CF910C949D
:109F6000D88CFC018281938120E030E028173907EA
:109F7000D1F0A481B581A20FB31F4C91411110C043
:109F800081E08C9380819181289FA001299F500DB1
:109F9000389F500D112486819781840F951F089555
:109FA0002F5F3F4FE3CF80E090E00895FC012681D2
:109FB00037814281538180E090E084179507C9F092
:109FC0002617370781F4A481B581A80FB91F2C91FA
:109FD000121614F421502C930480F581E02DE80F23
:109FE000F91F80810895A081B1812A0F3B1F01963E
:109FF000E4CF8FEF0895FC01868197816817790778
:10A00000A0F0A081B18142815381A49F9001A59FBE
:10A01000300DB49F300D1124280F391F81E090E0DE
:10A020006217730720F080E0089580E090E00895C3
:10A03000FC01118210820895FC01808191810895B4
:10A04000FB0120813181FC01318320830895DC01F3
:10A05000ED91FC91309731F080819181009729F04A
:10A06000FC01FACF80E090E00895CF010895DC0173
:10A07000ED91FC9111973097A9F020813181232B2C
:10A0800021F41D921C92CF010895A081B1818D9180
:10A090009C911197892B11F0FD01F7CF118210824D
:10A0A000CD01089580E090E00895DC01ED91FC91F0
:10A0B0001197309721F0208131812D933C93CF016E
:10A0C0000895DC01ED91FC913097A9F0A0E0B0E09B
:10A0D00020813181E617F70741F4109709F4DC017C
:10A0E0002D933C931182108208952115310519F0AA
:10A0F000DF01F901EDCF08950F931F93CF93DF9305
:10A100008C01EB010E94615019821882C8010E94E3
:10A110002750009711F4F80101C0FC01D183C083DE
:10A12000DF91CF911F910F9108950F931F93CF93BC
:10A13000DF93EC018B010E94615088819981F801C5
:10A140009183808319830883DF91CF911F910F91B1
:10A150000895DC01ED91FC9180E090E0309729F0CA
:10A1600001960190F081E02DF9CF0895FB01309721
:10A1700019F4BA010C94955080819181DA018D9384
:10A180009C93518340830895009721F0FC018081C6
:10A190009181089580E090E0089580915C12909103
:10A1A0005D12892B29F410925B1210925A120895B5
:10A1B0000E94C15FE0915C12F0915D1222813381B7
:10A1C00040815181240F351F281B390B0480F581F4
:10A1D000E02D309769F04281538160817181460F93
:10A1E000571F481B590B4217530780F79A01EECFB0
:10A1F000280F391F30935B1220935A1208958CE771
:10A2000092E00C947D4FEF92FF920F931F93CF93A8
:10A21000DF938C01FC0180819181009799F08A3550
:10A220009105D9F0F8011182108283E068C086811F
:10A2300097818417950709F049C00480F581E02DC6
:10A240003097A9F710925D1210925C128AE590E0A7
:10A25000F8019183808381E052C0673891F16238C0
:10A26000A9F7C0915C12D0915D12E12CF12C2097DE
:10A2700069F3CE010E94386E892BF1F0AE0168E8D7
:10A280008E819F810E942F4F892BA1F41F821E82F5
:10A290008C819D81E114F10421F0F7019583848381
:10A2A00004C090935D1280935C121D821C820E94F8
:10A2B000CD50D7CF0E94FF507E010C80DD81C02D94
:10A2C000D6CFE0915C12F0915D12BACFF0935D129F
:10A2D000E0935C12A481B581109709F4B7CF16966C
:10A2E0008D919C9117978417950711F0FD01F2CF7E
:10A2F00014968D919C91159795838483EBCFDF9174
:10A30000CF911F910F91FF90EF900895CF93DF931E
:10A31000EC010E94FF508E819F8130915C12209150
:10A320005D12892B59F0E32FF22F309739F0EC179B
:10A33000FD0781F00480F581E02DF7CF8091AA110F
:10A340009091AB119F838E833C832D83D0935D12BC
:10A35000C0935C12DF91CF910C94CD50CF93DF93DB
:10A36000EC010E94186ECE01DF91CF910C948651C2
:10A37000CF93DF93EC010E94246ECE01DF91CF9149
:10A380000C948651CF93DF93EC010E942E6ECE0188
:10A39000DF91CF910C948651FC0120813181260FF1
:10A3A000371F318320830C94CD5021E030E0FC0135
:10A3B00086819781892B11F020E030E0C901089552
:10A3C000FC012281338180819181820F931F089546
:10A3D000FC0180819181089581E090E020915C12E0
:10A3E00030915D12232B11F480E090E0089580916C
:10A3F0005C1290915D12892B29F080915A129091F4
:10A400005B12089580E090E00895CF93DF93EC0114
:10A41000E0915C12F0915D128E179F0769F48C81B8
:10A420009D8190935D1280935C120DC08481958113
:10A430008C179D0721F0FC013097C1F706C08C8175
:10A440009D81958384830E94CD501D821C821F8232
:10A450001E82DF91CF910895EF92FF920F931F9389
:10A46000CF93DF938C017A01FC0180819181009769
:10A4700041F08B34910501F1F8011182108283E0E3
:10A4800048C08FE592E10E941C50EC01209751F0EA
:10A490006C817D81CE0102960E94AE510990D881D7
:10A4A000C02DF4CF81E080935E128BE490E0F80140
:10A4B0009183808381E02DC06838E1F78FE592E1D8
:10A4C0000E941C50EC01209781F3CE010296E81601
:10A4D000F906D9F4BE018FE592E10E946150E09047
:10A4E000AA11F090AB118A859B859093AB11809354
:10A4F000AA11EC85FD85309719F08E859F85099509
:10A50000F092AB11E092AA11D0CF0990D881C02D62
:10A51000DACFDF91CF911F910F91FF90EF900895C7
:10A5200010925E128FE592E10E94185060E070E098
:10A5300086E892E00C945C4F0F931F93CF93DF93C8
:10A54000EC010091AA111091AB111B870A875D875E
:10A550004C873F872E8780915E12882379F086E8AA
:10A5600092E09093AB118093AA11CE0102960E94C3
:10A57000AE511093AB110093AA1102C07D836C837E
:10A58000BE018FE592E10E946150BE018FE592E12C
:10A59000DF91CF911F910F910C947C500F931F93DB
:10A5A000CF93DF93EC0180915E12882391F00091AC
:10A5B000AA111091AB1186E892E09093AB118093B1
:10A5C000AA11CE0102960E94B8511093AB110093CC
:10A5D000AA11BE018FE592E10E946150BE018FE594
:10A5E00092E1DF91CF911F910F910C947C500F93CA
:10A5F0001F93CF93DF93EC0180915E12882391F03B
:10A600000091AA111091AB1186E892E09093AB11E2
:10A610008093AA11CE0102960E94C2511093AB11F1
:10A620000093AA11BE018FE592E10E946150BE0124
:10A630008FE592E1DF91CF911F910F910C947C50A7
:10A64000CF93DF93EC0180915E12882329F0CE0135
:10A6500002960E94055204C01F821E821986188627
:10A66000BE018FE592E1DF91CF910C946150CF93C1
:10A67000DF93EC0180915E12882331F0CE010296C7
:10A68000DF91CF910C94D5518FE592E10E941C503F
:10A69000009739F08C179D0739F0FC01808191817A
:10A6A000F7CF81E090E002C080E090E0DF91CF91B1
:10A6B00008952F923F924F925F926F927F928F9266
:10A6C0009F92AF92BF92CF92DF92EF92FF920F9341
:10A6D0001F93CF93DF93CDB7DEB7E8970FB6F8940B
:10A6E000DEBF0FBECDBFEDE8FAE2208131814281AD
:10A6F0005381E9E8FAE25080418032802380E5E826
:10A70000FAE28081898391819A83A281AB836380FD
:10A71000E1E8FAE2B081BC8381818D8392819E83DE
:10A72000A381AF83EDE7FAE2B081B88781818987A1
:10A7300092819A87A381AB87E9E7FAE2B081BC876F
:10A7400081818D8792819E87A381AF87E5E7FAE2B9
:10A75000B081B88B8181898B92819A8BA381AB8BDD
:10A76000E1E7FAE2B081BC8B81818D8B92819E8B77
:10A77000A381AF8BEDE6FAE2B081B88F8181898F3A
:10A7800092819A8FA381AB8FE9E6FAE2B081BC8F08
:10A7900081818D8F92819E8FA381AF8FE5E6FAE252
:10A7A000B081B8A3818189A392819AA3A381ABA32D
:10A7B000E1E6FAE2B081BCA381818DA392819EA3E0
:10A7C000A381AFA3EDE5FAE2B081B8A7818189A7A3
:10A7D00092819AA7A381ABA7E9E5FAE2B081BCA771
:10A7E00081818DA792819EA7A381AFA7E5E5FAE2BB
:10A7F000B081B8AB818189AB92819AAB7380E1E57E
:10A80000FAE2B080A18092808380EDE4FAE2F080E9
:10A81000E180D280C380E9E4FAE2A081AFABB181EC
:10A82000B8AF128103812BAB3CAB4DAB5EAB0E944A
:10A83000EF5F5EA95F934DA94F933CA93F932BA96E
:10A840002F932F923F924F925F926F922B812F9373
:10A850002A812F9329812F932F812F932E812F933C
:10A860002D812F932C812F932B852F932A852F9326
:10A8700029852F9328852F932F852F932E852F930E
:10A880002D852F932C852F932B892F932A892F93F6
:10A8900029892F9328892F932F892F932E892F93DE
:10A8A0002D892F932C892F932B8D2F932A8D2F93C6
:10A8B000298D2F93288D2F932F8D2F932E8D2F93AE
:10A8C0002D8D2F932C8D2F932BA12F932AA12F9376
:10A8D00029A12F9328A12F932FA12F932EA12F933E
:10A8E0002DA12F932CA12F932BA52F932AA52F9326
:10A8F00029A52F9328A52F932FA52F932EA52F930E
:10A900002DA52F932CA52F937F922AA92F9329A9A8
:10A910002F9328A92F938F929F92AF92BF92CF929D
:10A92000DF92EF92FF920F931F9328AD2F932FA9E1
:10A930002F939F938F937F936F93A7E5B8E28C91AA
:10A940001F928F93E6E5F8E280811F928F9385E94D
:10A950009EE09F938F930E94968DEDEBFAE220810B
:10A96000318142815381E9EBFAE2508041803280AB
:10A970002380EDEAFAE29080818072806380E9EAC8
:10A98000FAE28081898391819A83A281AB83B3812A
:10A99000BC83E5EAFAE280818D8391819E83A28166
:10A9A000AF83B381B887E1EAFAE280818987918138
:10A9B0009A87A281AB87B381BC87EDE9FAE28081F7
:10A9C0008D8791819E87A281AF87B381B88BE9E99A
:10A9D000FAE28081898B91819A8BB280A380E5E92C
:10A9E000FAE2F080E180D280C380E1E9FAE2A0815E
:10A9F000AB8BB181BC8B128103810FB6F894DEBFA3
:10AA00000FBECDBF2BAB3CAB4DAB5EAB0E94EF5F3F
:10AA10005EA95F934DA94F933CA93F932BA92F9318
:10AA20002F923F924F925F926F927F928F929F925E
:10AA30002C812F932B812F932A812F9329812F9360
:10AA400028852F932F812F932E812F932D812F9344
:10AA50002C852F932B852F932A852F9329852F9330
:10AA600028892F932F852F932E852F932D852F9314
:10AA7000AF92BF922A892F9329892F93CF92DF9289
:10AA8000EF92FF920F931F932C892F932B892F9373
:10AA90009F938F937F936F93A7E5B8E28C911F925A
:10AAA0008F93E6E5F8E280811F928F9386E29EE025
:10AAB0009F938F930E94968D0FB6F894DEBF0FBEC2
:10AAC000CDBFE8960FB6F894DEBF0FBECDBFDF91C5
:10AAD000CF911F910F91FF90EF90DF90CF90BF909B
:10AAE000AF909F908F907F906F905F904F903F902E
:10AAF0002F90089580E3809315130895CF93DF93EB
:10AB00006091151370E0C0E3D0E0C61BD70B6D5900
:10AB10007D4EAE010E94CF8CCE01DF91CF91089582
:10AB2000CF92DF92EF92FF920F931F93CF93DF9319
:10AB30007C01C0901813D09019136091151370E028
:10AB4000E601E096C61BD70BC138D105D8F400E367
:10AB500010E0061B170B6D597D4EA8010E94CF8C8B
:10AB60006091611270916212809116139091171387
:10AB7000680F791FA601C701800F911F0E94CF8C1B
:10AB8000CE0102C080E090E0DF91CF911F910F9144
:10AB9000FF90EF90DF90CF90089590911513980F4C
:10ABA0009093151308954091181350911913481755
:10ABB000590798F02091161330911713280F391F59
:10ABC0003093171320931613481B590B50931913E6
:10ABD0004093181381E090E0089580E090E008959C
:10ABE00090931913809318130895809116139091E0
:10ABF00017138D569D4E08958091151390E08D5931
:10AC00009D4E089581E090E0209161123091621292
:10AC10002359324111F480E090E008950E940256D9
:10AC2000892B61F06091611270916212409118134A
:10AC30005091191383E992E10C94CF8C2091161353
:10AC40003091171321153105B9F0809118139091A7
:10AC50001913C096E3E9F2E1AF0143565241481798
:10AC6000590734F4DF01A20FB31F4C914193F4CF85
:10AC700010921713109216130895809161129091FB
:10AC8000621208958091181390911913089590916C
:10AC9000151380E3891B089520E380911513281B69
:10ACA0008091181390911913820F911D08951F938D
:10ACB000CF93DF93EC0110911513812F90E08C1747
:10ACC0009D076CF00E944C568C0F9D1F813891059A
:10ACD00030F41C1B1093151381E090E002C080E05B
:10ACE00090E0DF91CF911F910895CF93DF93E0E63D
:10ACF000F8E21192119288E2E039F807D1F7C8E53D
:10AD0000D8E264EF72E0CE010E94084D229688E2FC
:10AD1000C036D807B1F7DF91CF910895109217137D
:10AD200010921613109219131092181380E3809347
:10AD3000151383E992E190936212809361120C944F
:10AD40007556EF92FF920F931F93CF93DF9300D02E
:10AD5000CDB7DEB78C0169837A830E948E566981F4
:10AD6000E62E7A81F72E81E8E816F10418F080E8E3
:10AD7000E82EF12CA701B801809161129091621226
:10AD80000E94CF8CF0921913E0921813C7010F9014
:10AD90000F90DF91CF911F910F91FF90EF90089549
:10ADA0000F931F93CF93DF938C01EB010E948E567C
:10ADB0001093621200936112D0931913C093181369
:10ADC000DF91CF911F910F91089520E3E0E6F8E223
:10ADD000DC0101900D922A95E1F788E0E8E5F8E2C0
:10ADE000DB0101900D928A95E1F7089520E3FC01C3
:10ADF000A0E6B8E201900D922A95E1F788E0FB0108
:10AE0000A8E5B8E201900D928A95E1F70895E82F40
:10AE1000F0E0EE0FFF1FE05AF74D7183608381E091
:10AE200090E00895E82FF0E0EE0FFF1FE05AF74D95
:10AE300080819181089590E0880F991F885D974DDA
:10AE40000E94084D81E090E0089590E0880F991FDE
:10AE5000885D974D08958115910511F00197F1F7DF
:10AE60000895E0919328F091942890818091922800
:10AE700089230895E0919028F09191288081909104
:10AE80009228892B8083E0919528F09196288081E3
:10AE900090919228892B80830895E0919028F091D9
:10AEA0009128908180919228809589238083E091D8
:10AEB0009528F091962890818091922880958923F9
:10AEC000808308951F93CF93DF93E0919028F091B2
:10AED0009128908180919228809589238083E091A8
:10AEE0009528F0919628808190919228892B8083D3
:10AEF0008FEB93E00E942B571FB7F894E0919528B1
:10AF0000F091962890818091922880958923808362
:10AF100083E890E00E942B57E0919328F0919428C9
:10AF2000D081C09192281FBF78948BE393E00E9458
:10AF30002B57E0919328F09194289081809192284A
:10AF4000982319F08D2F8C2301C081E0DF91CF91E0
:10AF50001F910895509396284093952870939128B7
:10AF600060939028909394288093932881E001C067
:10AF7000880F2A95EAF7809392280C946257CF9312
:10AF8000DF93C82FDFB7F894E0919528F0919628C9
:10AF9000808190919228892B808383E090E00E94A9
:10AFA0002B57CC2351F0E0919528F0919628808181
:10AFB0009091922890959823908387E190E00E9449
:10AFC0002B57E0919328F0919428808190919228BA
:10AFD000892309F4C0E089E590E00E942B57E091B5
:10AFE0009528F091962880819091922890959823A9
:10AFF0009083DFBF8BE390E00E942B578C2FDF9173
:10B00000CF910895CF93DF93C82FD8E08C2F817014
:10B010000E94BF57C6958111C068D150B9F78C2FD7
:10B02000DF91CF9108958FEF0C940258DF92EF9249
:10B03000FF920F931F93CF93DF93E82EEB010E94B3
:10B04000625781112FC080EF0E940258F12C10E44A
:10B0500088EFD82ED10E81E00E94BF57082F81E0E3
:10B060000E94BF57882319F0002361F01DC0011111
:10B0700009C01E1528F0888180FF04C0E11611F078
:10B08000F12E01E0802F0E94BF5798819695011103
:10B090009068988311501D11DECF21961111D8CFE1
:10B0A0008F2D03C08FEF01C08EEFDF91CF911F91E5
:10B0B0000F91FF90EF90DF900895FF920F931F93F1
:10B0C000CF93DF93F82EEB010E946257209769F02F
:10B0D00085E50E9402588E01085F1F4F89910E94EA
:10B0E0000258C017D107D1F703C08CEC0E94025858
:10B0F0008F2DDF91CF911F910F91FF900C940258EB
:10B100000F931F93CF93DF93DB01EC9111969C91EA
:10B110001197F0E0F92B803181F4BF016E7FE3E0FD
:10B12000660F771FEA95E1F716969C911697ECE06B
:10B13000F0E0E91BF109E60FF71FF7FF07C091E008
:10B14000EA019883F195E195F10902C0EA011882BC
:10B15000883279F414968C91982F9076903649F035
:10B1600086FF02C0EE7F05C085FF02C0EC7F01C0F4
:10B17000E87FCF0144E0969587954A95E1F7D9019C
:10B180008C93EF70E801E88380E0DF91CF911F910D
:10B190000F9108950F931F93CF93DF93EC018B01D1
:10B1A000B80188810E941658888381508D3F30F401
:10B1B000F8018081883211F0803191F7DF91CF91D1
:10B1C0001F910F910895CF93DF93EC010E94625776
:10B1D000BE0184EB0E945D5881E00E94BF57C82FDA
:10B1E0000E94625781E0C11101C080E0DF91CF91E0
:10B1F00008951F93CF93DF9300D0CDB7DEB7182FFC
:10B2000069837A830E9462570E94315769817A81EB
:10B21000882341F084E40E945D58113029F00E9497
:10B220003A5702C082E001C080E00F900F90DF919A
:10B23000CF911F9108954F925F926F927F928F925C
:10B240009F92AF92BF92CF92DF92EF92FF920F93B5
:10B250001F93CF93DF93CDB7DEB729970FB6F8943E
:10B26000DEBF0FBECDBF6C015B014A0189010E94A8
:10B270006257B6018EEB0E945D58CE0101967C01AB
:10B280003E019AE0690E711C27010E941358F701D4
:10B2900081937F01E615F705C1F769E070E0C2010F
:10B2A0000E94A972811109C09401A501B201F601A1
:10B2B00080810E94805880E001C083E029960FB60B
:10B2C000F894DEBF0FBECDBFDF91CF911F910F91DC
:10B2D000FF90EF90DF90CF90BF90AF909F908F90B6
:10B2E0007F906F905F904F9008955F926F927F92E2
:10B2F0008F929F92AF92BF92CF92DF92EF92FF9286
:10B300000F931F93CF93DF93CDB7DEB729970FB677
:10B31000F894DEBF0FBECDBF582E6B015A018901D4
:10B3200060E070E08EEB0E945D58CE0101967C01DA
:10B330004E019AE0890E911C37010E941358F701C3
:10B3400081937F01E815F905C1F769E070E0C30159
:10B350000E94A972811108C09501A601B301852D33
:10B360000E94805880E001C083E029960FB6F894CF
:10B37000DEBF0FBECDBFDF91CF911F910F91FF9028
:10B38000EF90DF90CF90BF90AF909F908F907F9085
:10B390006F905F9008950F931F93CF93DF93CDB776
:10B3A000DEB728970FB6F894DEBF0FBECDBF182FBB
:10B3B000062F98E0E0E0F3E0DE01119601900D9297
:10B3C0009A95E1F7242F332727FD309541E752E086
:10B3D000249FC001259F900D349F900D112464E699
:10B3E00070E00E94EA86CB0144E6049F800D911D27
:10B3F0001124FE013196AE01475F5F4F619170E00D
:10B400002617370711F4019603C0E417F507B1F7C3
:10B41000112319F091958195910928960FB6F8940A
:10B42000DEBF0FBECDBFDF91CF911F910F91089569
:10B43000EF92FF920F931F93CF93DF93CDB7DEB7B9
:10B440002B970FB6F894DEBF0FBECDBFF82EE92EB6
:10B45000682F792F88E08F0D0E94F958882319F002
:10B4600084E391E243C066E471E48FE090E00E94DF
:10B47000835A8E01075F1F4F9801AE01465F5F4FF1
:10B48000BE01655F7F4F8F2D9E2D0E941B5981113C
:10B49000E7CF88E0E0E0F3E0DE01119601900D9245
:10B4A0008A95E1F7498521E732E0429FC001439F39
:10B4B000900D112464E670E00E94EA868A8594E685
:10B4C000899F600D711D1124FE01319681914813F1
:10B4D00003C06F5F7F4F03C0E017F107B9F78B859B
:10B4E000882319F0719561957109CB012B960FB6E0
:10B4F000F894DEBF0FBECDBFDF91CF911F910F91AA
:10B50000FF90EF900895DC01CB0181159105A10515
:10B51000B10529F081509040A040B040D9F708957E
:10B520001092B90080E28093B800089594EA909355
:10B53000BC0040EA56E861E070E09091BC0097FDE5
:10B540000BC041505109610971094115510561054F
:10B55000710599F781E008959091B900987F98302E
:10B5600011F09031B9F78093BB0084E88093BC0060
:10B5700080EA96E8A1E0B0E02091BC0027FD08C079
:10B580000197A109B1090097A105B105A9F7E2CF7B
:10B590008091B900887F883111F08034D9F680E03D
:10B5A000089524EA34E844E92093BC009091BC005B
:10B5B00097FFFCCF9091B900987F983011F09031AF
:10B5C00099F78093BB003093BC009091BC0097FF2B
:10B5D000FCCF9091B900987F903211F0983539F4F2
:10B5E0004093BC009091BC0094FDFCCFDDCF08954A
:10B5F0000C94965A84E98093BC008091BC0084FD31
:10B60000FCCF08958093BB0084E88093BC008091B8
:10B61000BC0087FFFCCF9091B900987F81E0983201
:10B6200009F480E0089584EC8093BC008091BC0014
:10B6300087FFFCCF8091BB00089584E88093BC0015
:10B640008091BC0087FFFCCF8091BB000895E0E1B2
:10B65000DC01FD91CD01F0933F01E150C9F78091EC
:10B660003C018F7D80933C0180913C01877F8093DA
:10B670003C01FB0180E1919190933E018150D9F70B
:10B6800080913C01806880933C0180913D0180FF66
:10B69000FCCF4051510980913C01806280933C0174
:10B6A00080913C01877F80933C01141615069CF421
:10B6B000FB0180E1919190933E018150D9F78091F7
:10B6C0003C01806880933C0180913D0180FFFCCF6C
:10B6D00040515109EACFF90180E190913E019193E7
:10B6E0008150D9F781E090E008950F931F93CF9395
:10B6F000DF93EC018CE70E94D15A8CE70E94025B39
:10B700008E01005F1F4F89910E94025BC017D10715
:10B71000D1F7DF91CF911F910F910C94FA5A81309C
:10B7200019F440E050E002C040EC50E060E070E00E
:10B730008CE790E00C940111813019F44EE050E058
:10B7400002C048E050E060E070E08CE790E00C94CC
:10B75000011141E050E060E070E08CE790E00E9471
:10B7600001116AE67AE080E090E00C94835A48E3A5
:10B7700050E060E070E08CE790E00E94011149E346
:10B7800050E060E070E08CE790E00E94011144E13D
:10B7900050E060E070E08CE790E00E94011148E723
:10B7A00050E060E070E08CE790E00E9401114EE50F
:10B7B00050E060E070E08CE790E00E9401114DE6FF
:10B7C00050E060E070E08CE790E00E9401116CE1D5
:10B7D0007AE186E090E00E94835A4CE050E060E01D
:10B7E00070E08CE790E00E94011141E050E060E0E1
:10B7F00070E08CE790E00E94011146E050E060E0CC
:10B8000070E08CE790E00E9401116AE67AE080E047
:10B8100090E00C94835ACF93DF93CDB7DEB7A29715
:10B820000FB6F894DEBF0FBECDBF81E1E9EEF8E0C0
:10B83000DE01529601900D928A95E1F781E1EAEFDF
:10B84000F8E0DE01119601900D928A95E1F70E94D1
:10B85000B75BCE0142960E94755B82E00E948F5BCF
:10B860006AE67AE080E090E00E94835ACE01019679
:10B870000E94755B60E17EEA88E290E00E94835A54
:10B8800080E00E949C5B60E17EEA88E290E00E949A
:10B89000835A4EE050E060E070E08CE790E00E9458
:10B8A0000111A2960FB6F894DEBF0FBECDBFDF9197
:10B8B000CF910895CF92DF92EF92FF920F931F9353
:10B8C000CF93DF9300D01F92CDB7DEB7F82E042FB1
:10B8D000122F213031F0223031F0243031F0283075
:10B8E00031F090E005C091E003C092E001C093E028
:10B8F0000C3059F00E3011F4946007C0003111F48F
:10B90000986003C0023109F49C60613059F06230E4
:10B9100011F4906207C0633011F4906403C0643086
:10B9200009F490669068692F70E023E030E0AE0182
:10B930004F5F5F4F8F2D90E00E94181169E07AE110
:10B9400080E090E00E94835A8F2D8160F82E0E9443
:10B95000965A0E94135B89830E94135B8A8302318B
:10B9600019F40E94135B8B830E94135B87FDF1CF58
:10B970000E941D5B0E94FA5A69E07AE180E090E043
:10B980000E94835A8F2D0E94965A0E94135B8983CE
:10B990000E94135B8A83023119F40E941D5B8B8322
:10B9A0000E941D5B0E94FA5A39812A81023149F5B1
:10B9B000832F90E0A0E0B0E04B817727662731FF2E
:10B9C0000EC030E0322F2227620F731F811D911DA0
:10B9D000640F711D811D911D8C6F9F6F0BC030E036
:10B9E000322F2227620F731F811D911D640F711D5D
:10B9F000811D911D0E94F78320E83FEF4FEF57E430
:10BA000020C0632F70E0762F6627620F711D882794
:10BA100077FD8095982F0E94F7830C3029F420E061
:10BA200030EE4FEF54E40DC00E3029F420E038EF33
:10BA30004FEF55E406C0003131F420E03EEF4FEF08
:10BA400056E40E9458832FE632E143E050E40E941E
:10BA5000D5856B017C01612F70E080E090E00E9451
:10BA6000F7839B01AC01C701B6010E9458830F9078
:10BA70000F900F90DF91CF911F910F91FF90EF905A
:10BA8000DF90CF900895E6E4F1E0808120819081FD
:10BA90003081829586958695837022952F70822BB2
:10BAA000832B92959F70892B08950F931F93CF93AB
:10BAB000DF9300D0CDB7DEB746E06CE080E00E94B7
:10BAC000856089E18093C4001092C50082E0809374
:10BAD000C00080E00E9410610E94B15F84B784B70B
:10BAE00084B784B784B7E7E1F1E322E432E4318339
:10BAF00020833A968DB79EB70A97E817F907B8F3EF
:10BB00008BE099E09F938F9382EE9FE09F938F93BA
:10BB10000E94968D0E94EC6E0E94B44E60E070E030
:10BB20008CE792E00E945C4F0E949052E0910803E3
:10BB3000F091090309950E94435D90E00E94286FEF
:10BB4000CE0101960E94E65E0F900F900F900F902D
:10BB5000882341F082EC9FE09F938F930E94968D03
:10BB60000F900F90CE0101960E94234D0E94F45E2B
:10BB70008C010E94F05EAE014F5F5F4FB8010E94E2
:10BB8000DC630E94605E0E94BD630E94F85E0E94BA
:10BB9000166585EB9FE09F938F930E94968D8A8117
:10BBA0001F928F9301EB1FE01F930F930E94968DBE
:10BBB00089811F928F931F930F930E94968D8FEA16
:10BBC0009FE09F938F930E94968D0E942C6FE0912F
:10BBD0004503F09146030995E0913703F09138034E
:10BBE0000995E0911E03F0911F0309950E941D65C0
:10BBF000182F0E94BA631F921F931F928F938091F8
:10BC000044038F93809143038F93809136038F93E6
:10BC1000809135038F9384E99FE09F938F930E94D7
:10BC2000968DE0914F03F09150030FB6F894DEBF6C
:10BC30000FBECDBF309791F00995BC0180E890E030
:10BC40000E94D6867F936F9381E89FE09F938F93A6
:10BC50000E94968D0F900F900F900F908FE79FE0AE
:10BC60009F938F930E94968D60E070E082ED92E04A
:10BC70000E945C4F84EE92E00E94FC6D87E79FE09B
:10BC80009F938F930E94968D0F900F900F900F901F
:10BC90000F900F90DF91CF911F910F9108957F9397
:10BCA0006F939F938F9381E79FE09F938F930E9461
:10BCB000968D0F900F900F900F900F900F9008950A
:10BCC0001F93CF93DF93CDB7DEB7A0970FB6F8944D
:10BCD000DEBF0FBECDBF83E590E00E94028F182F1C
:10BCE000282F35EF380F303108F0982F909529170D
:10BCF00009F461C08DEF9FE09F938F930E94968D12
:10BD0000E2E4F0E10F900F90DE01119684918D93A3
:10BD1000319680E1EA34F807C9F7F89448E050E03A
:10BD20006FE670E0CE0101960E94088FE4E3F0E137
:10BD3000DE01119684918D93319680E1E234F8070B
:10BD4000C9F74EE050E061E670E0CE0101960E9436
:10BD5000088FEAE2F0E1DE01119684918D9331962D
:10BD600080E1E433F807C9F74AE050E067E570E0A6
:10BD7000CE0101960E94088F6DEC7BEA81E590E090
:10BD80000E94208F60E070E08FE490E00E94208F9E
:10BD900060E08EE490E00E94128F60E070E085E544
:10BDA00090E00E94208F1AE16AE175EE83E590E051
:10BDB0000E94208F7894812FA0960FB6F894DEBF52
:10BDC0000FBECDBFDF91CF911F910895F89442E04F
:10BDD00050E06FE670E00E94EA8E789480E008956B
:10BDE00081E590E00C94028F8FE490E00C94028F38
:10BDF0008EE490E00C94FA8E4091A5285091A628EC
:10BE00006091A7287091A82890E0A0E0B0E0480FCA
:10BE1000591F6A1F7B1F4093A5285093A628609343
:10BE2000A7287093A8284091A1285091A22860913A
:10BE3000A3287091A428480F591F6A1F7B1F4093A5
:10BE4000A1285093A2286093A3287093A42820913E
:10BE5000452A2223A1F040919D2850919E2860916F
:10BE60009F287091A028480F591F6A1F7B1F40937D
:10BE70009D2850939E2860939F287093A028089532
:10BE80001F920F920FB60F9211240BB60F922F93A1
:10BE90003F934F935F936F937F938F939F93AF9352
:10BEA000BF93EF93FF9380911C1390911D13019604
:10BEB00090931D1380931C1380911B138F5F8093AD
:10BEC0001B138038A9F410921B138091A528909120
:10BED000A628A091A728B091A8280196A11DB11D60
:10BEE0008093A5289093A628A093A728B093A8286C
:10BEF0008091452A8823E1F080911A138F5F809307
:10BF00001A138038A9F410921A1380919D289091E9
:10BF10009E28A0919F28B091A0280196A11DB11D37
:10BF200080939D2890939E28A0939F28B093A0284B
:10BF30000E94EC51892B11F00E94FF50FF91EF916C
:10BF4000BF91AF919F918F917F916F915F914F9131
:10BF50003F912F910F900BBE0F900FBE0F901F902F
:10BF60001895F8941092B60016BC83EF87BD82E056
:10BF700084BD94E095BD95B395BB80936E00789495
:10BF8000089580911C1390911D1320911C133091E2
:10BF90001D1382179307A9F70895009751F022E324
:10BFA00030E000002150310921153105D1F701970A
:10BFB000F4CF08950F931F93CF93DF93EC010E946A
:10BFC000C15F8C010E94C15F801B910B8C179D0784
:10BFD000C8F3DF91CF911F910F91089508950F93AA
:10BFE0001F936091A5287091A6288091A728909111
:10BFF000A8280091A5281091A6282091A728309163
:10C00000A828601771078207930759F71F910F91AE
:10C0100008951F920F920FB60F9211241092A8024A
:10C020000F900FBE0F901F9018951F920F920FB692
:10C030000F9211240BB60F922F933F934F935F9360
:10C040006F937F938F939F93AF93BF93EF93FF93E0
:10C05000E0919E02F0919F028081E091A902F0910F
:10C06000AA02309709F00995FF91EF91BF91AF9126
:10C070009F918F917F916F915F914F913F912F9100
:10C080000F900BBE0F900FBE0F901F9018951F9230
:10C090000F920FB60F9211241092B5020F900FBE9F
:10C0A0000F901F9018951F920F920FB60F921124A8
:10C0B0000BB60F922F933F934F935F936F937F93A2
:10C0C0008F939F93AF93BF93EF93FF93E091AB0256
:10C0D000F091AC028081E091B602F091B702309706
:10C0E00009F00995FF91EF91BF91AF919F918F91C9
:10C0F0007F916F915F914F913F912F910F900BBE68
:10C100000F900FBE0F901F9018959DE0899FF00132
:10C110001124E256FD4FA281B3811C92A481B58106
:10C120006C93A681B78188ED8C93A085B1854C93E3
:10C1300012861486138608959DE0899FF0011124CC
:10C14000E256FD4F81E08287A081B1816C933A96DF
:10C1500080818111FDCF08951F93CF93DF93182F16
:10C16000EB01FE016491662329F0812F0E949C60FF
:10C170002196F7CFDF91CF911F9108951F93CF9311
:10C18000DF93182FEB018881882369F08A3021F42E
:10C190006DE0812F0E949C6069916D30A1F3812F29
:10C1A0000E949C60F0CFDF91CF911F910895CF93B3
:10C1B000DF93CDB7DEB79E01285F3F4F4E815F8191
:10C1C00060E470E08EE193E10E94538E6EE173E1D2
:10C1D0008D810E94BE60DF91CF910895CF93C82FCB
:10C1E0008A3031F46DE080915E130E949C6002C041
:10C1F0008D3029F06C2F80915E130E949C6080E04E
:10C2000090E0CF9108959DE0899FF0011124E256BE
:10C21000FD4F748763870895682F80E00C949C60BD
:10C2200080935E1380E992E09093123180931131F4
:10C23000089584B7877F84BF88E10FB6F894809310
:10C240006000109260000FBE08952FE088E190E03A
:10C250000FB6F894A895809360000FBE20936000FD
:10C260000895A895089588E10FB6F894809360002A
:10C27000109260000FBE0895F89428E088E190E0E5
:10C280000FB6F894A895809360000FBE20936000CD
:10C29000FFCF8091B0288091B02890E0089540E0D1
:10C2A0006FE181E491E00C94B266E9E3F1E0808112
:10C2B00080818D7F80838DE090E00197F1F723E00E
:10C2C00040E06FE182E491E00E94BC6683E090E090
:10C2D0000197F1F708959091390191FD0AC0282F37
:10C2E000803108F02FE040E06FE085E491E00C94AD
:10C2F000BC6608958091390181FD0EC040E06FE178
:10C3000081E491E00E94B266282F2F7E81E090E0C8
:10C31000213021F080E0089580E090E00895809140
:10C32000390181FD10C040E06FE181E491E00E949D
:10C33000B2668F3131F0982F9F7E915081E092301C
:10C3400018F480E0089581E008950E948F618823A9
:10C35000E1F30895CF93DF93C82F0E94A5610E9457
:10C360004F61D82FC81789F1C83019F40E94556160
:10C3700025C0C93121F4863189F429E005C0C631D0
:10C3800069F4893159F426E040E06FE182E491E0FC
:10C390000E94BC66E3E0F0E03197F1F72C2F40E01B
:10C3A0006FE182E491E00E94BC66D83019F4E9E6BE
:10C3B000F1E002C0E3E0F0E03197F1F70E944F6155
:10C3C0008C1719F083E490E002C080E490E0DF91E4
:10C3D000CF9108950E94A5611092452A0E9455614F
:10C3E000809139018260809339018091C82A882325
:10C3F000D9F180919400909195004091D92A509163
:10C40000DA2A84179507A0F48091A52A9091A62A8C
:10C41000A091A72AB091A82A8C57914EAF4FBF4F39
:10C420008093A52A9093A62AA093A72AB093A82A1E
:10C430002091940030919500241B350B8091A52A02
:10C440009091A62AA091A72AB091A82A820F931FA3
:10C45000A11DB11D8093A52A9093A62AA093A72A77
:10C46000B093A82A1092C82A8091CA2A8823D9F1A9
:10C4700080919400909195004091DD2A5091DE2AA0
:10C4800084179507A0F48091AD2A9091AE2AA091CF
:10C49000AF2AB091B02A8C57914EAF4FBF4F8093C7
:10C4A000AD2A9093AE2AA093AF2AB093B02A2091E0
:10C4B000940030919500241B350B8091AD2A90910A
:10C4C000AE2AA091AF2AB091B02A820F931FA11D6E
:10C4D000B11D8093AD2A9093AE2AA093AF2AB0935A
:10C4E000B02A1092CA2A08958091452A882381F0A3
:10C4F0008091E213811104C00E948F61811106C0F6
:10C5000081E08093E01381E090E008950E94EA6169
:10C5100080E090E008958091940090919500909330
:10C52000DE2A8093DD2A21E02093CA2A80913901F6
:10C5300081FD08C08091390181FD1AC086E10E9409
:10C54000AA6116C02093442A80919400909195008E
:10C550009093DA2A8093D92A2093C82A80913901AE
:10C560008D7F809339018091442A8111FCCFE2CFE5
:10C5700081E08093452A08958091452A81110AC05F
:10C580008091E213882321F081E08093E11302C0BF
:10C590000E948B6281E090E008951F93CF93DF9318
:10C5A0001F92CDB7DEB78FB789838091E2138111D7
:10C5B00026C0F8948091452A882351F08091390152
:10C5C00081FD1BC00E948F618823B9F080E003C009
:10C5D0000E94BC6281E02091470191E02E3008F07A
:10C5E00090E0192F119581110E947462107429F046
:10C5F00089818FBF81E090E004C089818FBF80E096
:10C6000090E00F90DF91CF911F9108958091E113F9
:10C61000882321F00E948B621092E1138091E01335
:10C62000882321F00E94EA611092E0131092E21335
:10C6300008950F931F93AB0121E02093E213009123
:10C64000892A10918A2A20918B2A30918C2A0F5F97
:10C650001F4F2F4F3F4F0093892A10938A2A209310
:10C660008B2A30938C2A22E0260F27FF0CC0809162
:10C67000422A9091432A01969093432A8093422A1A
:10C680000FEF1FEF07C0BC018FE593E10E94CF8C35
:10C6900000E010E00E940663C8011F910F91089509
:10C6A0008093E41308950E944F61823011F082312B
:10C6B00011F480E0089581E0089508958FEF80934C
:10C6C0004E0122E044E060EF8CE691E00E94BC66FF
:10C6D00025E041E06EE08CE290E00E94BC6680E8DC
:10C6E00080936F018091460180936D0121E045E0C8
:10C6F00060E284E491E00C94BC668DEF93E00197D6
:10C70000F1F70E94A8661092B92810923B29109266
:10C71000BD291092B8281092B728E9E3F1E0808192
:10C720008E7F808380818D7F80838DE090E0019774
:10C73000F1F7E9E3F1E080818160808323E040E06C
:10C740006FE182E491E00E94BC668DEF93E0019777
:10C75000F1F780915D0180915E010E945E6360E06F
:10C7600070E088EB92E00E945C4F0E948B6281E057
:10C7700090E008958091E3130895CF93DF931F9283
:10C78000CDB7DEB789830E94A56189818093E313C9
:10C79000282F40E06FE188E491E00F90DF91CF9186
:10C7A0000C94BC660E94BD638091390181FD03C079
:10C7B00086E00C94AA610895FA0180936201909337
:10C7C000630160936001709361013097C1F08081D3
:10C7D00080936B01818180936A01828180936901DA
:10C7E0008381809368018481809367018581809330
:10C7F0006601868180936501878180936401089535
:10C8000088EB92E00E947D4F81E08093B028809178
:10C81000B1289091B22801969093B2288093B128C4
:10C8200081E090E008958091B82892E8899FF00116
:10C830001124E754F74D10828F5F833018F48093F2
:10C84000B82802C01092B828E091B82882E8E89F82
:10C85000F0011124E754F74D808181110C9400649C
:10C860001092B02808951F93CF93DF932091B8289A
:10C8700012E8129F90011124D901A754B74D4C9191
:10C88000411103C00E94136493C05091390151FDBE
:10C890008FC05091452A552309F48AC047FF16C01E
:10C8A0000E9413648091792A90917A2AA0917B2A20
:10C8B000B0917C2A0196A11DB11D8093792A909395
:10C8C0007A2AA0937B2AB0937C2A72C04330B0F4BA
:10C8D0000E9413648091752A9091762AA091772AFC
:10C8E000B091782A0196A11DB11D8093752A90936D
:10C8F000762AA093772AB093782A5AC050E0EA01AA
:10C9000022976C177D07B0F40E9413648091712AFE
:10C910009091722AA091732AB091742A0196A11D58
:10C92000B11D8093712A9093722AA093732AB093B9
:10C93000742A3EC0B9016654774D0E94CF8CE091B5
:10C94000B8281E9FF0011124E75CF64D808180938A
:10C95000A9280E941364809147018093AA2890918E
:10C96000AF28992311F0891710F48093AF286091B4
:10C97000AA2870E084E00E9407576091A92870E01F
:10C9800083E00E94075740918D2A50918E2A609132
:10C990008F2A7091902A4F5F5F4F6F4F7F4F409368
:10C9A0008D2A50938E2A60938F2A7093902A02C00A
:10C9B000C0E0D0E0CE01DF91CF911F910895CF93D9
:10C9C000DF93EC01888199810097E9F087309540E9
:10C9D00021F01982188283E026C06238C1F41092D7
:10C9E000B0280E948E560E94F55560E870E00E94C3
:10C9F0003364181619066CF40E94F055E09149034F
:10CA0000F0914A03099587E095E09983888381E056
:10CA10000AC08091AD289091AE2801969093AE28DF
:10CA20008093AD28F0CFDF91CF91089591E090935E
:10CA3000E2130E946B610C9406638091390181FDC1
:10CA400006C040E06FE085E491E00C94B26680E1BE
:10CA500008950F931F93CF93DF93182F21E0209316
:10CA6000E2130091452A8091390181FF16C080911F
:10CA70009400909195009093DA2A8093D92A20937C
:10CA8000C82A2093442A809139018D7F80933901EF
:10CA90008091442A8111FCCF00E00E94A561809121
:10CAA000452A882309F43FC08091CA2A8823D9F1F6
:10CAB0008091940090919500E091DD2AF091DE2A1A
:10CAC0008E179F07A0F44091AD2A5091AE2A609135
:10CAD000AF2A7091B02A4C57514E6F4F7F4F409301
:10CAE000AD2A5093AE2A6093AF2A7093B02A20915A
:10CAF0009400309195002E1B3F0B4091AD2A509130
:10CB0000AE2A6091AF2A7091B02A420F531F611D67
:10CB1000711D4093AD2A5093AE2A6093AF2A709353
:10CB2000B02A1092CA2A8091390181FD03C089E19F
:10CB30000E94AA6186E00E941257892B51F00E9440
:10CB40001D65C82F86E00E94125781500E946B61BC
:10CB500002C0C0E0D0E02091940030919500309365
:10CB6000DC2A2093DB2A81E08093C92AF894809103
:10CB70003901826080933901809139018D7F8093E2
:10CB8000390162E0610F8FE593E10E94ED667894D0
:10CB900020913F2A3091402A2F5F3F4F3093402A07
:10CBA00020933F2A0E94A56145E060EE82E491E077
:10CBB0000E94B266182F86E00E941257892B19F046
:10CBC0008C2F0E946B61002319F00E948B6202C0BF
:10CBD0000E94EA618091C92A8823D9F1809194004A
:10CBE00090919500E091DB2AF091DC2A8E179F0747
:10CBF000A0F44091A92A5091AA2A6091AB2A709181
:10CC0000AC2A4C57514E6F4F7F4F4093A92A5093F7
:10CC1000AA2A6093AB2A7093AC2A20919400309199
:10CC200095002E1B3F0B4091A92A5091AA2A609192
:10CC3000AB2A7091AC2A420F531F611D711D4093A6
:10CC4000A92A5093AA2A6093AB2A7093AC2A109217
:10CC5000C92A8091452A882361F02091940030915F
:10CC600095003093DE2A2093DD2A81E08093CA2A42
:10CC700007C023E040E06FE182E491E00E94BC66DF
:10CC80000E9406631130E9F01330A9F48091812AE3
:10CC90009091822AA091832AB091842A0196A11DA5
:10CCA000B11D8093812A9093822AA093832AB09306
:10CCB000842A12E009C0153031F0173029F411E050
:10CCC00003C010E001C013E0812F90E0DF91CF910D
:10CCD0001F910F910895CF93DF93EB010E94196389
:10CCE000009729F4CE010E942965009751F0209108
:10CCF000422A3091432A2F5F3F4F3093432A20939B
:10CD0000422ADF91CF910895CF93DF938091452AF6
:10CD1000811104C00E94BC62D1E001C0D0E00E9439
:10CD20004F61863111F0813119F4C091470109C07A
:10CD300040E06FE186E491E00E94B266C82FCC0F1C
:10CD4000C80FD1110E9474628C2FDF91CF9108958A
:10CD50001092E6131092E513EFE6F0E08081806216
:10CD600080830895FC018081862390E002C0959520
:10CD700087954A95E2F70895F894FC015081362F83
:10CD800030955323042E01C0220F0A94EAF726237C
:10CD9000522B50837894089540917B01FC0141937C
:10CDA000A0E8B1E050E8540F9D012F5F3F4F6C9118
:10CDB0006193521711F0D901F7CF4150E42FF0E001
:10CDC000E058FE4F2181FC01E058FF4F2083FC0119
:10CDD000EF57FF4F21E02083089560938001E1E841
:10CDE000F1E061589F012F5F3F4FDC014D91CD0174
:10CDF0004083621711F0F901F5CF08951F920F9249
:10CE00000FB60F9211240BB60F922F933F934F93AF
:10CE10005F936F937F938F939F93AF93BF93EF93A2
:10CE2000FF93809147018093AA288091B72822E838
:10CE3000829FC00111248754974D0E94CC66809137
:10CE4000B7288F5F833018F48093B72802C0109200
:10CE5000B7280E940064FF91EF91BF91AF919F911D
:10CE60008F917F916F915F914F913F912F910F9093
:10CE70000BBE0F900FBE0F901F9018951F920F9230
:10CE80000FB60F9211240F900FBE0F901F901895A0
:10CE90001F920F920FB60F9211240F900FBE0F909A
:10CEA0001F9018951F920F920FB60F9211240F909A
:10CEB0000FBE0F901F9018951F920F920FB60F92F2
:10CEC00011241092442A0F900FBE0F901F901895B6
:10CED0001F920F920FB60F9211241092442A0F90B6
:10CEE0000FBE0F901F9018951F920F920FB60F92C2
:10CEF00011248F9381E08093B0288F910F900FBE03
:10CF00000F901F9018951F920F920FB60F92112439
:10CF10001092442A0F900FBE0F901F9018951F92E9
:10CF20000F920FB60F9211248F939F938091E51368
:10CF30009091E61301969093E6138093E5139F91E9
:10CF40008F910F900FBE0F901F901895CF92DF9288
:10CF5000EF92FF920F931F93CF93DF937C018B018E
:10CF60006A0187EE93E10E941C50EC01009751F09A
:10CF7000EC81FD81309711F0C8010995CE010E9426
:10CF8000C450F3CFA601B801C701DF91CF911F9123
:10CF90000F91FF90EF90DF90CF900C94A64D0F93E0
:10CFA0001F93CF93DF9300D0CDB7DEB780914D2A8A
:10CFB00090914E2AA0914F2AB091502A0196A11D1E
:10CFC000B11D80934D2A90934E2AA0934F2AB0937F
:10CFD000502A0E94396A8C0187EE93E10E941C500E
:10CFE000009779F0DC011296ED91FC911397309740
:10CFF00029F089839A8309959A8189810E94C45076
:10D00000EFCF0115110549F0C8010F900F90DF9186
:10D01000CF911F910F910C949D4D0F900F90DF9128
:10D02000CF911F910F9108950E942C6F0E948E56F0
:10D030000E94606885E393E09093482A8093472A92
:10D040000E94376A2FEF31E040E05EE160E074E07B
:10D0500082E090E00C94006ABC0187EE93E10C94AE
:10D060007C50BC0187EE93E10C946150CF93DF9329
:10D07000EC014091492A50914A2A60914B2A7091C3
:10D080004C2A4F5F5F4F6F4F7F4F4093492A509319
:10D090004A2A60934B2A70934C2A0E944C6A00974C
:10D0A00061F00E940E56E0913903F0913A03BE01FF
:10D0B00086EA97E6099581E090E0DF91CF910895A7
:10D0C0008DEE93E10C9418500F93CF93DF93EC0106
:10D0D0007B836A8318865F834E83BC018DEE93E168
:10D0E0000E947C50E091E913F091EA13309749F0E7
:10D0F0004C815D8101E020E030E068858A819B8180
:10D100000995DF91CF910F910895BC018DEE93E1C8
:10D110000C9461500F93DC0118961C921897E091C3
:10D12000E913F091EA13309759F000E020E030E085
:10D1300040E050E060E012968D919C911397099524
:10D140000F9108950F93DC01AB0114962D913C9142
:10D15000159781E018968C93189715967C936E938B
:10D160001497E091E913F091EA13309739F000E059
:10D1700061E012968D919C91139709950F910895F6
:10D180000F93DC01E091E913F091EA13309771F00D
:10D1900014964D915C91159701E09A0118966C9147
:10D1A000189712968D919C91139709950F91089558
:10D1B000E091EB13F091EC13309709F00994089586
:10D1C0009093EC138093EB1308959093EA1380935C
:10D1D000E91308958DEE93E10C941C50EF92FF92A9
:10D1E0000F931F93CF93DF938C01EB017A018DEEA8
:10D1F00093E10E941C500097D9F0DC0112962D910A
:10D200003C9113972C173D0781F41696ED91FC91F4
:10D210001797309769F09701AE01B801DF91CF9170
:10D220001F910F91FF90EF9009940E94C450E3CF9B
:10D23000DF91CF911F910F91FF90EF900895089586
:10D24000CF93DF93C0E2D4E16881798120E030E0C0
:10D250004FE359E68AE094E10E949C520E942A6FB3
:10D26000688179810E94D68620E030E043E559E666
:10D27000BC018AEF93E1DF91CF910C949C52809195
:10D2800020149091211420911E1430911F14880FA6
:10D29000991F2817390708F4C90190932114809326
:10D2A00020140C942069CF93DF930E948E560E9425
:10D2B000F555EC01198218820E94EA6828813981AB
:10D2C000009719F1FC0140854423F9F0FC014281EB
:10D2D0005381F901EE0FFF1FEE0FFF1FEC0FFD1F33
:10D2E00053834283FC01448155812F5F3F4FF901F5
:10D2F000EE0FFF1FEE0FFF1FEC0FFD1F518340834A
:10D30000398328830E94C450D9CFC901880F991F3F
:10D31000880F991F02960E94F05588819981892B68
:10D3200031F08FEE93E1DF91CF910C94744DDF914A
:10D33000CF910895AF92BF92CF92DF92EF92FF927A
:10D340000F931F93CF93DF9300D0CDB7DEB76B0160
:10D350000E94F555FC01008111811A8309830C306C
:10D36000110518F4E12CF12C0DC01F930F9389E2E5
:10D3700099E09F938F930E94848D0F900F900F9050
:10D380000F9021C0E016F106F1F00E94F555F7016B
:10D39000EE0FFF1FEE0FFF1FE80FF91FA280B380F3
:10D3A0000E94F555FFEFEF1AFF0AF701EE0FFF1F7E
:10D3B000EE0FFF1FE80FF91F40815181B501C60133
:10D3C0000E94EE68DFCF0F900F90DF91CF911F91F9
:10D3D0000F91FF90EF90DF90CF90BF90AF900895A6
:10D3E0000F93013059F480911A1490911B1490936B
:10D3F0002114809320140F910C9420690F910895AB
:10D40000EF92FF920F931F93CF93DF938B01EA016B
:10D41000790142E253E0BC018FEE93E10E94584D46
:10D4200010931B1400931A14D0931D14C0931C1452
:10D43000F0921F14E0921E1480EF99E6DF91CF91D5
:10D440001F910F91FF90EF900C94E5688AE094E1B2
:10D450000E9420538AEF93E10E9420538FEE93E1C4
:10D460000C94724D809120149091211408950C9485
:10D47000B24DCF93DF93E0912603F09127030995F6
:10D48000EC01009729F06A817B8181E00E940757B7
:10D49000CE01DF91CF9108950F931F93CF93DF9328
:10D4A000EC01E0912803F091290309958C016A8130
:10D4B0007B8181E00E94075781E090E0012B11F40D
:10D4C00080E090E0DF91CF911F910F910895E0915E
:10D4D0002A03F0912B03099420E030E00296FC012E
:10D4E00032974081442331F0FC0131974081240F71
:10D4F000311DF4CFC9010895FC01208130E0322FA5
:10D5000022278181282B02C0220F331F6A95E2F760
:10D51000832F9927FA01E45DFC4F208130E08223BC
:10D52000932328E030E0241B350B02C096958795A5
:10D530002A95E2F708956F927F928F929F92AF9211
:10D54000BF92CF92DF92EF92FF920F931F93CF93F0
:10D55000DF938C01EB016A0179012830310524F455
:10D56000A901B601CE014AC0590123E0B594A794A0
:10D570002A95E1F74115510521F04801612C712CE4
:10D5800003C0D801FB0120C048E050E0B601CE0145
:10D59000860D971D0E947C6AF40181934F01FFEF75
:10D5A0006F1A7F0A6A147B047CF3C501B7FE02C0C0
:10D5B00080E090E0A701477055274115510511F112
:10D5C000080F191FB60118C0CF018C1B9D0B8A15BF
:10D5D0009B051CF481918D93F7CFC501B7FE02C066
:10D5E00080E090E0A701477055274115510551F0A3
:10D5F000080F191F60E070E08C0F9D1F0E947C6A6D
:10D60000F8018083DF91CF911F910F91FF90EF90F0
:10D61000DF90CF90BF90AF909F908F907F906F9052
:10D6200008958F929F92AF92BF92CF92DF92EF9226
:10D63000FF920F931F93CF93DF9300D0CDB7DEB748
:10D640000E94F5558C0182E090E00E94D355892B11
:10D6500019F480E090E05DC0F801818190E0982F9E
:10D6600088272081820F911D0E94C34D7C01009765
:10D6700081F30E94F5554C01F7012681822F869592
:10D680008695869590E0422F477021E030E011F4B6
:10D6900020E030E0820F931F0E94D355892BC9F2FE
:10D6A000F70104811581C12CD12CF80180818823D8
:10D6B00079F1F801A180B12CB60133E07595679539
:10D6C0003A95E1F7A60147705527680D791D883115
:10D6D00068F09501CE0101960E949B6ABE016F5FC2
:10D6E0007F4FF80180810E941B570DC01A8219825A
:10D6F0009501CE0101960E949B6A69817A81F801A9
:10D7000080810E940757CA0CDB1C0E5F1F4FCDCFD4
:10D71000C7010F900F90DF91CF911F910F91FF9054
:10D72000EF90DF90CF90BF90AF909F908F90089533
:10D73000DC0150E0E0E1F0E0E61BF70BE21BF30B4D
:10D7400002C0440F551FEA95E2F78C91852B8C930C
:10D7500011968C911197842B11968C9308956F924A
:10D760007F928F929F92AF92BF92CF92DF92EF9271
:10D77000FF920F931F93CF93DF938C016B01EA010C
:10D780007901283031051CF44881C8015CC0390199
:10D7900053E0759467945A95E1F76115710521F08E
:10D7A0004E01A12CB12C03C0D801FE0127C0F40109
:10D7B00041914F0128E030E0B601C8018A0D9B1D60
:10D7C0000E94986BFFEFAF1ABF0AA614B7047CF350
:10D7D000C30177FE02C080E090E0970127703327F5
:10D7E0002115310509F43FC0C80FD91F488150E009
:10D7F000B601621B730B685F7F4F1CC0CF018C1B8F
:10D800009D0B861597051CF481918D93F7CFC3016D
:10D8100077FE02C080E090E0970127703327211542
:10D82000310509F1C80FD91F488150E068E070E068
:10D83000621B730B02C0559547956A95E2F760E04D
:10D8400070E0800F911FDF91CF911F910F91FF909A
:10D85000EF90DF90CF90BF90AF909F908F907F9090
:10D860006F900C94986BDF91CF911F910F91FF9067
:10D87000EF90DF90CF90BF90AF909F908F907F9070
:10D880006F9008956F927F928F929F92AF92BF9206
:10D89000CF92DF92EF92FF920F931F93CF93DF937C
:10D8A00000D0CDB7DEB78C01FC018681E82EE6946E
:10D8B000E694E694F12C282F277081E090E011F493
:10D8C00080E090E0E80EF91EC70102960E945756CC
:10D8D000009709F445C00E94FC55F8012281FC0123
:10D8E0002083F8012381FC0121830E94FC550296CC
:10D8F0005C01A70160E070E00E94D88CF80104810F
:10D900001581E12CF12CF8018081882339F1F8018F
:10D910008180912C670163E0D594C7946A95E1F703
:10D920003701F7E06F227724CA0CDB1C883128F01E
:10D930000E9425579401AC0108C00E9412579A8397
:10D9400089839401AE014F5F5F4FB301C6010E940E
:10D95000AF6BE80CF91C0E5F1F4FD5CF81E090E054
:10D960000F900F90DF91CF911F910F91FF90EF904B
:10D97000DF90CF90BF90AF909F908F907F906F90EF
:10D980000895E0914703F09148030994E091200342
:10D99000F09121030994E0914B03F0914C03099419
:10D9A000E0914D03F0914E03099480E090E00895DA
:10D9B0000895E0911803F0911903099480E090E034
:10D9C00008950F931F93CF93DF93CDB7DEB7E09702
:10D9D0000FB6F894DEBF0FBECDBF0E9442568C0139
:10D9E0000E94F555AE014F5F5F4F602F0E94B174EA
:10D9F000882309F446C088A99801281B3109C90168
:10DA00000E94D355892BE9F12E8121110CC0BE0152
:10DA10006A5E7F4F88E10E941B57E0913B03F091C3
:10DA20003C0309952EC08A859B858D3C3BEA930774
:10DA300011F0019631F5223019F088E090E002C033
:10DA400082E090E001979C012F5F3F4F1216130672
:10DA5000F4F6E1E0F0E0EC0FFD1FE80FF91F23857D
:10DA60002F3F81F3BE01645F7F4F89E10E941B5706
:10DA700089E10E94255766E578E20E94114D892BC5
:10DA800031F6E0960FB6F894DEBF0FBECDBFDF9142
:10DA9000CF911F910F910895AF92BF92CF92DF92D5
:10DAA000EF92FF920F931F93CF93DF93CDB7DEB723
:10DAB000E0970FB6F894DEBF0FBECDBF8C016B01AF
:10DAC000CE0101967C0180E3F70111928A95E9F776
:10DAD00081E089838CE00E9412578C831D821F8213
:10DAE0008091241491E0980F90932414898783E007
:10DAF000B82EB8868DEC9BEA9B878A8789E10E94C5
:10DB0000255764EF72E00E94114D892B31F082E0BD
:10DB10008E838FEF8C878D8709C089E10E942557FE
:10DB2000BC01CE010C960E94084DBE828DEC9BEA92
:10DB30009D8B8C8B66E578E2CE0146960E94084D5F
:10DB40000E94F5559FA78EA70E94425688ABC70139
:10DB50000E94AA73B82E90E00E945756892B31F18B
:10DB60000E94FC55BC014B2DC7010E94C873E09078
:10DB70000E03F0900F030E944C565C010E94FC556E
:10DB8000B501F70109950115110581F0009739F0EC
:10DB9000019761F441E050E064E070E004C041E0CE
:10DBA00050E060E070E0C601F8010995E0960FB61C
:10DBB000F894DEBF0FBECDBFDF91CF911F910F91C3
:10DBC000FF90EF90DF90CF90BF90AF9008950E94AC
:10DBD0002A6F80932414E0911803F091190309949B
:10DBE000892B29F0E0911803F091190304C0E0910A
:10DBF0001A03F0911B030994CF93DF93EC018991F1
:10DC00009991009729F060E070E00E945C4FF7CF97
:10DC1000DF91CF910895CF93DF93EC018991999192
:10DC2000009719F00E94AE4EF9CFDF91CF91089581
:10DC3000CF93DF93EC017B836A830E94C15F99835A
:10DC40008883DF91CF910895FC01808191812281A9
:10DC50003381820F931F918380830895CF93DF9345
:10DC6000EC010E94C15F99838883DF91CF91089571
:10DC7000CF93DF93EC010E94C15F28813981821B21
:10DC8000930B9C012F5F3F4F81E090E04A815B81C5
:10DC90004217530710F080E090E0DF91CF91089594
:10DCA000CF93DF93FC01C281D38180819181C80F22
:10DCB000D91F0E94C15F9E01281B390BC901DF914A
:10DCC000CF910895CF93DF93EFECFAE2C1E9DAE266
:10DCD000A3ECBAE211921192199219921992199227
:10DCE0001D928AE2E73EF807A9F7DF91CF910895E8
:10DCF000CF93DF93FC01ED53F54D40819C01220F42
:10DD0000331F220F331F442301F1A0919400B091DF
:10DD10009500FC01EE0FFF1FE153F54D80819181CD
:10DD2000AD01481B590BCA01E901CF56D54D4881B9
:10DD300059816A817B81480F591F611D711D48837C
:10DD400059836A837B83B183A083F901EF56F54D34
:10DD50006081718182819381DF91CF91089560E02C
:10DD600070E0CB010895FC01EE0FFF1FEE0FFF1FC7
:10DD7000EF56F54D40835183628373830895CF93AB
:10DD8000DF9323EC3AE2C1E9DAE2EFECFAE2D901FF
:10DD90008D919D018823B9F0409194005091950098
:10DDA00080819181BA01681B790B88819981AA8150
:10DDB000BB81860F971FA11DB11D88839983AA83FC
:10DDC000BB835183408324963296BAE22F3C3B07B3
:10DDD000F1F6DF91CF9108950C9439730F931F934F
:10DDE000FC01CB01409125145091261433832283EA
:10DDF0001583048371836083F0932614E0932514C4
:10DE0000452B11F40E94537380E090E01F910F9115
:10DE1000089580912514909126140097C1F01092D6
:10DE2000261410922514DC0114966D917C9115979F
:10DE30001296ED91FC9113970995E0912514F091BC
:10DE40002614309721F0808191810C9453730895AA
:10DE50000C9462890C945E898AEC92E00E94934F44
:10DE600082EC92E00C94934FCF93DF930E94025682
:10DE7000892BA9F082EC92E00E94B14FEC0100974F
:10DE800021F10E944256998388830E943D569B83CC
:10DE90008A83CE0104960E947E558CAB14C08AEC16
:10DEA00092E00E94B14FEC01009779F002960E9437
:10DEB000905599838883BE016E547F4FCE018E5753
:10DEC0009F4F0E94E556CE0102C080E090E0DF91B6
:10DED000CF910895BC016E547F4F8E579F4F0C9485
:10DEE000E556CF93DF93EC01BC018AEC92E00E94EF
:10DEF000FB4FBE01892B19F08AEC92E009C082EC3D
:10DF000092E00E94FB4F892B39F0BE0182EC92E037
:10DF1000DF91CF910C94D64FDF91CF9108950F935D
:10DF20001F93CF93DF93EC01BC018AEC92E00E9437
:10DF3000FB4F892B91F0FE0161917191CF010E94FD
:10DF4000A156BE016E547F4FCE018E579F4FDF9179
:10DF5000CF911F910F910C94F656BE0182EC92E086
:10DF60000E94FB4F892BD1F00E948E5668817981E7
:10DF70008A819B810E94A1568CA990E00E945756ED
:10DF80000CA910E00E94FC55BE016C5F7F4FA801F8
:10DF9000DF91CF911F910F910C94CF8CDF91CF9196
:10DFA0001F910F910895CF93DF93EC01BC018AEC90
:10DFB00092E00E94FB4F892B19F0CE0102960CC013
:10DFC000BE0182EC92E00E94FB4F892B19F08A81FE
:10DFD0009B8102C080E090E0DF91CF910895FC0129
:10DFE000808191810895860F911D860F911D8E5716
:10DFF0009F4F0895860F911D860F911D8E579F4F3D
:10E00000FC01808191810895089584E89AE10E943D
:10E01000D551892B21F084E89AE10C94C2510895DE
:10E02000E091701AF091711A309709F0099480E02C
:10E030000895EF92FF920F931F93CF93DF937C018C
:10E04000EA01FC0180819181009741F08C3093407E
:10E0500071F1F7011182108283E0F2C080E024E0C8
:10E06000829FF0011124EE58F54E118210828F5FCD
:10E070008430A8F380936F1A8091AA119091AB110C
:10E080009093831A8093821A0E94A74E8093E72A66
:10E0900060E470E084E89AE10E94AE510E94277625
:10E0A0008CE093E0F7019183808381E0C9C0623006
:10E0B000D9F48091E82A9091E92A892B89F38091FB
:10E0C000F92A863029F48091112B81FD0E94057078
:10E0D00081E00E9465778091E82A9091E92A892B56
:10E0E000F9F20E942972DCCF633060F5611114C02F
:10E0F0002097B1F2D093F62FC093F52F83E00E94C2
:10E1000065778091E82A9091E92A892B11F00E9485
:10E1100010700E940570C4CF613011F6209709F489
:10E12000BFCFD093F22FC093F12F85E00E94657787
:10E130008091E82A9091E92A892B09F4B1CF0E94B5
:10E140001070AECF6738E9F510926E1A02E71AE147
:10E1500080916E1A8430B8F4F801828193818C1713
:10E160009D0749F4808191810E943277F8011182E4
:10E170001082138212820C5F1F4F80916E1A8F5F84
:10E1800080936E1AE5CFE0E1F0E3838194818C17F0
:10E190009D0719F4148213821082B09620E3E039AF
:10E1A000F20799F7EDE8F0E3818592858C179D07DA
:10E1B00011F4158214823D9681E3EF30F807A1F740
:10E1C0006FCF683809F06CCFC458DA4109F068CFD6
:10E1D00084E89AE10E94D551892B09F461CF10920D
:10E1E0006E1AE0916E1AE43008F05ACF20E2E29FF6
:10E1F000F0011124E950F04D818D8823D9F084E895
:10E200009AE10E94C25180916E1AE0E28E9FC00195
:10E2100011248950904D9093F62F8093F52F82E032
:10E220000E9465778091E82A9091E92A892B11F064
:10E230000E94107080916E1A8F5F80936E1AD1CFFA
:10E24000DF91CF911F910F91FF90EF9008959093E0
:10E25000711A8093701A08952091AA113091AB1110
:10E2600060E0E2E7FAE1643098F4408151814817B8
:10E27000590759F4428153814217530731F460938F
:10E280006D1A118210820C94327734966F5FEBCF47
:10E2900060936D1A089540E0E2E7FAE14430A8F493
:10E2A00051E0540F20813181232B61F440936C1A8B
:10E2B000918380832091AA113091AB113383228303
:10E2C0000C944C773496452FE9CF40936C1A0895FF
:10E2D0002091AA113091AB11FC01358F248F778FDB
:10E2E000668F08952091AA113091AB11FC013287FD
:10E2F0002187748763870895CF93DF93EA010E9493
:10E30000D576009749F02091AA113091AB11FC010C
:10E3100032872187D487C387DF91CF9108950F93E8
:10E320001F93CF93DF9300D000D0CDB7DEB78C0121
:10E33000AB018FEF89838A838B838C83B801CE01F5
:10E3400001960E947C71009719F0FC0115830483EB
:10E350000F900F900F900F90DF91CF911F910F9121
:10E36000089540E050E062E082ED92E00E944D4F5F
:10E370001092E92A1092E82A0895AC0161E082ED3A
:10E3800092E00C942F4FAC0160E082ED92E00C948F
:10E390002F4F0F931F93CF93DF938A010E945376E1
:10E3A000EC01009759F08091AA119091AB119D8FCB
:10E3B0008C8F1F8F0E8FCE010E94C371CE01DF9113
:10E3C000CF911F910F910895CF93DF93A091F52FD7
:10E3D000B091F62F109719F0ED016C9605C0C09121
:10E3E000F12FD091F22F29968091F02F86FF22C035
:10E3F00010926B1A40E0E2E7FAE14430B8F4208171
:10E40000318114968D919C9115972817390759F4ED
:10E4100082819381009739F040936B1A99838883A6
:10E420001B821A8205C034964F5FE7CF40936B1A68
:10E430000E94057088819981009741F04A815B8133
:10E440006091E72ADF91CF910C944D4FDF91CF91EE
:10E4500008950F931F93CF93DF938091F92A86300D
:10E4600009F071C08091E82A9091E92A81159540C0
:10E4700009F069C0C4E9D2E0D093E92AC093E82A40
:10E4800002E00093F22A14E91093F32A1092152B5C
:10E490001092142B0E942176809590959093152BC5
:10E4A0008093142B1092FB2A1092FA2A0E94107665
:10E4B000809590959093FB2A8093FA2A0E94107081
:10E4C000D093E92AC093E82A0093F22A1093F32A02
:10E4D000A091F32FB091F42FFD01E459FD4F8CE68C
:10E4E00092E001900D920197E1F76CE672E088E00E
:10E4F0009BE20E94CF758091EC2A8093082B80913B
:10E50000ED2A8093092B8091EE2A80930A2B80912B
:10E51000EF2A80930B2B1092152B1092142B0E9434
:10E520002176809590959093152B8093142B1092C3
:10E53000FB2A1092FA2A0E9410768095909590936B
:10E54000FB2A8093FA2ADF91CF911F910F910C94AF
:10E550001070FC01680F791F80E048E1E617F707AB
:10E5600081F0219198E0322F3827532F517030FDE0
:10E5700084278695513009F480682695915099F743
:10E58000EDCF08951F920F920FB60F9211240BB684
:10E590000F922F933F934F935F936F937F938F933C
:10E5A0009F93AF93BF93EF93FF93809194009091CB
:10E5B00095009093D42A8093D32A81E08093C52A32
:10E5C00080917100807D809371000E94096F80911D
:10E5D000C52A8823D9F180919400909195004091AB
:10E5E000D32A5091D42A84179507A0F48091992AB0
:10E5F00090919A2AA0919B2AB0919C2A8C57914E77
:10E60000AF4FBF4F8093992A90939A2AA0939B2A49
:10E61000B0939C2A2091940030919500241B350BD7
:10E620008091992A90919A2AA0919B2AB0919C2A34
:10E63000820F931FA11DB11D8093992A90939A2A4E
:10E64000A0939B2AB0939C2A1092C52AFF91EF9128
:10E65000BF91AF919F918F917F916F915F914F91FA
:10E660003F912F910F900BBE0F900FBE0F901F90F8
:10E6700018959FB7F894E1E7F0E08081807D808372
:10E6800088B38F6288BB10929000E1E9F0E01082BD
:10E6900010929200109295001092940080818560F3
:10E6A00080839FBF08952FB7F8949093990080932B
:10E6B000980088B38F6288BBE1E7F0E080818260D8
:10E6C00080832FBF0895CF93DF93FC01DB0185E0AA
:10E6D000EB0119928A95E9F78581837011F082E048
:10E6E0008C938781837021F082E012968C9312972D
:10E6F0008581837081F08781837069F023893489F3
:10E70000818592852817390731F481E08483129638
:10E710001C92129701C0148285818370823021F08F
:10E72000833021F080E003C082E001C088E01196D0
:10E730008C93119787818370823021F0833021F090
:10E7400080E003C082E001C088E013968C93DF91E3
:10E75000CF910895CF93DF9300D000D01F92CDB713
:10E76000DEB7BE016F5F7F4F0E94637389819A811C
:10E77000890F8D5F9B81890F9C81890F9D81890FF6
:10E780000F900F900F900F900F90DF91CF91089501
:10E790004F925F926F927F928F929F92AF92BF92B1
:10E7A000CF92DF92EF92FF920F931F93CF93DF935D
:10E7B00000D000D000D0CDB7DEB78C017B01BE0108
:10E7C0006F5F7F4F4E830E946373B981AA815B8024
:10E7D0004C808B2F90E003962A2F30E0820F931FFE
:10E7E000850D911D642D70E0860F971F5D81850F4B
:10E7F000911D4E8150E0481759070CF49AC0F8015A
:10E80000818180FB662460F8712C43E0660C771CE4
:10E810004A95E1F7828180FB882480F8912C54E0AE
:10E82000880C991C5A95E1F7862880818770882A80
:10E83000838180FBAA24A0F8B12C85E0AA0CBB1C24
:10E840008A95E1F78A28848180FBCC24C0F8D12CFA
:10E8500096E0CC0CDD1C9A95E1F78C28F7018082BC
:10E86000F80145814370F4E04F9FA0011124F801A5
:10E8700086818370F0E18F9FC0011124482BF8013D
:10E880008781F0E48F9FC0011124482BF701418359
:10E89000F8018085F7018283B23059F4F80181854F
:10E8A000F7018383F8018285F701848395E0C92EFF
:10E8B00002C083E0C82EB0E080E090E0200F311F5E
:10E8C000DB2EDC0C0197BA1761F0A901480F591F24
:10E8D000FA01B384A7014D0D511DFA01B082BF5F4B
:10E8E000EFCF9D2DF2E05F120EC0D701AD0DB11D2F
:10E8F000F80183898C9381E08D0DD701A80FB11D9C
:10E900009E5F84898C9340E020E030E0060F171F63
:10E91000842F890F21503109441561F0D801A20FCD
:10E92000B31F55965C91D701A80FB11D5C934F5F43
:10E93000EFCF80E026960FB6F894DEBF0FBECDBFB6
:10E94000DF91CF911F910F91FF90EF90DF90CF90CB
:10E95000BF90AF909F908F907F906F905F904F90FF
:10E960000895BF92CF92DF92EF92FF920F931F9381
:10E97000CF93DF937C01D62EEA0182E0861708F060
:10E98000B2C0F701808186FBBB24B0F89181292FAA
:10E99000269526952370C92EC294C694C69453E03A
:10E9A000C522382F3770388383FB332730F93983FA
:10E9B00084FB332730F93A8385FB882780F98B83E2
:10E9C000BC822D83892F829583708E83CF82828132
:10E9D0008887222391F13381848190E0982F8827C2
:10E9E000830F911D9A87898787010B5F1F4F223004
:10E9F00079F464EF72E0CE010B960E94084DF701A6
:10EA000086818B8785818C878701095F1F4F20C096
:10EA10002330F1F4F7013D9680E090E03E2F2F2F58
:10EA20004291DE01A80FB91F1B964C9301968830C6
:10EA30009105B1F7032F122F0BC087010D5F1F4FF8
:10EA400064EF72E0CE010B960E94084D1A8619867B
:10EA5000CC20B9F1B1100DC0F8012081818190E086
:10EA6000982F8827820F911D9C8B8B8B0E5F1F4FD9
:10EA700004C089859A859C8B8B8BF2E0CF120EC0E7
:10EA800064EF72E0CE0145960E94084DF801818145
:10EA90008D8B80818E8B0E5F1F4F1BC0F3E0CF12DA
:10EAA00018C0085F1F4FF80180E090E02291DE015E
:10EAB000A80FB91F55962C93019688309105B1F790
:10EAC00008C064EF72E0CE0145960E94084D1C8A92
:10EAD0001B8AC8018E199F092D2D281B2FA71EA741
:10EAE0000DA7D81608F480E0DF91CF911F910F9108
:10EAF000FF90EF90DF90CF90BF900895FB014150C1
:10EB00005109460F571FE417F50778F4208130E0CC
:10EB1000322F22276181260F311D820F931F82170A
:10EB2000930708F401963296EECFE417F50751F4F7
:10EB3000208130E0322F2227820F931F8217930704
:10EB400008F401960895CF93DF93C091F32AD0E0A3
:10EB500064972091F22A30E0322F2227C20FD31F70
:10EB600048E050E06CEF7AE29E01280F311DC901A8
:10EB70000E947E75AE0164E07BE20E947E75009784
:10EB800021F098278927982702C08FEF9FEFDF9108
:10EB9000CF91089590939D1A80939C1A0895FC013B
:10EBA0005381560F5093EF2A872F99274281480FA0
:10EBB0004093EE2AA181A093ED2AE081E093EC2A14
:10EBC000242F30E02817390748F481E08A0F80931A
:10EBD000ED2A811103C0EF5FE093EC2A852F90E0CE
:10EBE00077278617970788F44F5F4093EE2A4111E5
:10EBF0000CC08091ED2A8F5F8093ED2A811105C0B2
:10EC00008091EC2A8F5F8093EC2A0895AB01BC01C0
:10EC100080E090E00E947E759827892798270895C4
:10EC200044E150E060EF7AE280E090E00E947E757F
:10EC3000009721F098278927982708958FEF9FEF55
:10EC4000089586E00C94A37581E10C94A37580E08F
:10EC5000E82FF0E0EE0FFF1FE958FF4C1182108201
:10EC60008F5F8430A8F380E090E2899FF001112447
:10EC7000E950F04D118E8F5F8430B0F380E094E066
:10EC80009093971A8093961A80E09DE0989FF001E8
:10EC90001124E357FF4C158214828F5F8A30B0F342
:10ECA0008093951A0895CF932091961A3091971AD0
:10ECB0002F5F3F4F21154DE7340710F020E030E182
:10ECC000522F432FE7EFFFE2C0E0C43059F0A18D8F
:10ECD000AA2329F0A481B581A417B50749F3CF5F12
:10ECE000B096F3CF3093971A2093961A1092951AF4
:10ECF00020E0E0E0F0E02430E8F430E2239FD001AF
:10ED00001124A950B04D59963C915997311104C026
:10ED10002093951AFD0110C0373041F4309739F037
:10ED20005A964C915A97328D341708F0DF012F5FB5
:10ED3000FD01E1CF2093951A3097A1F122E0218FB8
:10ED40002091981A24872091991A258720919A1A40
:10ED5000268720919B1A278728ED34E0338B228B5E
:10ED6000358B248B21E030E0318B208B138E21E01A
:10ED7000228F23E0208F168A20E1278B2091961A7C
:10ED80003091971A322723273227358324837783BC
:10ED90006683DC014D915D916D917C91408351833F
:10EDA00062837383CF01CF910895CF93DF93209136
:10EDB000961A3091971A2F5F3F4F21154DE7340770
:10EDC00010F020E030E1522F432FE1E9F0E3C0E002
:10EDD000CA3041F0A081B181CF5F3D96A417B5073D
:10EDE000B9F7E9CF3093971A2093961A40E05DE087
:10EDF0004A30A0F4A1E0A40F549FF0011124E3577E
:10EE0000FF4C24813581232B39F44093951A309798
:10EE100041F480E090E023C04A2FEACF4093951A56
:10EE2000F8CF2091961A3091971A3227232732274C
:10EE30003583248377836683009729F410821182B7
:10EE40001282138209C0EC0188819981AA81BB8159
:10EE500080839183A283B38380E48087CF01DF9195
:10EE6000CF91089540E04430A0F4E42FF0E051E069
:10EE7000540FEE0FFF1FE958FF4C208131812817F6
:10EE8000390729F44093951A118210820895452F6D
:10EE9000EACF4093951A089540E0443098F4E42F67
:10EEA000F0E051E0540FEE0FFF1FE958FF4C2081B6
:10EEB0003181232B29F44093951A918380830895FF
:10EEC000452FEBCF4093951A0895AF92BF92CF9202
:10EED000DF92EF92FF920F931F93CF93DF93C09136
:10EEE000F52FD091F62F843009F4DCC128E13BE204
:10EEF0003093F42F2093F32F3093EB2A2093EA2AB8
:10EF0000833059F4898D8F70833009F06BC0888904
:10EF10009989892B09F0DFC67FC0823009F080C053
:10EF200080919B1A8F5F80939B1A811113C08091EF
:10EF30009A1A8F5F80939A1A81110CC08091991A46
:10EF40008F5F8093991A811105C08091981A8F5F05
:10EF50008093981A1092E92A1092E82A10928C3025
:10EF600010928B30298D822F8D7F853041F48A8DD0
:10EF70008F5F8A8F843109F0AEC6198EACC622230A
:10EF800009F4A9C688899989892B09F441C08A8D19
:10EF90009FEF980F9A8F81119EC68B8D883031F02C
:10EFA0009FEF920F923048F4853039F4198E80E843
:10EFB0008093F02F0E94E47147C5853038F493E0C8
:10EFC000082E01C0990F0A94EAF701C090E39A8FC6
:10EFD0008F5F8B8F822F8F708330A1F048F4813048
:10EFE00009F44FC3823009F076C61092112B4CC33E
:10EFF000863009F4C8C4883009F4C5C4843009F0E7
:10F000006AC6C1C484E08093F02F0E94E4714EC5AB
:10F010002F70233009F05FC688E08093F02F09C578
:10F02000853019F5E091F12FF091F22F84819581CF
:10F03000892B09F450C61092F62F1092F52F8CE010
:10F040009BE29093F42F8093F32F9093EB2A80937D
:10F05000EA2A10928C3010928B301092E92A10928A
:10F06000E82A88E08093F02F1BC18091F02A853434
:10F0700009F031C60091F22A10E0102F002780918C
:10F08000F32A080F111D8091E82A9091E92A801730
:10F09000910708F420C61093E92A0093E82A80918A
:10F0A000F62A8F7309F017C68091F72A811113C6CB
:10F0B0008091873090918830C0915103D091520354
:10F0C0008C179D0759F44091893050918A302091D6
:10F0D00053033091540342175307A1F02091002BA2
:10F0E0003091012B2817390709F0F5C52091022B23
:10F0F0003091032B8091893090918A3028173907FD
:10F1000009F0E9C50E941076019609F0E4C58091E6
:10F11000F92A863009F429C18131E9F1813009F0F9
:10F12000DAC58091042B883009F0D5C51092042BE4
:10F130008091062B9091072B873F3FEF930710F0AC
:10F14000099601C008969093072B8093062B809117
:10F15000FC2A9091FD2AA091FE2AB091FF2A80936B
:10F16000002B9093012BA093022BB093032B809143
:10F17000873090918830A0918930B0918A30809307
:10F18000FC2A9093FD2AA093FE2AB093FF2A80E4E4
:10F190008093F82A7DC50C5111091093E92A009338
:10F1A000E82A8CE09BE29093F42F8093F32F8091D8
:10F1B0000A2B90910B2B892B29F00E942476019623
:10F1C00009F089C52091062B3091072B21153105B7
:10F1D00009F481C58DE890E39093F22F8093F12F8D
:10F1E000A090042BB090052B4091530350915403F1
:10F1F0006091550370915603A0915703B091580345
:10F200000091FC2A1091FD2AE090FE2AF090FF2A3E
:10F21000E091F12FF091F22F81E3EF30F80708F041
:10F220005AC584819581009721F12817390709F57E
:10F2300086819781009719F0A816B906D1F48081CC
:10F2400091818C179D0729F4C280D380C416D506FE
:10F25000B1F08617970729F4C280D380CA16DB065F
:10F2600071F00817190729F482819381E816F906CD
:10F2700031F03D96F093F22FE093F12FC9CF109229
:10F28000F62F1092F52F82E08093F02F8CE09BE216
:10F290009093EB2A8093EA2A10928C3010928B3054
:10F2A0000E94E47180918B3090918C30009709F42A
:10F2B00012C59C01245E3F4F3093E92A2093E82A2F
:10F2C0003093F22A2093F32AE091F12FF091F22F5C
:10F2D00020852093F82A21E12093F92A089698277F
:10F2E000892798279093092B8093082B10920B2B3A
:10F2F00010920A2B848195819093052B8093042B87
:10F30000868197819093072B8093062B809187307D
:10F3100090918830A0918930B0918A308093FC2AF6
:10F320009093FD2AA093FE2AB093FF2A80819181B9
:10F33000A281B3818093002B9093012BA093022B89
:10F34000B093032B88E19BE29093F42F8093F32FEB
:10F350000E94247680959095009711F48FEF9FEF8F
:10F3600090930B2B80930A2B93C40E9421760196D5
:10F3700009F0B1C48091062B9091072B009709F4F6
:10F38000AAC42091042B3091052B2115310509F4D5
:10F39000A2C44091FC2A5091FD2A6091FE2A7091EE
:10F3A000FF2AE0E1F0E3C7EFDFE2F080FF20A9F001
:10F3B000AC81BD818A179B0781F4AE81BF812A177A
:10F3C0003B0759F4A881B9814A175B0731F4AA8138
:10F3D000BB816A177B0709F46FC1A096B096A0E3C2
:10F3E000C737DA0711F72091112B2F732230D9F488
:10F3F0009093931A8093921A40E0443090F4E42F53
:10F40000F0E0EE0FFF1FE958FF4C208131814F5F84
:10F410008217930791F71092951A20E0C0E0D0E090
:10F420007EC04093951A8091112B82FD54C484E1D3
:10F430008093112B88E290E09093E92A8093E82A48
:10F4400080E58093102B80910B2B90910F2B909344
:10F450000B2B30910A2B90910E2B90930A2B30930B
:10F460000E2B2091092B90910D2B9093092B20931B
:10F470000D2B9091082B9093951A40910C2B409353
:10F48000082B90930C2B8F5F80930F2B81110FC053
:10F4900081E0830F80930E2B811109C081E0820FE0
:10F4A00080930D2B811103C09F5F90930C2B809153
:10F4B000042B9091052B9093931A8093921A20918C
:10F4C000062B3091072B3093052B2093042B909320
:10F4D000072B8093062B8091FC2A9091FD2AA09106
:10F4E000FE2AB091FF2A8093002B9093012BA093CA
:10F4F000022BB093032B8091873090918830A0919C
:10F500008930B0918A308093FC2A9093FD2AA09391
:10F51000FE2AB093FF2AA1C3373089F02F5F243031
:10F52000C0F430E2239FC0011124FC01E950F04DEA
:10F53000318D3111F1CF2093951AEF010CC0209736
:10F5400021F0428D3A8D341748F7EC01C950D04D67
:10F55000E5CF2093951A209709F4BDC3D093F62FD9
:10F56000C093F52F83E08A8F888F1E8A84E08F8B6B
:10F570001B8E8091062B9091072B9D838C8380910D
:10F58000042B9091052B9F838E838091FC2A909170
:10F59000FD2AA091FE2AB091FF2A88839983AA832D
:10F5A000BB8381E0898F8091981A8C878091991A0A
:10F5B0008D8780919A1A8E8780919B1A8F8781E020
:10F5C00090E0998B888B80910B2B8B8780910A2BF5
:10F5D0008A878091092B89878091082B888781E011
:10F5E00090E00E94CF7E8091102B282F207F30E06A
:10F5F000213531050CF445C082958F7090E0059758
:10F60000880F991F880F991F3091941A20E0E22FDC
:10F61000F0E0E817F9078CF5E051F54D30A5311110
:10F6200005C02093951A1092941A2BC0313011F412
:10F630002F5FEDCF3230E1F441A54430C9F420937F
:10F64000951A3093941A82A590E0982F882723A5C5
:10F65000822B9093931A8093921A893DA4E09A0783
:10F6600010F088ED94E09B8B8A8B9D8B8C8B09C06E
:10F6700041A5442311F0240FCACF2093951A30934B
:10F68000941A80E18093112B8091112B82608093DA
:10F69000112B82E08093182B84E08093192B8093A8
:10F6A0001A2B88ED80931B2B8CE290E09093E92A33
:10F6B0008093E82A80E67EC2D093F62FC093F52F80
:10F6C0001092F02F9091112B92FF03C0198E80E2BF
:10F6D0001AC28091102B82958F70880F880F8093AB
:10F6E000951A081B1109045111091093E92A009376
:10F6F000E82A8F2D8F70823029F4892F8F73823101
:10F7000039F41FC0813021F4892F8F738230C9F002
:10F71000012B19F4892F8370A1F02091082B888583
:10F7200028133EC22091092B8985281339C22091C4
:10F730000A2B8A85281334C220910B2B8B85281322
:10F740002FC294FF4AC0688979896115710509F44F
:10F7500044C0CE010C960E94CF7530910C2B809145
:10F76000EC2A38133AC020910D2B8091ED2A2813F2
:10F7700034C090910E2B8091EE2A98132EC0809168
:10F780000F2B4091EF2A841328C03C872D879E873A
:10F790008F878B8D81111AC02E89888D9A8D891B38
:10F7A000922F969596959695891B280F2E8B87FDFF
:10F7B00081959F89392F36953695931B980F9F8B8E
:10F7C000822F869586958695890F888F81E0809314
:10F7D000F02F888D8A8F198A188A498D842F8F700F
:10F7E00090E0FC013197E830F10508F074C2E05771
:10F7F000FF4F0C949A888091F02F80FF14C083E013
:10F80000898F80E48093F02F198A188A8091E82AE2
:10F810009091E92A009709F408C122E42093F02F7F
:10F820000E94CF7E02C18091112B8F73823009F02C
:10F8300052C227CF8091F02F80FF70C08091112B92
:10F840008F73823109F06AC08091102B282F207F9E
:10F8500030E0213531050CF445C082958F7090E081
:10F860000597880F991F880F991F3091941A20E0EF
:10F87000E22FF0E0E817F9078CF5E051F54D30A5DF
:10F88000311105C02093951A1092941A2BC0313073
:10F8900011F42F5FEDCF3230E1F441A54430C9F4CB
:10F8A0002093951A3093941A82A590E0982F882778
:10F8B00023A5822B9093931A8093921A893D24E07A
:10F8C000920710F088ED94E09B8B8A8B9D8B8C8B3C
:10F8D00009C041A5442311F0240FCACF2093951AE3
:10F8E0003093941A83E0898F8091082B88878091C8
:10F8F000092B898780910A2B8A8780910B2B8B8714
:10F9000081E090E00E94CF7E82E48093F02F198AFC
:10F91000188A1092E92A1092E82A87C080E2809320
:10F92000F02F0E94E471E091F52FF091F62F118EE7
:10F930007ACD8091112B80FF28C044FD26C0888994
:10F940009989892B09F0C7C18091E82A9091E92A09
:10F9500001960E94CF7E2091F02F822F80618093AC
:10F96000F02F8091E82A9091E92A892B19F02261E1
:10F970002093F02F0E94E47181E090E0998B888BB6
:10F9800088E0898F1B8E81E10CC185FF1CC08091AE
:10F99000162B90E0982F88272091172B822B2091EF
:10F9A000F32F3091F42F280F391F3093F42F209329
:10F9B000F32F2091E82A3091E92A281B390B309344
:10F9C000E92A2093E82A8091E82A9091E92A009771
:10F9D00049F044FD07C02091F02F22602093F02FC2
:10F9E0000E94CF7E8091122B90E0982F8827209143
:10F9F000132B820F911D9093931A8093921A2C8946
:10FA00003D892817390710F0892B21F43093931A78
:10FA10002093921A8091921A9091931A9B8B8A8BC1
:10FA20008091F02F837009F456C110928C3010929F
:10FA30008B300E94E4718091F02F85FF07C01092F7
:10FA40008C3010928B30198E84E1ABC084FF0AC0D9
:10FA500010928C3010928B3081E090E0998B888BE3
:10FA600084E08FCF20918B3030918C30211531057F
:10FA7000E1F080FF02C0198A188A88899989009765
:10FA800081F48A899B898217930720F490938C30A4
:10FA900080938B3080918B3090918C30998B888BB8
:10FAA00004C090938C3080938B301B8E8091EA2A17
:10FAB0009091EB2A9093F42F8093F32F80918B30C9
:10FAC00090918C30892B59F088899989009739F069
:10FAD00088969093E92A8093E82A88E10BC0809168
:10FAE000F02F81FFF8C088E290E09093E92A80939C
:10FAF000E82A80E18093112B5CC08091F02F80FF79
:10FB0000EAC0198E80E18093F02F0E94E471E3C077
:10FB10008091E82A9091E92A009711F00E94CF7E07
:10FB20009091112B8091F02F90FF0BC080FF06C0A9
:10FB300087E0898F1A8E198A188A19C086E0898F02
:10FB400016C080FF1EC085E0898F198A188AC3C03D
:10FB50008091E82A9091E92A009711F00E94CF7EC7
:10FB60008091112B80FF0DC087E0898F1A8E81E074
:10FB700090E00E94CF7E80E18093F02F0E94E4719C
:10FB80000FC08091E82A9091E92A892B49F4A3C0FB
:10FB90008091F02F80FF9FC087E0898F1A8E9BC0D5
:10FBA00080E18093112B88E290E09093E92A809382
:10FBB000E82A80E58093102B888580930C2B89851B
:10FBC00080930D2B8A8580930E2B8B8580930F2B32
:10FBD0008C858093082B8D858093092B8E8580934F
:10FBE0000A2B8F8580930B2B86E08093F92A8C81DA
:10FBF0009D819093052B8093042B8E819F81909300
:10FC0000072B8093062B8091873090918830A091AC
:10FC10008930B0918A308093FC2A9093FD2AA0937A
:10FC2000FE2AB093FF2A88819981AA81BB818093A3
:10FC3000002B9093012BA093022BB093032B898D63
:10FC400084FF05C01092132B1092122B06C084E083
:10FC50008093122B88ED8093132B80E48093F82AF5
:10FC60008091E82A9091E92A9093F22A8093F32ACE
:10FC70001092172B1092162B1092152B1092142BFA
:10FC80000E942176809590959093152B8093142B4C
:10FC900085E48093F02A1092F12A1092F72A1092AC
:10FCA000F62A80919C1A90919D1A019690939D1A24
:10FCB00080939C1A9093F42A8093F52A1092FB2A41
:10FCC0001092FA2A0E941076809590959093FB2AC4
:10FCD0008093FA2A04C01092E92A1092E82A10921E
:10FCE000F02FDF91CF911F910F91FF90EF90DF9058
:10FCF000CF90BF90AF9008959827892798270895AF
:10FD00000E94A0880895FC018091EA2A9091EB2A34
:10FD100020EF3FE2281B390BAB01261737070CF405
:10FD2000A9011416150654F450938C3040938B306F
:10FD3000E817F90719F0BF010C94CF8C089580E8FB
:10FD400080936100109261000E94555D0E94C44E34
:10FD50000E9431618091972890919828009729F00E
:10FD600001979093982880939728C0909928D090D5
:10FD70009A28E0909B28F0909C280E94EF5FC6167E
:10FD8000D706E806F90611F30E94EF5F6093992801
:10FD900070939A2880939B2890939C28D7CF20918A
:10FDA000F52F3091F62FBC01C90108960E94CF753E
:10FDB000E091F52FF091F62F8091EC2A80878091C9
:10FDC000ED2A81878091EE2A82878091EF2A8387AE
:10FDD00008952F923F924F925F926F927F928F92EF
:10FDE0009F92AF92BF92CF92DF92EF92FF920F93CA
:10FDF0001F93CF93DF93CDB7DEB763970FB6F89419
:10FE0000DEBF0FBECDBF7C011B016A01FC01178262
:10FE10001682838181FF66C3BE016F5F7F4F4B01F6
:10FE2000F7019381F10193FD859193FF81911F016A
:10FE3000882309F453C3853239F493FD859193FFE8
:10FE400081911F01853239F4B70190E00E94528DF3
:10FE500056016501E5CF10E0512C20E02032A0F4DE
:10FE60008B3269F030F4803259F0833269F42061CA
:10FE70002CC08D3239F0803339F4216026C02260E5
:10FE8000246023C0286021C027FD27C030ED380F33
:10FE90003A3078F426FF06C0FAE01F9F300D112497
:10FEA000132F13C06AE0569E300D1124532E20628A
:10FEB0000CC08E3221F426FD11C3206406C08C369E
:10FEC00011F4206802C0883641F4F10193FD859158
:10FED00093FF81911F018111C1CF9BEB980F93304C
:10FEE00018F42061805E06C09BE9980F933008F0FB
:10FEF000AAC12F7E26FF16E02F73722E853621F4BD
:10FF0000F22FF0647F2E08C0863621F4622F6068DD
:10FF1000762E02C01111115077FE07C01C3348F431
:10FF200044244394410E27E00BC0183030F4212FB5
:10FF300006C027E04CE3442E03C027E017E0412C25
:10FF4000560174E0A70EB11CF601608171818281B7
:10FF50009381042DA4010E94D78B6C01098100FFBD
:10FF600002C003FF06C071FC07C072FC08C0612C10
:10FF700008C03DE2632E05C02BE2622E02C090E273
:10FF8000692E802F8C7099F1662011F084E001C0F9
:10FF900083E0851510F0512C0BC0581A73FC08C073
:10FFA000B70180E290E00E94528D5A94C9F7F3CFD6
:10FFB000662029F0B701862D90E00E94528D03FD46
:10FFC00003C00EE410E102C00AE410E1F72DF07165
:10FFD0007F2EF8018491882309F476C27110805233
:10FFE000B70190E00E94528D0F5F1F4FF2CF77FE56
:10FFF0000FC04C0C04FF04C08A81813309F44A9479
:020000021000EC
:10000000141474F5F8E0F41578F588E0482E2CC047
:1000100076FC2AC0812F90E08C159D059CF06CEF3A
:10002000C6166FEFD60674F0772D7068772E0AC06B
:10003000E2E0F0E0EC0FFD1FE10FF11D8081803365
:1000400019F411501111F4CF77FE0EC044244394DB
:10005000410E812F90E0C816D9062CF41C1904C05B
:100060004424439401C010E077FE07C01C141D0413
:100070003CF496012F5F3F4F05C025E030E002C001
:1000800021E030E0662011F02F5F3F4F112331F067
:10009000412F50E04F5F5F4F240F351F452D50E03B
:1000A0002417350714F4521A01C0512C872D89707A
:1000B00049F4552039F0B70180E290E00E94528D5A
:1000C0005A94F7CF662029F0B701862D90E00E9460
:1000D000528D73FC09C0552039F0B70180E390E0E0
:1000E0000E94528D5A94F7CF77FE5FC09C2D8D2DC4
:1000F000D7FE02C090E080E0692E782E40E050E00C
:10010000C601841991099D878C87960126193709A4
:10011000280D391D812F90E0EE27FF27E81BF90BF2
:10012000FF87EE87FFEF6F167F0669F4B7018EE257
:1001300090E02B8B3A8B488B598B0E94528D5989BA
:1001400048893A892B89C614D70454F06C857D857B
:10015000661577052CF4F901E40FF51F818101C0C4
:1001600080E371E0671A71084F5F5F4FEE85FF858E
:100170006E167F066CF0B70190E02B8B3A8B488BA4
:10018000598B0E94528D2B893A8948895989CACF47
:100190006C147D0439F49A81963318F4953311F474
:1001A00004FF81E3B70190E04BC08A81813309F0FD
:1001B0000F7EB70190E00E94528D111105C074FEB0
:1001C00018C085E490E017C0B7018EE290E00E946D
:1001D000528D82E066246394680EF401E80FF11DED
:1001E0008081B70190E00E94528D115041F3862D1D
:1001F000F1CF85E690E0B7010E94528DD7FC05C093
:10020000C114D10439F404FF05C0D194C194D108BC
:100210008DE201C08BE2B70190E00E94528D80E335
:100220006AE0C616D1042CF08F5FFAE0CF1AD1082D
:10023000F7CFB70190E00E94528DB701C601C0967A
:100240000E94528D41C1833631F0833779F0833576
:1002500009F058C021C0560172E0A70EB11CF6018A
:100260008081898301E010E0640114C05601F2E04E
:10027000AF0EB11CF601C080D18026FF03C0612FF4
:1002800070E002C06FEF7FEFC6012B8B0E94FE8CE7
:100290008C012B892F7715C05601F2E0AF0EB11CEF
:1002A000F601C080D18026FF03C0612F70E002C03C
:1002B0006FEF7FEFC6012B8B0E94C08C8C012B89C6
:1002C0002068722E23FD1AC0852D90E008171907AB
:1002D000A8F4B70180E290E00E94528D5A94F4CFC6
:1002E000F60177FC859177FE81916F01B70190E06F
:1002F0000E94528D51105A94015011090115110597
:1003000079F7E2C0843611F0893651F5560127FF9E
:1003100009C0F4E0AF0EB11CF601608171818281E9
:1003200093810AC0F2E0AF0EB11CF60160817181C9
:10033000882777FD8095982F022F0F7697FF08C0AA
:1003400090958095709561957F4F8F4F9F4F006876
:100350002AE030E0A4010E948C8EC82EC8183EC04E
:10036000022F853721F40F7E2AE030E01DC0097F7F
:100370008F3691F018F4883559F0B0C0803719F0F5
:10038000883711F0ABC0006104FF09C0046007C0EA
:1003900024FF08C0066006C028E030E005C020E168
:1003A00030E002C020E132E0560107FF09C0F4E06E
:1003B000AF0EB11CF601608171818281938108C00A
:1003C000F2E0AF0EB11CF6016081718180E090E037
:1003D000A4010E948C8EC82EC8180F7706FF0BC090
:1003E000202F2E7FC11650F404FF0AC002FD08C062
:1003F000202F2E7E05C0DC2C202F03C0DC2C01C05A
:10040000D12E24FF0DC0FE01EC0DF11D8081803343
:1004100011F4297E09C022FF06C0D394D39404C0EE
:10042000822F867809F0D39423FD13C020FF06C0E5
:100430001C2DD51418F4150D1D19D52CD51468F4E0
:10044000B70180E290E02B8B0E94528DD3942B89D0
:10045000F5CFD51410F45D1801C0512C24FF12C043
:10046000B70180E390E02B8B0E94528D2B8922FFF5
:1004700017C021FF03C088E590E002C088E790E044
:10048000B7010CC0822F867859F021FD02C080E2AE
:1004900001C08BE227FD8DE2B70190E00E94528DF2
:1004A000C11638F4B70180E390E00E94528D1150DC
:1004B000F7CFCA94F401EC0DF11D8081B70190E0F3
:1004C0000E94528DC110F5CF552009F4C2CCB7015E
:1004D00080E290E00E94528D5A94F6CFF701868117
:1004E000978102C08FEF9FEF63960FB6F894DEBF3F
:1004F0000FBECDBFDF91CF911F910F91FF90EF9075
:10050000DF90CF90BF90AF909F908F907F906F9033
:100510005F904F903F902F9008955058BB27AA2787
:100520000ED04EC23FD230F044D220F031F49F3F83
:1005300011F41EF4FFC10EF4E095E7FBF5C1E92FBD
:1005400050D280F3BA17620773078407950718F033
:1005500071F49EF568C20EF4E0950B2EBA2FA02D13
:100560000B01B90190010C01CA01A0011124FF2760
:10057000591B99F0593F50F4503E68F11A16F0405B
:10058000A22F232F342F4427585FF3CF469537955A
:100590002795A795F0405395C9F77EF41F16BA0B1F
:1005A000620B730B840BBAF09150A1F0FF0FBB1FCD
:1005B000661F771F881FC2F70EC0BA0F621F731F16
:1005C000841F48F4879577956795B795F7959E3F73
:1005D00008F0B3CF9395880F08F09927EE0F979501
:1005E00087950895DFD158F080E891E009F49EEFF7
:1005F000E0D128F040E851E059F45EEF09C09AC11B
:1006000012C2E92FE078EDD168F3092E052AC1F373
:10061000261737074807590738F00E2E07F8E02548
:1006200069F0E025E0640AC0EF6307F8009407FA78
:10063000DB01B9019D01DC01CA01AD01EF9347D097
:10064000BFD10AD05F91552331F02BED3FE049E453
:1006500050FD49EC63CF0895DF93DD27B92FBF77B5
:1006600040E85FE31616170648075B0710F4D92F1A
:10067000E1D19F938F937F936F9346D3E0E3F1E0B3
:100680006CD19ED12F913F914F915F919AD2DD23F2
:1006900049F09058A2EA2AED3FE049EC5FE3D078B8
:1006A0005D274DDFDF918CC11BD108F481E00895F7
:1006B0000CD086C17ED140F075D130F021F45F3F7F
:1006C00019F032C15111B0C135C18BD198F39923C2
:1006D000C9F35523B1F3951B550BBB27AA27621706
:1006E0007307840738F09F5F5F4F220F331F441F4B
:1006F000AA1FA9F333D00E2E3AF0E0E830D0915083
:100700005040E695001CCAF729D0FE2F27D0660F6F
:10071000771F881FBB1F261737074807AB07B0E8AE
:1007200009F0BB0B802DBF01FF2793585F4F2AF0C4
:100730009E3F510568F0F8C077C15F3FECF3983EEB
:10074000DCF3869577956795B795F7959F5FC9F721
:10075000880F911D9695879597F90895E1E0660FAA
:10076000771F881FBB1F621773078407BA0720F023
:10077000621B730B840BBA0BEE1F88F7E09508958C
:1007800019F40EF0D1C04FC1D5C033D1C8F396389B
:10079000C0F707F80F92E8942BE33AEA48EB5FE7DB
:1007A00012D20F920F920F924DB75EB70F92CAD12D
:1007B000EDE5F1E0D2D04F915F91EF91FF91E5959A
:1007C000EE1FFF1F49F0FE57E0684427EE0F441F5D
:1007D000FA95E1F74195550B36D10F9007FE2AC1E6
:1007E000089597FB0EF4A9D03EC0E89409C097FB8A
:1007F0003EF490958095709561957F4F8F4F9F4FF8
:100800009923A9F0F92F96E9BB279395F69587953B
:1008100077956795B795F111F8CFFAF4BB0F11F4FE
:1008200060FF1BC06F5F7F4F8F4F9F4F16C08823A5
:1008300011F096E911C0772321F09EE8872F762FDB
:1008400005C0662371F096E8862F70E060E02AF01C
:100850009A95660F771F881FDAF7880F9695879508
:1008600097F90895E894F92F96EBFF2381F012167B
:1008700013061406440B9395F6958795779567951F
:1008800057954040FF23B9F71BC099270895882347
:1008900051F49850D2F7872B762F652F542F432F82
:1008A000322F20E0B1F3121613061406440B8823EE
:1008B0003AF09A95440F551F661F771F881FCAF795
:1008C00055234AF4440F551F11F460FF04C06F5FB5
:1008D0007F4F8F4F9F4F880F9695879597F9089573
:1008E000990F0008550FAA0BE0E8FEEF1616170641
:1008F000E807F907C0F012161306E407F50798F0A9
:10090000621B730B840B950B39F40A2661F0232BC1
:10091000242B252B21F408950A2609F4A140A6953D
:100920008FEF811D811D089597F99F6780E870E022
:1009300060E008959FEF80EC089590958095709504
:10094000609550954095309521953F4F4F4F5F4FA3
:100950006F4F7F4F8F4F9F4F0895DF93CF931F931C
:100960000F93FF92EF92DF927B018C01689405C098
:10097000DA2EEF0126D1FE01E894A591259135915B
:1009800045915591AEF3EF01DADDFE019701A80123
:10099000DA9479F7DF90EF90FF900F911F91CF914C
:1009A000DF91089500240A94161617061806090602
:1009B000089500240A9412161306140605060895D5
:1009C000092E0394000C11F4882352F0BB0F40F45D
:1009D000BF2B11F460FF04C06F5F7F4F8F4F9F4F9D
:1009E000089557FD9058440F551F59F05F3F71F01F
:1009F0004795880F97FB991F61F09F3F79F0879586
:100A00000895121613061406551FF2CF4695F1DF0E
:100A100008C0161617061806991FF1CF869571059E
:100A2000610508940895E894BB2766277727CB01D2
:100A300097F908959B01AC0160E070E080E89FE3C6
:100A400037CE72CF64C1D5DFE8F39923D9F3940F81
:100A5000511DBBF39150504094F059F0882332F06F
:100A6000660F771F881F91505040C1F79E3F510578
:100A700044F7880F911D9695879597F908955F3FE4
:100A8000ACF0983E9CF0BB27869577956795B79517
:100A900008F4B1609395C1F7BB0F58F711F460FFEC
:100AA000E8CF6F5F7F4F8F4F9F4FE3CFBDCF0AD00F
:100AB00029ED3BE54EED5EE378C00EF028C13ACF5C
:100AC000689432CF96DFC8F39923D1F3C6F3DF934E
:100AD000CF931F930F93FF92C92FDD2788232AF00E
:100AE0002197660F771F881FDAF720E030E040E893
:100AF0005FEB9FE3883920F0803E30F021968F77BE
:100B00000DDDE5E8F1E003C009DDE2EBF1E025DF12
:100B10008B01BE01EC01FB2E6F5771097595771F94
:100B2000880B990B64DE28E132E741E35FE349D0AB
:100B3000AF2D9801AE01FF900F911F91CF91DF91E2
:100B4000FEDC3ECFFA01DC01AA0FBB1F9B01AC010A
:100B5000BF5728F422273327442750781FC0B751A6
:100B600088F4AB2F0024469537952795011CA39553
:100B7000D2F3002069F0220F331F441FB395DAF33C
:100B80000DD0CBCC61307105A0E88A07B94630F4AE
:100B90009B01AC016627772788279078309621F053
:100BA000208331834283538308950BD009CFFADE2B
:100BB00028F0FFDE18F0952309F0B6CEBBCE112445
:100BC00033CF0FDFA0F3959FD1F3950F50E0551F62
:100BD000629FF001729FBB27F00DB11D639FAA2792
:100BE000F00DB11DAA1F649F6627B00DA11D661FE1
:100BF000829F2227B00DA11D621F739FB00DA11D02
:100C0000621F839FA00D611D221F749F3327A00DBB
:100C1000611D231F849F600D211D822F762F6A2F57
:100C200011249F5750408AF0E1F088234AF0EE0FDC
:100C3000FF1FBB1F661F771F881F91505040A9F7E9
:100C40009E3F510570F070CEEFCE5F3FECF3983EC3
:100C5000DCF3869577956795B795F795E7959F5F50
:100C6000C1F7FE2B880F911D9695879597F90895EA
:100C7000FA01EE0FFF1F30962105310599F161153C
:100C8000710561F48038BFE39B0749F1689490389F
:100C9000810561F08038BFEF9B0741F0992342F551
:100CA000FF3FE1053105210511F1E8940894E7952E
:100CB000D901AA2329F4AB2FBE2FF85FD0F310C0BF
:100CC000FF5F70F4A695E0F7F73950F019F0FF3A9E
:100CD00038F49F779F930CD00F9007FC905808959D
:100CE0003EF028CE60E070E080E89FE308954FE793
:100CF0009F775F934F933F932F93E4DE2F913F9124
:100D00004F915F9152DF41CD9B01AC014ECF9F3F90
:100D100031F0915020F4879577956795B795880FB6
:100D2000911D9695879597F908950E949D86332386
:100D300012F48A1B9B0B0C94AE86A29FB001B39F4A
:100D4000C001A39F700D811D1124911DB29F700DD4
:100D5000811D1124911D08950E949D86B7FF08955D
:100D6000821B930B08950E949D86A59F900DB49FB2
:100D7000900DA49F800D911D11240895B7FF0C9430
:100D8000B3860E94B386821B930B0895DB018F9379
:100D90009F930E94B386BF91AF91A29F800D911D3A
:100DA000A39F900DB29F900D11240895AA1BBB1B09
:100DB00051E107C0AA1FBB1FA617B70710F0A61B5B
:100DC000B70B881F991F5A95A9F780959095BC017C
:100DD000CD01089597FB072E16F4009407D077FDF8
:100DE00009D00E94D68607FC05D03EF490958195E7
:100DF0009F4F0895709561957F4F0895A1E21A2E37
:100E0000AA1BBB1BFD010DC0AA1FBB1FEE1FFF1FAE
:100E1000A217B307E407F50720F0A21BB30BE40BFE
:100E2000F50B661F771F881F991F1A9469F7609545
:100E30007095809590959B01AC01BD01CF010895FF
:100E4000052E97FB1EF400940E944B8857FD07D097
:100E50000E94FE8607FC03D04EF40C944B885095FC
:100E60004095309521953F4F4F4F5F4F08956894BF
:100E700001C0E894F92FF12B12F00C946B87A0E0DD
:100E8000B0E0E5E4F7E80C946988092E059422F4B3
:100E90000E945388112392F4F0E80F26FFEFE094AC
:100EA000F09400951095B094C094D094A194BF0A8A
:100EB000CF0ADF0AEF0AFF0A0F0B1F0B0E94FA8707
:100EC00007FC0E945388CDB7DEB7ECE00C94858810
:100ED000689401C0E8948F929F92CF93DF930E9411
:100EE000FA87DF91CF919F908F900895DF93CF93F2
:100EF0001F930F939A9DF02D219FF00D8B9DF00D68
:100F00008A9DE02DF10D039FF00D029FE00DF11D74
:100F10004E9DE00DF11D5E9DF00D4F9DF00D7F93F8
:100F20006F93BF92AF925F934F93D5010E949D86BE
:100F30008B01AC01D7010E949D86EB01E80FF91FE0
:100F4000D6010E94C6872F913F91D6010E949D86AF
:100F5000C60FD71FE81FF91FAF91BF910E94C68728
:100F60002F913F910E949D86C60FD71FE81FF91F42
:100F7000D6010E949D86E60FF71F9801BE01CF01A2
:100F800011240F911F91CF91DF9108950E949D86AA
:100F9000460F571FC81FD91F08F431960895E894CB
:100FA000DF93CF93FC01DB010E949D867F936F93BB
:100FB000E9019A01AC01BF93AF933F932F93DF01F7
:100FC0000E949D8626F46C1B7D0B820B930B9E0169
:100FD000EB01FC010E94C687AF91BF912F913F9119
:100FE0000E94C687BE01CF01F9012F913F91CF9199
:100FF000DF91089588249924F401E401B0E49F93DB
:10100000AA279A158B049C04ED05FE05CF05D00791
:10101000A10798F4AD2FDC2FCF2FFE2FE92D982CB0
:10102000892E982F872F762F652F542F432F322FFD
:101030002227B85031F7BF9127C01B2EBF91BB2785
:10104000220F331F441F551F661F771F881F991FCC
:10105000881C991CEE1FFF1FCC1FDD1FAA1FBB1F82
:101060008A149B04EC05FD05CE05DF05A007B1073A
:1010700048F08A189B08EC09FD09CE09DF09A00B8E
:10108000B10B21601A94E1F62EF49401AF01BE0178
:10109000CD01000C089590958095709561957F4FD6
:1010A0008F4F9F4F089560957095809590953095DE
:1010B0004095509521953F4F4F4F5F4F6F4F7F4F5A
:1010C0008F4F9F4F08952F923F924F925F926F9252
:1010D0007F928F929F92AF92BF92CF92DF92EF92C8
:1010E000FF920F931F93CF93DF93CDB7DEB7CA1B49
:1010F000DB0B0FB6F894DEBF0FBECDBF09942A8874
:10110000398848885F846E847D848C849B84AA841B
:10111000B984C884DF80EE80FD800C811B81AA81A8
:10112000B981CE0FD11D0FB6F894DEBF0FBECDBF73
:10113000ED010895EE0FFF1F0590F491E02D099445
:1011400069279627692778278727782708950F9397
:10115000083090F0982F872F762F652F542F432F2C
:10116000322F22270850F4CF220F331F441F551F60
:10117000661F771F881F991F0A95B2F70F91089570
:1011800097FB10F8169400080F93083098F0085059
:10119000232F342F452F562F672F782F892F902DEF
:1011A000F4CF0594979587957795679557954795CB
:1011B000379527950A95AAF70F9108952A0D3B1D9B
:1011C0004C1D5D1D6E1D7F1D801F911F0895002405
:1011D000A7FD00942A0F301D401D501D601D701D7D
:1011E000801D901D08952A193B094C095D096E095F
:1011F0007F09800B910B08952A153B054C055D0571
:101200006E057F058007910708950024A7FD0094CF
:101210002A173005400550056005700580059005CA
:1012200008958F929F92AF92BF92CF92DF92EF92EA
:10123000FF92CF93DF93EC01688179818A819B8152
:10124000611571058105910521F464E279ED8BE565
:1012500097E02DE133EF41E050E00E942087490103
:101260005A019B01AC01A7EAB1E40E94B3866B016D
:101270007C01ACEEB4EFA50194010E94C186C60EBC
:10128000D71EE81EF91EF7FE06C081E0C81AD10875
:10129000E10880E8F80AC882D982EA82FB82C601A6
:1012A0009F77DF91CF91FF90EF90DF90CF90BF902D
:1012B000AF909F908F9008950C9411898CED92E0DF
:1012C0000C941189A0E0B0E08093DC029093DD02E1
:1012D000A093DE02B093DF0208952F923F925F92B7
:1012E0006F927F928F929F92AF92BF92CF92DF9236
:1012F000EF92FF920F931F93CF93DF938B01EA013D
:101300006115710521F0DB018C9311969C93209758
:1013100039F09E01225031092332310508F0FBC01B
:101320007C016701BFEFCB1ADB0A5601F701608031
:10133000862D90E00E94AF8C892B11F07601F1CFC1
:10134000FDE26F120AC0570182E0A80EB11CD7015E
:1013500011966C90772473940BC0BBE26B1207C09C
:101360005701E2E0AE0EB11CD70111966C90712CC2
:10137000CE018F7E892B89F4B0E36B1222C0F50178
:1013800080818F7D883541F56180F2E0AF0EB11C20
:10139000872D8260782EC0E1D0E0C830D105F1F011
:1013A0004CF4C230D10511F5C12CD12CE12CB0E4A4
:1013B000FB2E2FC0CA30D10531F0C031D10521F14B
:1013C00015C0209751F7CAE0D0E0ACECCA2EDC2C57
:1013D000EC2CACE0FA2E1DC02097F9F6C8E0D0E066
:1013E000C12CD12CE12CF0E1FF2E13C060E070E0A5
:1013F00080E090E89E01442737FD4095542F0E94DD
:10140000FE8669017A0105C0C12CD12CE12CE8E0EF
:10141000FE2EF50160E020E030E0A9014E01AA2493
:1014200097FCA094BA2C1F0170ED572E560CA9E022
:10143000A51570F48FEB860D8A3118F499EC592EAE
:1014400006C08FE9860D8A3130F589EA582E560C90
:10145000852D90E08C179D07F4F467FD18C0C21627
:10146000D306E406F50680F0C501B4010E94C686E5
:101470009B01AC01250D311D411D511D2130310550
:101480004105B0E85B0710F06FEF01C061E03196F5
:10149000D1016C90C8CF872D81700115110571F0B5
:1014A000662329F03197D801ED93FC9307C071FEB4
:1014B00019C03297D801ED93FC9314C067FF12C096
:1014C000882329F020E030E040E050E804C02FEF0E
:1014D0003FEF4FEF5FE782E290E090931631809309
:1014E000153116C0882341F05095409530952195CF
:1014F0003F4F4F4F5F4F0CC057FF0AC082E290E052
:1015000090931631809315312FEF3FEF4FEF5FE748
:10151000B901CA0104C060E070E080E090E0DF91B2
:10152000CF911F910F91FF90EF90DF90CF90BF90E0
:10153000AF909F908F907F906F905F903F902F9093
:1015400008952F923F925F926F927F928F929F9217
:10155000AF92BF92CF92DF92EF92FF920F931F93C1
:10156000CF93DF938B01EA016115710521F0DB0157
:101570008C9311969C93209739F09E01225031094B
:101580002332310508F0D8C07C016701BFEFCB1AC8
:10159000DB0A5601F7016080862D90E00E94AF8C37
:1015A000892B11F07601F1CFFDE26F120AC05701CD
:1015B00082E0A80EB11CD70111966C907724739429
:1015C0000BC0BBE26B1207C05701E2E0AE0EB11CCC
:1015D000D70111966C90712CCE018F7E892B89F4E6
:1015E000B0E36B1237C0F50180818F7D8835D1F46F
:1015F0006180F2E0AF0EB11C872D8260782EC0E1D1
:10160000D0E0CA30D10551F1C031D10521F0C83048
:10161000D10599F409C0CC24CA94DC2CEC2CAFE0A1
:10162000FA2E22C0209769F7C8E0D0E0CC24CA94F3
:10163000DC2CEC2CFFE1FF2E17C06FEF7FEFCB010E
:101640009E01442737FD4095542F0E94FE86690174
:101650007A010AC02097A9F6CAE0D0E0E9E9CE2EC7
:10166000DC2CEC2CE9E1FE2EF50160E020E030E01E
:10167000A9014E01AA2497FCA094BA2C1F0170ED79
:10168000572E560CA9E0A51570F48FEB860D8A3104
:1016900018F499EC592E06C08FE9860D8A3148F569
:1016A00089EA582E560C852D90E08C179D070CF575
:1016B0006F3FD9F0C216D306E406F50698F0C501CF
:1016C000B4010E94C6869B01AC01852D90E0A0E08C
:1016D000B0E0280F391F4A1F5B1F281739074A0738
:1016E0005B0710F46FEF01C061E03196D1016C909F
:1016F000C5CF0115110551F0662311F0319703C0D4
:1017000071FE04C03297D801ED93FC9370FE07C0C0
:1017100050954095309521953F4F4F4F5F4F67FF54
:1017200010C082E290E090931631809315316FEFF4
:101730007FEF8FEF9FEF07C060E070E080E090E008
:1017400002C0B901CA01DF91CF911F910F91FF90A3
:10175000EF90DF90CF90BF90AF909F908F907F9051
:101760006F905F903F902F900895662777270C9495
:10177000258FFC0188279927E89421912032E9F3ED
:10178000293010F02E30C8F32B3241F02D3239F4CD
:10179000689404C00E944A8D820F911D21912053AC
:1017A0002A30C0F31EF4909581959F4F08952830FC
:1017B00008F027E03327DA01990F311D87FD91608A
:1017C00000966105710539F432602E5F3D9330E378
:1017D0002A95E1F708959F3F30F080387105610543
:1017E00009F03C5F3C5F3D93913008F08068911DAB
:1017F000DF93CF931F930F93FF92EF92192F987F50
:101800009695E92F96959695E90FFF27E455FF4E9B
:1018100099273327EE24FF24A701E70105900894B8
:10182000079428F4360FE71EF81E491F511D660F56
:10183000771F881F991F0694A1F70590079428F435
:10184000E70EF81E491F561FC11D770F881F991FED
:10185000661F0694A1F70590079428F4F80E491F17
:10186000561FC71FD11D880F991F661F771F06942B
:10187000A1F70590079420F4490F561FC71FD81FE2
:10188000990F661F771F881F0694A9F784911095FA
:10189000177041F0D695C79557954795F794E794FB
:1018A0001A95C1F7E2E5F0E168941590159135912C
:1018B0006591959105907FE27395E118F10A430BCC
:1018C000560BC90BD009C0F7E10CF11E431F561F80
:1018D000C91FD01D7EF4703311F48A95E6CFE894C9
:1018E000015030F0080F0AF40027021708F4202FE7
:1018F0002395022F7A3328F079E37D932A95E9F72F
:1019000010C07D932A9589F606949795679537952B
:1019100017951794E118F10A430B560BC90BD00920
:1019200098F023957E9173957A3308F070E37C9359
:101930002013B8F77E9170617D9330F0839571E349
:101940007D9370E32A95E1F71124EF90FF900F91BA
:101950001F91CF91DF91992787FD9095089591115F
:10196000F1C3803219F089508550D0F70895FB01FA
:10197000DC018D91059080190110D9F3990B089520
:10198000FC010590615070400110D8F7809590954A
:101990008E0F9F1F08954EE95AE10C94238DFB0191
:1019A000DC0102C001900D9241505040D8F70895DB
:1019B000DC0101C06D9341505040E0F70895FB01F8
:1019C000DC018D91019080190110D9F3990B0895D4
:1019D000FB01DC0101900D920020E1F70895FB016D
:1019E000DC014150504048F001900D920020C9F7B1
:1019F00001C01D9241505040E0F70895FC01615034
:101A0000704001900110D8F7809590958E0F9F1F20
:101A10000895FB0151915523A9F0BF01DC014D91BF
:101A200045174111E1F759F4CD010190002049F02B
:101A30004D9140154111C9F3FB014111EFCF81E0F8
:101A400090E001970895FA01A191B081009719F4EF
:101A50001097E1F0CD01DC01CD010D90002011F4D3
:101A6000C00113C0FB012191222319F02015D9F7E1
:101A7000F3CFFB012191201519F41E92119606C097
:101A80002223C1F70D900020A1F7D001FA01A19304
:101A9000B08308957AE0979F902D879F802D910DB8
:101AA000112408950F931F93CF93DF93182F092FBD
:101AB000EB018B8181FD03C08FEF9FEF20C082FF80
:101AC00010C04E815F812C813D81421753077CF409
:101AD000E881F9819F012F5F3F4F3983288310836D
:101AE00006C0E885F985812F0995892B29F72E8174
:101AF0003F812F5F3F4F3F832E83812F902FDF91B8
:101B0000CF911F910F910895CF93DF93CDB7DEB79B
:101B1000FE01359661917191AF01809111319091E3
:101B200012310E94E97EDF91CF9108950F931F93A8
:101B3000CF93DF93CDB7DEB7FE01379661917191F8
:101B400001E111E3D8018D919C91DC0113962C9158
:101B50001397286013962C93AF010E94E97ED80159
:101B6000ED91FC912381277F2383DF91CF911F91FA
:101B70000F9108950F931F93CF93DF93E09111314D
:101B8000F0911231238121FF1BC0EC0100E010E035
:101B900089916091113170911231DB011896ED91AC
:101BA000FC911997882331F00995892B89F30FEF60
:101BB0001FEFEECF8AE00995892B11F4C80102C00E
:101BC0008FEF9FEFDF91CF911F910F9108950F93AA
:101BD0001F93CF93DF93CDB7DEB72E970FB6F89450
:101BE000DEBF0FBECDBF0D891E898F89988D26E07F
:101BF0002C831A83098397FF02C080E090E8019745
:101C00009E838D83AE01455E5F4F698D7A8DCE01D7
